:100000000C9464100C948C100C948C100C948C1028
:100010000C948C100C948C100C948C100C948C10F0
:100020000C948C100C948C100C9490160C94F66A12
:100030000C94386F0C94456B0C948C100C9419171D
:100040000C947E160C948C100C9434760C942574BD
:100050000C948C100C948C100C948C100C948C10B0
:100060000C94BB6F0C945F170C94AA6B0C940570E6
:100070000C948C100C948C100C94CD690C948C10F6
:100080000C948C100C948C100C948C10F518F9189E
:10009000BE18C418CA18CA18CA18ED18F118F518ED
:1000A000F91806190619FD186123612361236123DC
:1000B0008E238523852385238523852385238523F7
:1000C000712376237623062F102F262F732FB22F1E
:1000D00010301B301E3078307C30BC33D1336D345F
:1000E000F6357F36FD34B839FD370037083790379D
:1000F000FF38F742CA42CD42D142D742DB42E0420A
:100100007C4B8B4B964BAC4BB34BBA4BC94BE04B38
:10011000F84B644C8F4C974C9F4CAB4CD04CE04C04
:100120000A4D574D634D9E4DB64DC74DD34DDF4DD6
:10013000EB4D1151DD5BE45311596454DD5BDD5B24
:10014000E157775ADD5BDD5B2753215168554768DE
:100150003668306838683C684068336844684A6884
:10016000226E256E3C6E576E576E3C6E3C6E36713D
:1001700038713B714071517160716E717871887125
:1001800098719D71B371B671BA71BC71BE71C37152
:10019000C771D271D671DE71E571E971EB71EF71E2
:1001A000F171F371F571F971FD71027207720C72E0
:1001B00011721672204F6C642056657273696F6EEF
:1001C00020454550524F4D202020434845434B2069
:1001D00053455454494E47532F43414C49420041E3
:1001E0006C61726D732044697361626C6564004573
:1001F0004550524F4D206C6F77206D656D004C4F10
:100200004144494E47000553746F70706564006D3A
:10021000537461636B206F666C6F770053776974FA
:100220006368205761726E696E671F506C656173F9
:1002300065205265736574205377697463686573CC
:10024000005468726F74746C65206E6F74206964FA
:100250006C651F5265736574207468726F74746C7A
:1002600065004D45535341474500707265737320D7
:10027000616E79204B657900507265737320616EF1
:1002800079206B657920746F20736B6970004F461D
:10029000464F4E20544873544825002D2D2D002DD7
:1002A0002D2D2D0000006428100703010000000020
:1002B000010101020202020101030020414C4552EA
:1002C00054000001020300020103030102000302C3
:1002D00001000452756420456C6520546872204109
:1002E000696C20004F4E20004F4646000354485290
:1002F000525544454C4549443049443149443241C2
:10030000494C47454154524E4C31204C32204C33DD
:10031000204C34204C35204C36204C37204C382093
:100320004C39204C41204C42204C4320454C8045C8
:100330004C2D454C8152558052552D525581414985
:100340008041492D41498147458047452D47458199
:10035000504231504232001B1E272D36394B4E631E
:100360006C7278878D939CB1B4C6C9D2D8E1E4533E
:10037000706C6173680080400000000000000000A5
:10038000000000000000000000000000000000006D
:10039000000000000000000000000000000000005D
:1003A000000000000000000000000000000000004D
:1003B000000000000000000000000000000000003D
:1003C00000000080C0E0E0F0F8F8FCFCFCF8F8F871
:1003D000F04000000000008080800000000000006D
:1003E0000000000000000000000000000080C0C00D
:1003F000E0E0E0F0F0F0E0C00000000000C0F8FF36
:10040000FF9F878383838383838383838383838320
:10041000838383838383838383038380838383832F
:10042000838383838383838383838383838383839C
:10043000838383C3E3733F1F0000000080E0F0F874
:10044000FCFEFFFFFFFF7F3F1F1F0F0783C3E1E19C
:10045000E0E0C0000E1F3F7F7FFFF3E0E080000080
:10046000000000000000000080F0FCFEFFFFFFFF26
:100470007F3F0F0301010100000080F0FEFFFFC776
:10048000C1C1C1C1C1C1C1C1C1C1C1C1C1C1C1C15C
:10049000C1C1C1C1C1C101C1F0FEFF3F0F070F0DB6
:1004A0000D0D1D191919193131313171616161E178
:1004B000C1C1C18100000080E0F8FCFFFFFFFF2FF9
:1004C000170F038180C0E0F0F8FCFEFFFFFFFFFF85
:1004D000FF7F010000000000000001010307070E7C
:1004E0001E1C3870E0F0F8FEFFFF7F1F0F030001B5
:1004F00000000000000000000000000000000000FC
:1005000000000000000000000000000000000000EB
:1005100000000000000000000000000000000000DB
:1005200000000000000000000000000000000000CB
:100530000000000000007EFFFFFFFFFFFFFBF8FC54
:10054000FCFEFF7F3F1F0F07C3FFFFFFFFFFFF7F83
:10055000070000000000000000000000000000C0D4
:10056000E0F8FEFFFF7F1F0F1F3D7CF8F8F0E080F2
:10057000000000000000000000000000000000007B
:10058000000000000000000000000000000000006B
:10059000000000000000000000000000000000005B
:1005A000000000000000000000000000000000004B
:1005B0000000000000000000010101010103070725
:1005C000070301000000E0FCFFFFFFFFFF1F030027
:1005D00000000000000000000000C0F078DE2713DB
:1005E000090E0703000000000000000001030F7F58
:1005F000FFFC7878F8000000000000000000000018
:10060000808080808080808080008080008080006A
:1006100000000000000080808080808080808080DA
:1006200080808080808080800000000000000000CA
:1006300000000000000000000000000000000000BA
:1006400000000080F0FEFFFFFFFF3F0F01000000F1
:100650000000000000C0E0381E0F03000100000091
:10066000000000000000000000000000000000008A
:100670000000000303010000000000000000000073
:100680000E0E02020202020303000F0F000F0F08FA
:100690000808080808080F0F08080808080F0F00C6
:1006A0000000000F0F00000000000000000000002C
:1006B000000000000000000000000000000000003A
:1006C00000C0F8BFFFFFFF1F7F0100000000000017
:1006D0000000F0FCFF7F7830000000000000000008
:1006E000000000000000000000000000000000000A
:1006F00000000000000000000000000000000000FA
:1007000000000000000000000000000000000000E9
:1007100000000000000000000000000000000000D9
:1007200000000000000000000000000000000000C9
:100730000000000000000000000000000000003089
:100740001C070E0F07010000000000000000000061
:100750000000000000000000000000000000000099
:100760000000000000000000000000000000000089
:10077000000000000000000000564552533A205689
:10078000312E312D1F444154453A2033302E313221
:100790002E323031351F54494D453A2031303A35EB
:1007A000323A31331F2053564E3A20657239782D34
:1007B000723831391F204D4F443A204652534B591D
:1007C000204E5420202020003C06064F4E202020A2
:1007D000204F4646202020424F5448202031355398
:1007E0006563733330536563733630536563735693
:1007F000617269626C0056530007203820536563AC
:10080000733132205365637331362053656373004F
:100810001E030153415658004E756D626572205695
:100820006F6963652053770053616665747920535F
:100830007769746368657300434F50592054524977
:100840004D205B4D454E555D000D4F6E004C4F47A2
:100850004943414C205357495443484553003C01B8
:100860000A436F756E7420446F776E436F756E74B4
:1008700020557020200054696D65721F547269679D
:10088000676572411F54726967676572421F5469D8
:100890006D65721F52657365742053776974636860
:1008A0000020547970651F20436F756E7472791F34
:1008B00042696E641F52616E6765003C02094C50CC
:1008C000342F4C5035202044534D326F6E6C7920BC
:1008D00044534D322F44534D580044534D205479C6
:1008E000706500014E59000B4F7074696F6E000403
:1008F000486967684C6F7720003C00044E6F6E6556
:10090000003C010543473032335944383239003C0A
:100910000205475245454E424C554520444D303026
:1009200037003C020753594D4158202053594D413F
:10093000583543003C040759443731372020534B86
:1009400059574C4B5253594D4158322058494E58E3
:10095000554E204E494855492020003C010444533F
:100960004D3244534D58003C01054869736B79483A
:100970004B333130003C0306466C79736B79563942
:1009800078392020563678362020563931322020CA
:10099000003C0D06466C79736B7948756273616E25
:1009A0004672736B79204869736B792056327832BE
:1009B000202044534D3220204465766F2020594436
:1009C000373137204B4E2020202053796D6158203D
:1009D000534C54202020435831302020434730329C
:1009E0003320426179616E670050726F746F636F7C
:1009F0006C1F547970651F506F7765721F42696E66
:100A00006420202020204175746F62696E641F523B
:100A1000616E676500660103504F534E45470050B5
:100A20006F6C61726974790050504D2046724C654C
:100A30006E0D6D536563000C52784E756D00043475
:100A4000434820364348203843482031304348311A
:100A5000324348313443483136434800137553001C
:100A60000650504D20202050585820202044534DEF
:100A700032202050504D31362050504D53494D4D6D
:100A8000554C544920534255532020003173742053
:100A90004368616E1F50726F746F000444521F02EE
:100AA0004578706F1F1F015765696768741F1F4481
:100AB000725377311F447253773200034869204DD7
:100AC0006964204C6F77006604042D2D2D2D313282
:100AD000302031323058313430203930202000532A
:100AE0007761736820547970651F436F6C6C656320
:100AF000746976651F53776173682052696E671F4A
:100B0000454C4520446972656374696F6E1F4149A5
:100B10004C20446972656374696F6E1F434F4C20AB
:100B2000446972656374696F6E0052455441313295
:100B30003300540406457870202020457846696EBD
:100B40006546696E6520204D656469756D436F610A
:100B5000727365005472696D20496E631F54726927
:100B60006D2053771F48692E52657320536C6F7741
:100B70002F44656C61791F547261696E65721F4202
:100B800065657020436E74005A01062020456E642E
:100B90002043656E74726500452E204C696D697442
:100BA000731F5468722E2044656661756C741F54FF
:100BB00068726F74746C6520726576657273651FF8
:100BC0005468726F74746C65204F70656E1F542D7D
:100BD0005472696D1F542D4578706F2D44720066F4
:100BE00007032D2D2D5031205032205033204756F1
:100BF0003447563547563647563700446566617563
:100C00006C742053771F437573746F6D53746B4E00
:100C1000616D65731F4175746F204C696D697473E4
:100C20001F566F6C756D6520436F6E74726F6C002C
:100C3000566F69636520496E646578114D454E5560
:100C400000881341154C15391533152C157D1321CA
:100C50001516157713C016D1130D15564100566F92
:100C6000696365004D454E55204C4F4E4700446525
:100C70006C65746500566F6963652046696C650034
:100C80005402062D2D2D2D2D2D4E756D6265722071
:100C9000417564696F00660104506C61794D75742B
:100CA00065005402064E6F202020204265666F7258
:100CB00065416674657220004E03072D2D2D2D2D84
:100CC0002D2D4861707469633148617074696332B5
:100CD00048617074696333000776603D76616C200B
:100CE000763D76616C20200007280D2900506C614C
:100CF0007920536F757263651F4F6E206E6F20549D
:100D0000656C656D657472791F46696C65547970A0
:100D10006500536F757263651F46756E6374696F06
:100D20006E1F56616C75651F5377697463681F5237
:100D30006174651F48617074696300566F6963650B
:100D400020416C61726D00034D4F5645205354494C
:100D5000434B532F504F54530005534554204D4996
:100D600044504F494E5400035B4D454E555D205451
:100D70004F205354415254006607044E4F4E454590
:100D80005854314558543250433020504732205047
:100D9000423720504735204C2D575200454C4520B6
:100DA0007377697463681F41494C20737769746372
:100DB000681F504231207377697463681F50423254
:100DC000207377697463681F50473220496E7075CD
:100DD000741F50423720496E7075741F4C2D575246
:100DE00020496E7075740042616E64476170004303
:100DF000616C004D756C7469706C696572001802E5
:100E0000036F6666202B3D203A3D00036D6F6465DD
:100E10000A2520737263202073770007536C617674
:100E2000650012424700414E41000F504232000F10
:100E3000504231005472696D2D202B00204C6566A4
:100E4000741F52696768741F0355701F20446F77C1
:100E50006E1F20457869741F204D656E75004449EA
:100E6000414700537469636B5363726F6C6C00503D
:100E70006F745363726F6C6C0053706C6173682095
:100E80004E616D650053706C6173682073637265A9
:100E9000656E00416C61726D205761726E696E679C
:100EA000004D656D6F7279205761726E696E6700D3
:100EB0005468726F74746C65205761726E696E67E6
:100EC0000042617474657279207761726E696E6731
:100ED0001F496E616374697669747920616C61720F
:100EE0006D136D0043726F73735472696D1F546894
:100EF000726F74746C6520726576657273651F45D8
:100F00006E61626C652050504D53494D1F436861BE
:100F10006E6E656C204F726465721F4D6F64650064
:100F20002048617074696320537472656E677468D9
:100F30000042040A426565706572202020205069D5
:100F400053706B72202020204265657072566F6965
:100F50006365506953706B566F6963654D65676172
:100F6000536F756E642000540606517569657420D0
:100F70004E6F4B6579207853686F727453686F7247
:100F800074204E6F726D20204C6F6E672020784C5D
:100F90006F6E672000566F6C756D651F42656570DA
:100FA00065721F536F756E64204D6F64651F20530B
:100FB0007065616B6572205069746368004C696785
:100FC0006874207377697463681F4261636B6C692E
:100FD00067687420696E766572741F4C69676874FF
:100FE000206F66662061667465721F4C696768745D
:100FF000206F6E2053746B204D761F466C617368B2
:10100000206F6E206265657000436F6E747261734D
:101010007400E913A013C113D113B813AC13E11377
:10102000D91396138E13C81322047C5E54546D009A
:1010300003457870457846466E654D656443727326
:101040000011544F541F01544D45115453571F0163
:1010500053544B1153542500035B4D454E555D20B1
:10106000746F207265667265736800746D72314CBE
:101070006174206D61781275731F746D72314C61EB
:1010800074206D696E1275731F746D7231204A6918
:10109000747465721275731F746D61696E126D736D
:1010A0000053544154000966726565004D4F444534
:1010B0004C53454C0020464D300A524554410042A5
:1010C00041434B555020444F4E45004241434B5500
:1010D0005000524553544F52454400534156494ED7
:1010E0004700524553544F52494E47004C4F4144DC
:1010F000494E4700526573746F7265004261636BBD
:1011000075700020464D005377697463681F5472F0
:10111000696D731F4661646520496E1F4661646591
:10112000204F757400464C204D4F44450052414EAF
:10113000474520434845434B20525353493A000604
:1011400042494E44494E47004475706C696361746E
:10115000696E67206D6F64656C0044454C4554456D
:10116000204D4F44454C004455504C494341544553
:10117000204D4F44454C00012B2A52004D49584503
:10118000520020202020202020202020202020204D
:101190000044454C455445204D49583F00436C653B
:1011A000617220414C4C206D697865733F00035992
:1011B00045530B4E4F1F035B4D454E555D0B5B4535
:1011C0005849545D004D6178206D697865727320CF
:1011D00072656163683A2033321F1F507265737302
:1011E000205B455849545D20746F2061626F7274B2
:1011F000006601034F46464F4E20004E02084164F0
:101200006420202020204D756C7469706C795265C3
:10121000706C6163652000437572766500084469EF
:10122000666600114578706F0001557365204F7533
:10123000747075742020200001536F757263651FF0
:10124000015765696768741F014F66667365741F8F
:1012500001466978204F66667365741F01456E61AB
:10126000626C654578706F44521F015472696D1F3E
:101270001F1F015377697463681F014D4F44455325
:101280001F015761726E696E671F014D756C747036
:10129000781F0144656C617920446F776E1F0144AB
:1012A000656C61792055701F01536C6F7720204465
:1012B0006F776E1F01536C6F772020557000454487
:1012C0004954204D495820004F50005343092B0DDD
:1012D0002A122F00044C314C324C334C344C354CD8
:1012E000364C374C384C394C414C424C4300480149
:1012F0000546697273744C6173742000536F757284
:1013000063651F1F4F66667365741F4D756C746946
:10131000706C6965721F44697669736F721F556ED0
:1013200069741F5369676E1F446563696D616C73EF
:101330001F4F6666736574204174005B2D3E5D002F
:1013400043560050524553455400435552564500AC
:101350006A01032D2D2D494E560053575220003C53
:1013600002034431364438204C52503C0203416D54
:10137000654A6170457572566F696365004C2E53FE
:1013800077697463686573004D69786572004469B4
:101390006167416E610044696167537774636800F7
:1013A000417564696F4861707469630043616C6979
:1013B00062726174696F6E00436F6E74726F6C73EA
:1013C00000416C61726D730048617264776172658F
:1013D0000047656E6572616C0056657273696F6E69
:1013E00000547261696E657200446973706C617952
:1013F000005B4D454E555D205748454E20444F4EAD
:101400004500454449540053454C45435400534519
:101410004C2F4544495400434F5059004D4F5645B9
:101420000044454C455445004241434B5550005201
:101430004553544F5245004544495400494E534585
:10144000525400434F5059004D4F56450044454CAF
:1014500045544500434C45415220414C4C000473D7
:10146000494478735448527352554473454C4573FC
:1014700041494C734745417354524E0012081200C3
:10148000081C0808081C080000082200490022085F
:101490000000000000227F22000000082200490016
:1014A0002208000008220049002208000000227FD4
:1014B0002200000000000822004900220800000865
:1014C0001C0808081C0800534300475600054665E1
:1014D000657420566F6C74734465675F4344656739
:1014E0005F466D41682020416D7073204D657472B8
:1014F00065576174747300465643466D416D5718C5
:10150000242F2F0033383B01524554410050726F55
:10151000746F636F6C00476C6F62616C56617273BD
:101520000053616665747920537773004375727652
:101530006573004D6F646573004578706F2F44725A
:101540000048656C69205365747570004C696D695D
:101550007473004D6F64656C2053656C6563740033
:101560004D6F64656C205365747570004C617374C5
:10157000204D656E7500526164696F205365747506
:1015800070005374617469737469637300426565B4
:101590007020636F756E74646F776E004D696E7541
:1015A0007465206265657000032D2D2D52746D45A4
:1015B000746D54746D41746D52454E527564456C32
:1015C0006554687241696C5031205032205033208C
:1015D000000420204F4E204F4646424F54482041A1
:1015E0004C4C4F4E434500072D2D2D2D20202076AD
:1015F0003E76616C2020763C76616C20207C767C87
:101600003E76616C7C767C3C76616C414E44202059
:1016100020204F522020202020584F5220202020D0
:1016200076313D3D7632207631213D76322076315D
:101630003E7632202076313C763220204C61746335
:10164000682020462D466C6F702054696D654F668A
:101650006676603D76616C20004E616D65000657D0
:1016600061726E31205761726E3220436865657019
:101670002052696E672020536369466920526F6269
:101680006F74204368697270205461646120204344
:101690007269636B74536972656E20416C6D436C43
:1016A0006B5261746174615469636B20204861708E
:1016B00074633148617074633248617074633300DD
:1016C00054696D65720054524530313241474700CC
:1016D0000354783D537772002041424344454647C6
:1016E00048494A4B4C4D4E4F505152535455565702
:1016F00058595A6162636465666768696A6B6C6DA4
:101700006E6F707172737475767778797A30313262
:10171000333435363738395F2D2E00FEFFFDF6F7AE
:10172000F8F9FAFBFC042D2D2D2D54494D31544967
:101730004D32424154544776723147767232477681
:10174000723347767234477672354776723647760B
:10175000723700032D2D2D783E30783C307C787C1C
:10176000663E30663C307C667C63312063322063A9
:101770003320633420633520633620633720633899
:101780002063392063313063313163313263313367
:1017900063313463313563313600045031202050D9
:1017A0003220205033202048414C4646554C4C4373
:1017B000594331435943324359433350504D3150CB
:1017C000504D3250504D3350504D3450504D355097
:1017D000504D3650504D3750504D384348312043CE
:1017E000483220434833204348342043483520437F
:1017F000483620434837204348382043483920435F
:101800004831304348313143483132434831334322
:1018100048313443483135434831365357434847BC
:1018200056312047563220475633204756342047FA
:1018300056352047563620475637205448495300DE
:10184000537769746368205761726E696E670067C9
:10185000656E7772697465206572726F72004545B6
:1018600050524F4D20466F726D617474696E6700FF
:1018700042616420454570726F6D2044617461005F
:10188000434845434B204D4F44454C2054494D451A
:10189000525300434845434B204D49582F44522052
:1018A000534F5552434553004D4F44454C20202043
:1018B0002020004D452020202020202020004545CC
:1018C00050524F4D206F766572666C6F7700E2AEB6
:1018D000A1A6A4A2C02F25AF0000000000000000B8
:1018E0000000000000000000000000000000000BED
:1018F00007000000C0C0C0C0C0C0C00000000000A1
:1019000000000000000000000000000006060000CB
:10191000000080E0781E06181E0701000000F8FC99
:101920008EC66EFCF8070F1D181C0F07080CFEFE74
:1019300000000018181F1F1818000C0E86C6EE7C39
:10194000381E1F1B1918181806C6C6C6EEFC381814
:101950001818181D0F07C0E0B0988CFEFE01010199
:1019600001011F1F7E7E6666E6C686060C18181CDF
:101970000F07F8FCE666E6CC88070F1C181C0F075B
:10198000060606C6E67E1E001C1F0300000038FC8B
:10199000EEC6EEFC38070F1D181D0F0778FCCE862B
:1019A000CEFCF8040C1D191D0F070000003030009C
:1019B0000000000003030000E0F89C869CF8E01F94
:1019C0001F0101011F1FFEFEC6C6EEFC381F1F18B7
:1019D000181D0F07F8FC0E060E0C08070F1C181C2C
:1019E0000C04FEFE060E1CF8F01F1F181C0E070349
:1019F000FEFEC6C6C606061F1F1818181818FEFEDB
:101A0000C6C6C606061F1F0000000000F8FC0E0632
:101A1000CECCC8070F1C18181F0FFEFEC0C0C0FE9A
:101A2000FE1F1F0000001F1F0606FEFE0606001810
:101A3000181F1F18180000060606FEFE060E1E18C8
:101A4000181F0F00FEFEF0381C0E061F1F03070EA6
:101A50001C18FEFE00000000001F1F1818181818A0
:101A6000FEFC187018FCFE1F1F0000001F1FFEFC6C
:101A700070C080FEFE1F1F0000030F1FF8FC0E0643
:101A80000EFCF8070F1C181C0F07FEFEC6C6EE7CE6
:101A9000381F1F0000000000F8FC0E060EFCF807BF
:101AA0000F1C1B1E0F1BFEFE86C6EE7C381F1F037D
:101AB000070E1C18387CEEC6C68E0C0C1C18181DA0
:101AC0000F070606FEFE06060000001F1F000000AE
:101AD000FEFE000000FEFE070F1C181C0F07FEFE96
:101AE000000000FEFE01070E180E0701FEFE00803A
:101AF00000FEFE1F0F0603060F1F1E3EF0E0F03E25
:101B00001E1E1F0301031F1E7EFEC0C0FE7E0000BE
:101B1000001F1F0000000686C6E6F67E3E1F1F1B44
:101B200019181818000000000000001818181818DC
:101B300018180060606060E0C0060F1F1B1B1F1FAD
:101B4000FEFEE060E0C0801F1F1C181C0F07C0E0F5
:101B5000E06060E0C00F1F1C18181C0C80C0E06023
:101B6000E0FEFE070F1C181C1F1FC0E0606060E055
:101B7000C00F1F1B1B1B1B01C0F8FCCEC60E0C00A8
:101B80001F1F00000000C0E0703070E0C003C7CE2F
:101B9000CCEE7F3FFEFEC0E0E0C0801F1F010000D2
:101BA0001F1F000060E6E600000000181F1F18005D
:101BB00000000000E3E300307060607F3F00FEFE45
:101BC000C0E07038181F1F03070E1C18000006FE27
:101BD000FE00000000181F1F1800E0E060C060E079
:101BE000C01F1F0001001F1FE0E0C0E0E0C0801F19
:101BF0001F0100001F1F80C0E060E0C080070F1CB5
:101C0000181C0F07E0F0703070F0E0FFFF0E0C0EB4
:101C10000F07E0F0703070F0E0070F0E0C0EFFFFC2
:101C2000E0E0C06060E0E01F1F0000000000C0E0D6
:101C30006060606060191B1B1B1B1F0E6060FEFE56
:101C400060600000000F1F181C0CE0E0000000E0C6
:101C5000E0070F1C1C0E1F1FE0E0000000E0E00189
:101C6000070E180E0701E0E0000000E0E00F1F186B
:101C70000E181F0F60E0800080E060181C0703074B
:101C80001C18E0E0000000E0E007CFCECCEC7F3F86
:101C90006060606060E0E01C1E1E1B1B19190000E4
:101CA0000000000000006F000007000700147F1410
:101CB0007F14242A7F2A122313086462364955228E
:101CC000500005030000001C2241000041221C00BE
:101CD00014083E081408083E0808005030000008A8
:101CE0000808080800606000002010080402003E98
:101CF00049453E0000427F4000625149460041494B
:101D00004936001814127F0027454539003E4949DD
:101D10003200017905030036494936000649291E7B
:101D20000000363600000056360000081422411428
:101D3000141414144122140800020151090600066B
:101D40000909067E0909097E7F494949363E414114
:101D500041227F4141221C7F494949417F090909AC
:101D6000013E4149497A7F0808087F00417F4100D0
:101D70002040413F017F081422417F404040407F86
:101D8000020C027F7F0408107F3E4141413E7F09E3
:101D90000909063E4151215E7F0919294626494914
:101DA000493201017F01013F4040403F1F20402058
:101DB0001F3F4030403F6314081463070870080752
:101DC0006151494543007F41410002040810200051
:101DD00041417F00040201020440404040400804A9
:101DE00008100820545454787F48444438384444F8
:101DF0004420384444487F3854545418087E09011C
:101E0000020C5252523E7F0804047800447D400088
:101E10002040443D007F1028440000417F40007C6A
:101E2000041804787C0804047838444444387C144A
:101E3000141408081414187C7C080404084854542A
:101E40005420043F4440203C4040207C1C20402043
:101E50001C3C4020403C44281028440C5050503C2E
:101E60004464544C44000836410000007F000000E8
:101E7000413608000808221C08081C220808040231
:101E80007F020410207F20100102040810204080EF
:101E900040800804201002010000891112239B32A7
:101EA0002446AD573665BF74488CC19D5AAFD3BE2A
:101EB0006CCAE5DB7EE9F7F88110080193331A223A
:101EC000A5562C47B7753E64C99C408DDBBF52AE0A
:101ED000EDDA64CBFFF976E802218B30100299131A
:101EE0002667AF763444BD554AADC3BC588ED19FEA
:101EF0006EEBE7FA7CC8F5D983310A2091121803FA
:101F0000A7772E66B5543C45CBBD42ACD99E508FC9
:101F1000EFFB66EAFDD874C904428D5316619F70C9
:101F20002004A9153227BB364CCEC5DF5EEDD7FCA9
:101F30006888E1997AABF3BA85520C4397711E60B9
:101F4000A1142805B3373A26CDDE44CFDFFD56EC89
:101F5000E9986089FBBB72AA06638F7214409D5199
:101F60002225AB343006B9174EEFC7FE5CCCD5DD69
:101F70006AA9E3B8788AF19B87730E6295501C4179
:101F8000A3352A24B1163807CFFF46EEDDDC54CD49
:101F9000EBB962A8F99A708B088481951AA793B659
:101FA0002CC2A5D33EE1B7F04008C919522BDB3A49
:101FB000644EED5F766DFF7C899400859BB712A619
:101FC000ADD224C3BFF136E0C1184809D33B5A2A29
:101FD000E55E6C4FF77D7E6C0AA583B418869197F9
:101FE0002EE3A7F23CC0B5D14229CB38500AD91B09
:101FF000666FEF7E744CFD5D8BB502A499961087D9
:10200000AFF326E2BDD034C1C3394A28D11A580BE8
:10201000E77F6E6EF55C7C4D0CC685D71EE597F4A8
:102020002880A1913AA3B3B2444ACD5B5669DF78C8
:10203000600CE91D722FFB3E8DD604C79FF516E498
:10204000A9902081BBB332A2C55A4C4BD7795E68A8
:10205000E11C680DF33F7A2E0EE787F61CC495D578
:102060002AA1A3B03882B193466BCF7A5448DD5988
:10207000622DEB3C700EF91F8FF706E69DD414C558
:10208000ABB122A0B9923083C77B4E6AD5585C4968
:10209000E33D6A2CF11E780F2B050A0C0D0B102B5B
:1020A0002B082B2B2B2B2B2B0406171A1113141573
:1020B0001609181B122B2B2B2B07191C1D1E1F2753
:1020C000202122262B009C7911241FBECFEFD0E1C6
:1020D000DEBFCDBF11E0A0E0B1E0E2E2F5EF02C06B
:1020E00005900D92A231B107D9F71FE0A2E1B1E04E
:1020F00001C01D92A333B107E1F710E2C8ECD0E2B2
:1021000004C02297FE010E945A7AC63CD107C9F743
:102110000E944B780C948F7A0C940000E091510649
:1021200094E0E99FF0011124E80FF11DEE53FD4FFB
:1021300084918F5F0895F8948091590D90915A0D74
:1021400078940895E82FF0E0E555FD4F84910895C7
:102150002AE0829FC00111248B599D4F08959091D0
:10216000530691708091BC0586FB882780F98927EA
:1021700008950F93022F24FF03C00F7E9DE201C03C
:1021800094E2411104C024E04FE952E00EC0453012
:10219000A0F49091BC0594FF0BC0006194E0499FAE
:1021A000A00111244559594F24E00E94B6630DC087
:1021B0002FEF240F42ED52E006C0941730F02BEFC2
:1021C000240F4AE957E10E94DA630F9108954423EE
:1021D00011F04C5E01C040E0CCCFCF93DF93E5E837
:1021E000F1E080917F06108291E0918381FF09C028
:1021F00092E2928393E29383EF01259694E2948393
:1022000004C0EF01239692E0928382FF09C09FE110
:10221000988390E29983FE01339691E29A8304C0F9
:10222000FE01319693E0988394E0908395E091834A
:1022300096E0928384FF09C095E2938396E29483AB
:10224000EF01269697E2958304C0EF01249697E06C
:10225000938385FF09C098E2988399E29983DE0110
:1022600013969AE29A8304C0DE01119698E098834F
:1022700099E09C93FD0186FD02C0319604C0329620
:102280009BE2ED01998387FF03C08CE28083319646
:10229000DF018AE08D938F5F8631E1F78487CF017C
:1022A000895791408093570127E1258740E099277E
:1022B0000196242F30E08217930754F0F901EB5771
:1022C000FE4FE081F0E0E85AFE4F40834F5FF1CFD0
:1022D0009091830690FF0AC0809164008B7F809369
:1022E00064008091650084608093650091FF02C066
:1022F000BF98C79ADF91CF91089587FF03C081955A
:1023000091E001C090E0E82FFF27E7FDF095E85A43
:10231000FE4F808191118195089587FF03C08195BB
:1023200091E001C090E0E82FFF27E7FDF095EB5723
:10233000FE4F80819111819508950F931F93CF9344
:10234000DF93D62FC42F022F16E0180F442339F045
:10235000463141F04A3E81F448EE52E005C04BE977
:1023600052E002C044EE52E06D2F812FDF91CF91F9
:102370001F910F910C94EC6347FF04C041E20E944F
:102380002963C1952FEF2C0F273114F026EF2C0F66
:102390004CEE52E06D2F812F0E94DA63DF91CF91D6
:1023A0001F910F9108950F931F93CF93DF93D82F11
:1023B000162FC42F022F4D3234F04DE682E18D0FDF
:1023C0000E942963CC52202F4C2F612F8AEF8D0F52
:1023D000DF91CF911F910F91B0CFDF92EF92FF92DB
:1023E0000F931F93CF93DF93D82F162FF42E27FF31
:1023F00003C0E5E0F2E002C0E0E0F2E0C281D38099
:102400002370E22E81E0821718F1C4306CF483E06F
:10241000C802A001112442575D4F0F2D23E0612F08
:102420008D2F0E94B66318C0CD5F0F2D2C2F43E572
:1024300057E1612F8D2F0E94DA63C0310CF4D65022
:102440002F2D45E2612F82E18D0F0E94296304C088
:1024500082E028130AC004C0E11007C0C13029F48B
:102460002F2D4D2D612F8D2F9EDFDF91CF911F914D
:102470000F91FF90EF90DF900895873038F4E82FA8
:10248000F0E0EE0FFF1FEC5DF74F24C08C3050F1F1
:102490008431C0F4482F50E0DA01AA0FBB1FA45FBB
:1024A000BE4F2D913C91803148F4FA01EE0FFF1F91
:1024B000E95DF94F80819181281B390BC901880F93
:1024C000991F0895843248F4E82FF0E0EE0FFF1FC3
:1024D000E452F84F8081918108958E3218F484522D
:1024E0000C94102380E090E008950E9447788823A0
:1024F00011F0A895FACF1092890D08951F93CF93EC
:10250000DF93EC01162F0E94DD62BE0188E10E947C
:10251000116412FF04C067E182E10E942B7210FD7A
:1025200011C011FF06C068E772E080E30E941164E9
:1025300006C04AE652E068E38CE10E9427644BEB58
:1025400052E002C042E652E024E060E086E1DF9122
:10255000CF911F910C94EC6361E0D0DF0C942B675A
:102560000F93262F00E04CEE52E060E10E94DA6308
:102570000F9108951F93CF93DF93C6E110E08C2F46
:102580000E941168110F182BC150CE30C1F78091F5
:102590007F0682FF12C08FE10E94BB6824E0829F09
:1025A000E0011124137CC12B84E00E94BB6820E170
:1025B000829FC00111241C2F182B812FDF91CF91F6
:1025C0001F91089570E0882399F090E0019725E02D
:1025D000289FF001299FF00D1124E60FF71FEE0F41
:1025E000FF1FE05FFA4F808191818B509E4F0895CD
:1025F000FB01E35DFB4F8081992787FD909508954E
:102600001F93CF93DF93D82F162FC4E0DD2391F0D3
:10261000612F8D2FD7DF9C01253F81E0380764F0C3
:102620008BE0820F8D1710F08CE0820FC15029F0E3
:10263000D82FECCFC0E001C0CD2F8C2FDF91CF91F0
:102640001F910895CF93C62FDBDF6C2FCF91BACFA8
:102650008E3791053CF483382FEF920734F483E8EA
:102660009FEF03C08DE790E008950895FF920F93C8
:102670001F93CF93DF938A01C62FD0E08823D9F030
:10268000BFDFF82E8823B9F0C801E2DF2F2D30E03C
:102690002150310945E0429FF001439FF00D112484
:1026A000EC0FFD1FEE0FFF1FE05FFA4F855F9140BB
:1026B0009183808305C0C801CBDFC35DDB4F888376
:1026C00086E0DF91CF911F910F91FF900C944A5DAE
:1026D000AF92BF92CF92DF92EF92FF920F931F9330
:1026E000CF93DF938C017B016A01A22EB0900B0285
:1026F0009B2D9F7D943439F080910208882309F442
:1027000098C0933479F4B19906C080913E01E801F4
:10271000C80FD11D02C0E801219683E10E942172F9
:1027200085E010C0953419F0923409F088C0B19951
:1027300083C080913E01E801C81BD10984E10E9459
:10274000217284E00E941168811168C0E114F104D3
:10275000F9F481E0C816D104D9F480E6B81619F06E
:102760008EE2B81211C010920208C1E001151105E5
:1027700009F0C0E0D0E08B2D0E94DC688EE2B81238
:1027800006C01092380803C0C170DD2701C0B12C0B
:102790004091410150914201C41BD50B80913808F2
:1027A000813071F440911402B19905C084E148026E
:1027B000A001112403C0552747FD5095C40FD51F14
:1027C000CC16DD0644F48B2D0E94DC6883E10E9468
:1027D0002172E6010AC0CE15DF053CF48B2D0E9464
:1027E000DC6884E10E942172E701C017D10749F13A
:1027F000B19903C08FEF80939A06209751F48B2DE7
:102800000E94CC6817FF02C083E101C084E10E94EE
:1028100021728A2D83700E944A5D13C0CC27DD2768
:10282000C01BD10B85E00E94DC6884E00E94DC685C
:102830008DCF953421F47BCFE80121977FCFE8013C
:1028400085CFCE01DF91CF911F910F91FF90EF9037
:10285000DF90CF90BF90AF900895552747FD5095DA
:10286000772767FD7095992787FD909531CF209147
:10287000FB07F3CF462F2091FB0760E0EECF462FFA
:1028800050E02091FB0760E070E022CF90914A0178
:10289000911103C0811106C00895811103C08FEF0B
:1028A000890F01C080E080934A018EEB809349013B
:1028B0000895E0914A01F0E0EE0FFF1FE55BFE4F47
:1028C000918380838FEB8093490108958091550611
:1028D0002AEF829FC0011124880F991F20913A018D
:1028E00030913B012817390720F490933B018093E6
:1028F0003A010895EEE2FEE037A1303180F420A5E0
:1029000041E0420F40A7DF01A20FB11DA20FB11D90
:102910008D939C93403108F010A63F5F37A3089534
:1029200090E08C5F9E4FE6CF90E0E4CF809316025C
:1029300090E04097DFCF0F931F93CF93DF93EC018D
:1029400080915C0681FF07C180916D0686FF89C07A
:1029500012E001E00E94BB698F3F2FEF920781F0E8
:1029600029A9211104C08F31A9F709ABF3CF213078
:1029700011F419ABEFCF223069F78AAB19AAEACF6D
:102980008EA1813041F53FA1332309F452C029A51E
:10299000FE01E20FF11DE20FF11D808191812F5F99
:1029A000203108F020E029A731503FA32091C60133
:1029B00021FDE0C097FD02C021E101C028E22BA368
:1029C0002FE12AA722E02BA78CA79DA718AA84E0B5
:1029D0008FA72EA32EC0811106C08091580D8D3374
:1029E00040F186E025C0823021F19AA990788330A9
:1029F00049F4992329F08BA181508BA3811119C02F
:102A000084E016C0843021F4992399F083E00EC04D
:102A1000853039F48BA181508BA381110AC081E0EC
:102A200007C0863031F4992321F084E18BA385E03F
:102A30008EA38EA1823009F49DC08BA98F5F8BABD2
:102A40008A3008F497C01BAA8DE18AA781E08BA782
:102A500098A1911101C080E08CA718AA83E08FA7EC
:102A600089C098A189A1992311F0846001C08B7F4E
:102A700089A38EA1813081F5C79A2FA1222349F124
:102A800089A531E0380F39A7FE01E80FF11DE80FE5
:102A9000F11D808191819DA38CA3303108F019A68E
:102AA00021502FA32091C60121FD64C097FD02C0D3
:102AB00021E101C028E22BA329A12C7F97FD2260F0
:102AC00029A389A18BBBC7988FE18AA382E08EA33B
:102AD00051C089A18BBB4DC081110CC0C79A89A17F
:102AE000836089A38BBB8091580D8D3308F441C05E
:102AF00086E02FC0823009F43DC089A18BBBC79A04
:102B0000BF9800C0000000C086B38078BF9A9EA125
:102B1000933049F4882329F08BA181508BA3811134
:102B200028C084E016C0943021F4882311F183E09A
:102B30000EC0953039F48BA181508BA3811119C03F
:102B400081E007C09630A9F4882399F084E18BA333
:102B500085E08EA30EC08091830681FD0BC080911D
:102B6000590686FB882780F998A1981711F0C79A13
:102B700001C0C798DF91CF911F910F910895909157
:102B8000510690FD02C093E08927E82FF0E0EE5C4B
:102B9000F74FE081E7FDE95FE595E595E5951E16C0
:102BA00024F0EE2321F0E19502C080E801C080E02E
:102BB000E83008F0E7E0F0E0EC55FD4FE491EE235B
:102BC00019F099E0909355018E2B0895853030F4DB
:102BD0006FEF680F8091EA0635DD24C08D3080F4F8
:102BE000E82FF0E0EE0FFF1FE85EF74F8081918144
:102BF00097FD079653E0959587955A95E1F712C092
:102C00008D3170F4E82FF0E0EE0FFF1FE651F84F22
:102C1000808191816AE070E00E94077ACB0102C056
:102C200080E090E015CD482F833021F0882321F0FB
:102C3000E82F03C0E0E001C0E3E0F0E0EE0FFF1F8B
:102C4000ED5EFE4F80819181443080F420916E06CC
:102C500030E002C0359527954A95E2F720FF06C07F
:102C600020E038E0A901481B590BCA0108951F93C1
:102C7000CF93DF9310E0C0E0D0E0812FD4DFC80F06
:102C8000D91F1F5F1430C9F7C058DF4F8D2F90E058
:102C9000DF91CF911F910895CF938091510681705C
:102CA000C2E0C81B8C2FBFDF6C2F0E94003D20911B
:102CB000BC0525FF05C00F964F9728F080E004C0A3
:102CC00081319C4FDCF781E0CF910895E3E1F1E0A1
:102CD00040E0842F806487B9369A3699FECF24B1BC
:102CE00035B1369A3699FECF84B195B1820F931FD4
:102CF000819391934F5F483061F7089578941F92C4
:102D00000F920FB60F9211248F93809112018F5F53
:102D1000809312018F910F900FBE0F901F90189506
:102D200078941F920F920FB60F9211242F938F93C6
:102D30009F93CF93DF93EF93FF93F89487B78F7BA5
:102D400087BF78942091CA018091CC0190915C0654
:102D5000882359F090FF07C08091320F820F809333
:102D6000320F87FF02C01B9A01C01B9891FF50C011
:102D700080916D0686FF22C0EEE2FEE087A58823E3
:102D800009F446C080910A02811142C080919B00E3
:102D900085FF0DC080A991E0980F90ABEF01C80F9F
:102DA000D11D8AA580939C0087A5815087A787A500
:102DB00081112EC086A1823059F526C0809142092A
:102DC000811126C0EEE2FEE086A1823009F583A1E2
:102DD000882311F081501BC021A1C79A82A180FDD8
:102DE00009C02D7F84A195A196FD2260880F991FAF
:102DF00095A384A381E082278BBB81A3C79882A17E
:102E0000815082A3811104C083E086A385E083A35F
:102E1000F89487B7806487BF7894FF91EF91DF9132
:102E2000CF919F918F912F910F900FBE0F901F9078
:102E3000189578941F920F920FB60F9211242F932A
:102E40003F934F935F936F937F938F939F93AF9332
:102E5000BF93EF93FF9381B7845681BF88EC91E0D5
:102E60000E9469700E94EB688091910D826080934E
:102E7000910DE2E0F1E08081815011F0808304C087
:102E800084E6808381E081838281815011F0828396
:102E900005C08AE08283838181608383FF91EF9103
:102EA000BF91AF919F918F917F916F915F914F9162
:102EB0003F912F910F900FBE0F901F90189578940F
:102EC0001F920F920FB60F9211242F933F934F939F
:102ED0005F936F937F938F939F93AF93BF93EF9382
:102EE000FF932091800030918100F89480917D00C3
:102EF0008F7D80937D0078948091970690919806BD
:102F0000A901481B590BCA019695879530939806DD
:102F100020939706409123019C01215A3F402F3D69
:102F20003E4230F12FEF240F283028F59C0121522A
:102F3000334027373540F0F424E620931502E42F80
:102F4000F0E0EE0FFF1FEE5DFE4F9C012C5D354063
:102F500050915706565F529FC001539F900D112408
:102F60006AE070E00E94077A718360834F5F03C05C
:102F700041E001C040E040932301F89480917D003E
:102F8000806280937D007894FF91EF91BF91AF9123
:102F90009F918F917F916F915F914F913F912F9171
:102FA0000F900FBE0F901F90189592EC980F81E034
:102FB000973008F080E00895FC018081882359F063
:102FC000843218F085520C943F23815056DA40E049
:102FD00060E00C94337208959C0155E03595279577
:102FE0005A95E1F7280F391FAC01440F452F441FB4
:102FF000550B241B350B892F990F990B8595820F43
:10300000931F08959DE7980F9B3F88F08E57E82FF8
:10301000F0E0EE0FFF1FEE5FFA4F808186171CF481
:103020006083862F0895481714F44083842F0895F1
:1030300044E66CE9E7CF982F80915C0284FF03C0DF
:1030400081E0923009F080E0089549E28402900125
:103050001124359527953595279587FD815C86FB4D
:10306000880F880B80F9A901481B510987FD5395EA
:10307000CA0108954F925F926F927F928F929F92B2
:10308000AF92BF92CF92DF92EF92FF920F931F9376
:10309000CF93DF93782E642E882309F4D6C086E17F
:1030A000781621F09AEE791203C0D1C081E0D5C024
:1030B000872D992787FD909597FF03C0919581955E
:1030C0009109873191056CF00E945168982F81E039
:1030D00017141CF49111C1C0BAC0992309F4BDC0E2
:1030E000B6C0872D87FD81958A3040F4825F0E94AB
:1030F000116817140CF4B1C091E0A5C08A50E82EF5
:10310000F12C6701CC0CDD1CE601CE0DDF1DCF5587
:10311000DB4F8A818F7009F49AC094E0961530F4E1
:10312000F701EC57F94F908191708AC0588049801F
:1031300009D8811107C08FEF850D9FD98C01898136
:1031400084DF0EC0823041F48FEF850D96D98C015B
:103150008981815092D904C080E090E000E010E0C5
:103160002A812F70822E912CF4013197EE30F105D7
:1031700008F071C0EA5BFF4F0C94587A17FF35C016
:1031800011950195110931C017FF33C011950195B3
:1031900011092FC001E0060D402F60E0852D6ADF88
:1031A000182F402F60E0842D65DF2A812F70253095
:1031B00061F4112309F44FC0882309F44CC08A81BB
:1031C00082958F7059F591E031C0263019F41111B4
:1031D000F6CFF2CF982F91271EC008171907D9F5FF
:1031E000EECF0817190759F736C0801791073CF33F
:1031F00032C0081719071CF32EC0F601E255FE4F26
:1032000091819095991F9927991F05C0F701EC5757
:10321000F94F908191709111D2CF08C089300CF094
:103220008F5F41E0460D60E025DF982F2A812F70E7
:1032300030E02C30310524F4F701EC57F94F90833E
:1032400017143CF081E0892708C0862F06C080E073
:1032500004C0892F02C090E0E9CFDF91CF911F9188
:103260000F91FF90EF90DF90CF90BF90AF909F9025
:103270008F907F906F905F904F90089540E060E056
:10328000F9CE80913E06FADF811113C080913A0198
:1032900090913B01892B69F410924E0E8091580D4C
:1032A00090919906981749F0809399068EE29EE0D6
:1032B00042CB81E080934E0EF1CF0895CF93DF9300
:1032C000C62F20914802222339F090934A0280931E
:1032D0004902DF91CF91089564E010D90E942B67D5
:1032E000C11103C080913B0601C089E10E94F966CB
:1032F000FCD8D1E00E944778882319F0DF91CF9164
:10330000F4C88091910D833019F4A8951092910D15
:10331000CC2319F0D0934E0E02C010924E0EB1DFA6
:10332000E9CF60E0CBCFE0914A01E43018F08FE0C4
:1033300092E0F7CF2FEB20934901EF5FE0934A0132
:10334000F0E0EE0FFF1FE55BFE4F91838083089551
:103350008091500680FD16C0B9DC9EDC811112C040
:1033600066E081E492E0CAD80E942B67BED8AEDC4A
:1033700088DFA89591DC811105C00E9447788823D9
:10338000B1F3B3C80895DF92EF92FF920F931F93AA
:10339000CF93DF938091500681FD8FC0C091FA04D6
:1033A000F0900C0680917F0682FD0CC08C2F8873F4
:1033B000883041F0803131F0803221F0C77CC86024
:1033C000C093FA04E12CDD24D394D4D8182F85E2DD
:1033D0000E94BB68082FD12FDC276E2D62608CE124
:1033E00092E08CD8D0FF03C060E082E0B9D8D1FF72
:1033F00003C061E087E1B4D880917F0682FF1AC0E4
:103400008D2F8C7051F0612F70E0759567957595D3
:10341000679563706B5E8CE2A3D88D2F8073F9F093
:10342000612F70E044E0759567954A95E1F7637008
:103430006D5F13C0D2FF03C062E08CE291D88D2F84
:10344000887369F013FF02C063E007C014FF02C075
:1034500064E003C015FF03C065E081E481D880917A
:103460007F0684FF0AC0802F8F25837061F0602F54
:103470006370655E86E574D806C0D6FF03C066E05B
:1034800086E56ED80F2DD7FF03C067E08BE668D8BE
:103490000E942B67DD2021F028D834E0E32E01C004
:1034A000E12C1C1302C00F1541F00E9447788111D6
:1034B00004C0E7DEA895D12C88CFDF91CF911F9172
:1034C0000F91FF90EF90DF9008958111FFD98091C7
:1034D0003A0190913B01009709F001972091390141
:1034E000222361F020915D064AEF249F9001112470
:1034F000220F331F8217930708F4C90190933B01F1
:1035000080933A01BECE1F93CF93DF93C8E1D5E0FD
:1035100090E0888111E0190F882329F0AFDE88231D
:1035200011F0812F05C0912F2A96143091F780E079
:10353000DF91CF911F9108958F929F92AF92BF928A
:10354000CF92DF92EF92FF920F931F93CF93DF936F
:10355000EC01A62EB12C6501CC0CDD1CF601E95E58
:10356000FD4F008111818981882309F457C08D8026
:103570009E80888181500E943D127C018981853026
:1035800038F4833050F4813079F0823091F039C0D2
:103590008530A1F0863071F134C0F7FE03C0F1949C
:1035A000E194F108833029F481E08E149F043CF10A
:1035B00025C081E0E814F90414F120C08881F5DC0D
:1035C000882369F08AE09701829F7001839FF00C45
:1035D0001124F4018E9F40018F9F900C1124E81854
:1035E000F908FFE1EF0EF11C81E02FE3E216F10490
:1035F00030F004C081E0E814F90409F080E0E82E1E
:10360000F12C8A81811104C0EF2829F081E01BC0D0
:1036100035DE8111F9CF00E010E014C08A818823E3
:1036200031F02CDE81110BC00FEF1FEF0CC08B812E
:10363000833040F09C81907681E029F403C080E0E3
:1036400091E002C080E090E0892BF501E95DFD4F3B
:103650005F01F080209105019B8121FD2EC09330F8
:1036600059F48A810E94BB68F81689F1FF24F3940B
:10367000F80E00E010E02CC0813041F4F11003C0DE
:10368000292F2D7FB1F0913089F421C0F1E0FF1294
:103690000CC08FEF890F823040F480E000E010E032
:1036A0009230B1F4E2E0FE2E13C080E0913219F4C2
:1036B0000CC000E010E0F82E0BC0FF24F394913210
:1036C00009F0F12C0FEF1FEF03C00FEF1FEFF12CEC
:1036D000F50180838C8187FD03C0F1100AC07BC097
:1036E00088818530D0F3855283D7882309F473C04D
:1036F000F4CF17FF04C08B81833028F46CC0011510
:10370000110509F055C08C818076803211F4CE010C
:1037100053DC8C81877059F1813021F52F81822F04
:1037200098858C3FF1E09F0740F040E050E060E07A
:1037300070E084E0820FE2D60DC0853F21E0920761
:1037400048F0FC01EE0FFF1FE85EFE4F80819927D5
:1037500087FD90952F2D30E021503109820F931F66
:10376000C9D805C060E070E08F810E9426728C810C
:103770008076803411F4CE011FDC8C81282F2871D3
:1037800081F0869586958695837090E0029724F067
:10379000283121F48FE003C08DE001C08EE00E944B
:1037A00021728B8183508E31A0F00FEF1FEF13C079
:1037B0001016110684F40F5F1F4F8B813AE0839F30
:1037C000C00111244397081719072CF000E010E0FE
:1037D00002C001E010E0F601E95EFD4F11830083B5
:1037E000DF91CF911F910F91FF90EF90DF90CF90DD
:1037F000BF90AF909F908F9008951F93CF93DF93CA
:10380000C4ECD5E010E0612FCE0196DE29961F5F53
:103810001830C9F7DF91CF911F9108959F92AF9211
:10382000BF92CF92DF92EF92FF920F931F93CF93AD
:10383000DF93109237088091120102B79091120124
:103840008913F9CF10E0182B41DA8EE587B91BBA3E
:103850008FE18ABB00C099B38FEF8ABBECE0F2E046
:103860008781882311F080E202C0892F807E8483C3
:10387000292F207C8081281759F08074880F907838
:103880003181891711F0315001C03F5F31832083AE
:1038900082819381891711F0838381838091590DEF
:1038A00090919306282F291B20933C018093930627
:1038B00080910A02811106C060E08AED97E00E94C3
:1038C000C54701C0A89580913C01882309F4CCC26A
:1038D000C4E3D1E080910008882319F081508093DF
:1038E0000008C5D92B813C818217930741F09C8346
:1038F0008B831A82198281E0809339012DC06091F7
:103900005206665F49F180913D01823328F188813A
:103910008F5F8883803100F189819A8101969A8333
:103920008983188247E751E0649F9001659F300DBD
:1039300011242817390780F48F719927019761F4B2
:103940008091C6018D7F8093C60186E00E94961407
:103950006DE280E10E942B720E947F310E949A30BA
:1039600080911502882319F081508093150280E020
:103970000E949C5D0E94DD620E94A567D82E809106
:103980000A028111B4C13D2D3F70A32E4AEFA40E4F
:10399000C0915D02C43021F0C33019F4C4E001C00D
:1039A000C8E057E05A1508F495C08D2D807F80320D
:1039B00009F490C08A2D86950E948E1090916D0614
:1039C00090FD04C0CC24CA94C80E03C0E4E0CE2EFF
:1039D000C81A6C2D8091EA060E940013B82E6C2D37
:1039E0000E9422137C01C1110CC0EC0197FF04C09E
:1039F000CC27DD27C81BD90BD595C795D595C7957D
:103A0000CF5F82E0C8120FC080915C0280FD02C0CF
:103A1000912C03C099249394C2E00E94AF10882394
:103A200019F0C19501C0912CDD27C7FDD095A0FEEE
:103A300003C0CE0DDF1D04C0F701EC1BFD0BEF0131
:103A4000209721F08D2F8F2587FF11C091100FC077
:103A5000EF2869F040E050E06C2D8B2D0E9436136A
:103A60008D2D0E94DC6886E10E942172C8C39E01F0
:103A700024583F4F293F310548F4AE016C2D8B2D62
:103A80000E9436136C2FC7FF18C016C01C161D06E7
:103A90001CF44DE750E002C043E85FEF6C2D8B2D26
:103AA0000E943613CE0183589F4F8B3F910508F03B
:103AB000A6C36C2F1C160CF4619567FD6D5F6595B0
:103AC0006595772767FD7095645C7F4F85E10E945F
:103AD000267295C38D2D8F7B71F480919A06B199D2
:103AE0008AC38F3F31F08F5F883C19F48FEF6DEB05
:103AF000D62E80939A06EFE3F1E080913008909102
:103B0000310820813181281B390B37FF02C0215E2B
:103B10003F4F55E0359527955A95E1F72115310529
:103B200061F024813581281B390B37FF02C02F5FDC
:103B30003F4F35952795918380839583848380912A
:103B4000530685FD04C08091FE07882311F020E014
:103B500030E033832283CCE0D2E02D818981821B47
:103B60008F3F09F480E087FD8F5F85958887982FC8
:103B7000990F920F9D838D29A8DCF0906906F7E0DC
:103B8000FF0EE0914A01F0E0EE0FFF1FE55BFE4FF4
:103B9000208131812255354409F040C080915A0876
:103BA00081113CC02885222371F08E81332727FDA7
:103BB0003095F901E80FF11D87FDFA95CF010E94BC
:103BC00028138E831886E091C7048E2F807E31F1F2
:103BD000E295E695E770F0E0E430F10554F4EE0F7D
:103BE000FF1FE65DF74F208131813C5F60E078E0A8
:103BF0000CC0EE0FFF1FE650FB4F2081332727FD3F
:103C0000309523583F4F6AEF70E047E0429FC00174
:103C1000439F900D11240E94F379F62E8091160295
:103C2000F81619F08F2D0E9496148091590687FF7F
:103C30003CC0809156018823C1F1809155018823B1
:103C4000B1F18091920687FD03C08F5F8093920649
:103C500082E00E94BF15982F9F7789F020919206ED
:103C6000921728F510929206D11021C0D82ED09428
:103C7000DD1CDD24DD1C83E68D19D82E18C083E001
:103C80000E94BF15982F9F7791F02091920692176E
:103C900070F410929206D1100AC0D82ED094DD1C78
:103CA000DD24DD1CF4E6DF0E02C01092550181E038
:103CB00080935601E0901202FF24E7FCF094C3E0E9
:103CC000D5E08881882371F0853031F00E94E615B7
:103CD000992787FD909501C0C7010E942813FE0116
:103CE00031978083229625E0C131D20751F7809128
:103CF000490290914A020097B1F060E00E947E1262
:103D00000E94477890919106992339F0811128C03B
:103D100010924A021092490223C0882309F181E0DF
:103D2000809391061DC010929106C0914901CC2349
:103D300031F01092490187E10E942172DC2E84E16A
:103D400080933E01D0920B02E0914A01F0E0EE0F29
:103D5000FF1FE55BFE4F0190F081E02D8D2D099551
:103D60000E942B67C091650088EC91E00E9455701D
:103D7000882311F084E105C08091310F882321F060
:103D800081508093310F06C08091630086958170C9
:103D90008093300F8091300F80934702882309F47D
:103DA0002CC28091590685FD28C2CF7EC093650044
:103DB0008091580D8F71823009F054C0809121019B
:103DC00090912201AC01A4E0440F551FAA95E1F7A0
:103DD00097FD0796BC01F3E075956795FA95E1F7B5
:103DE00020913D06332727FD30952A5F3F4F629F84
:103DF000C001639F900D729F900D1124840F951F39
:103E00002091530626FD05C06091000170910101CB
:103E100002C060EF70E00E94F37980913D01680F6D
:103E2000711D6F5F7F4F7595679560933D01809120
:103E30009006805F80939006811114C080913C06AB
:103E4000681780F4623370F06EE281E10E942B7299
:103E50008091530683FF06C082E390E090933B017C
:103E600080933A01109239018EE587B9369A3699D6
:103E7000FECF84B195B190930101809300018091B0
:103E8000910D833019F4A8951092910D2091120193
:103E900082B7909112012913F9CF90E0922B801BE9
:103EA000910B20910801309109012817390720F45E
:103EB000909309018093080180910501882309F4FA
:103EC00019C100919506109196060F5F1F4F109330
:103ED0009606009395068091C7048F7150E1B52E28
:103EE000B81AF7E1FB1508F477C0EB2CF12CE701C9
:103EF000CC0FDD1FC853DB4F3FE03B1528F4E70133
:103F0000CC0FDD1FC45DDA4F8881C82EC294C694E1
:103F100027E0C222D98045E04C1550F05AEF5D15DC
:103F200038F4ED2DF0E0EE0FFF1FEE5EFC4FD08079
:103F30008F7109F44FC0A2D9A82E80910501F70115
:103F4000E15DFD4F7F0181FD43C08C2D857049F4FB
:103F50008081811106C0AA2021F08D2D90E00E9461
:103F60007A148FEF8C0D823058F4F7018081813004
:103F700079F5A1102DC0F2E0CF1226C0D39424C051
:103F800025E02C1548F4F7018081811121C0AA2079
:103F9000F9F0898174D31CC0F2E0FC15C8F4AA20A2
:103FA000B9F024E0C21631F035E0C31631F066E90D
:103FB00070E005C06CE271E002C068E572E0C80123
:103FC0000E94F379892B21F48D2D90E00E947A14C0
:103FD000F701A082B39485CF01EA14E0B4E8AB2ED8
:103FE000B6E0BB2ECEEACC2EC1E0DC2EE12CF12CCB
:103FF000F8019280892D8F700E94A2108330D9F52C
:10400000F601C081D181209771F4F801C081C7FD0C
:1040100006C0C095FAE0CF02E00111241BC0DD27E5
:10402000C7FDD09517C0D7FF14C0219699F4F701AA
:10403000EE55FB4FC081C7FD06C0CF5F2AE0C2022C
:10404000E001112406C0DD27C7FDD095C095D095AD
:1040500001C02197892D807F59F0892D82958F701D
:1040600089300CF08F5F0AD9811102C0CFEFDFEFEA
:10407000F601D183C083F501C081F80182818F7080
:104080008C3071F48081FAD8811109C0F701EE55A6
:10409000FB4F8081F3D8882319F0C0E001C0C1E054
:1040A000F80182818F708D3091F48081E7D8882368
:1040B00059F0C1FD0CC0F701EE55FB4F8081DED8F1
:1040C000882321F0C3E003C0CD7F01C0C2E0F50129
:1040D000C1935F010D5F1F4FF3E0EF0EF11C22E073
:1040E000C20ED11C34E2E316F10409F081CF85DB66
:1040F0001092050180910301882309F482C0209168
:1041000094062F5E822F8F7090E00C970CF0207F2A
:10411000209394068091C7048F71A0E1FA2EF81ABB
:10412000CBE4D2E0E12C422F4073D42E522F5F70AB
:10413000C52E822F8077B82E207FA22EEF1409F48F
:1041400050C08E0103581D4FF8018081982F907C3C
:104150009034A9F4D11013C0880F880F85958595E8
:104160008DD8882361F080915C0680FF05C0FE0138
:10417000E258FD4F808101C081E00E942172F80168
:104180008081982F907C903849F5880F880F85950D
:1041900085958731B4F08751813039F018F082303D
:1041A00039F01CC0B1101AC006C0C11017C003C03E
:1041B000F0E2AF1213C0FE01E258FD4F80815FD2E2
:1041C0000DC0D1100BC05AD8882341F0FE01E2582F
:1041D000FD4F8081805890E00E947A14E3942296EB
:1041E000ADCF1092030180915501882351F0815089
:1041F0008093550106C080E07CCCC061D7CDD12C26
:104200006CCCDF91CF911F910F91FF90EF90DF90D9
:10421000CF90BF90AF909F900895282F30E08830C6
:1042200058F02850310949E0429FC001439F900D4A
:104230001124875A9B4F089545E0429FC001439F38
:10424000900D11248F5C9B4F0895813641F40E949C
:10425000DC6881E00E9446148BE09EE464D865EC43
:1042600071E180E10C941164CF93C82F80918F0D80
:1042700080FF03C06FE371E102C06DE271E188E18C
:104280000E941164C13629F410928F0D80E00E94C3
:1042900046148091D80881508093D808811103C0BA
:1042A00081E00E942172CF910895CF93DF93EB01BB
:1042B000E7E5F8E08F3B19F49091570803C08E3B77
:1042C00021F490819150988310829281992321F05A
:1042D00091819F779083128290819923A1F08132FE
:1042E00011F08E3871F520910208211108C091500B
:1042F000988310820E94DC6887E10E9421721092EC
:10430000020880E01EC09881843621F49417C0F41E
:10431000995F16C0853621F4973090F0975010C001
:10432000803611F08E3261F49F5F908390689183A4
:104330000E94DC6810920B021092D90790E080E096
:104340009883DF91CF9108951F93CF93DF93182F18
:10435000D62FC42F662329F06FE0842F0E943A14D1
:10436000C82F80915C024C2F83FF02C0440FD062A3
:1043700050E02D2F612F80E60E9414668C2FDF9174
:10438000CF911F910895FF920F931F93CF93DF93C7
:10439000182FF62E0AE08AE0189FE0011124CB596D
:1043A000DD4F2FE130E0211B3109029FA001039F67
:1043B000500D1124BE01CE010A960E94677AFF209B
:1043C00049F0BE016A5071094AE050E0CE010E94F6
:1043D000677A0DC0FE0111920A95E9F78091E30812
:1043E0008883898384E68A838F8188608F83109392
:1043F000E50882E0DF91CF911F910F91FF900C941F
:104400004A5DEF92FF920F931F93CF93DF93E62EB7
:10441000142FEC0188E0F82E00E0FE016591749104
:104420008F2D0E9411640E1540F4FE013E964591B9
:1044300054916F2D85E40E9427640F5F229688E0D7
:10444000F80E073051F74FE360E083E40E94C76441
:104450001123B1F0612F660F660F660F183028F038
:10446000685320E04BE385E403C020E042E480E0B1
:10447000DF91CF911F910F91FF90EF900C944D64BD
:10448000DF91CF911F910F91FF90EF9008950F93BF
:10449000443051F490915A029F70913029F44AE5CA
:1044A00053E10F910C94EC63022F242F45E257E166
:1044B0000E94DA630F9108959C01220F331F280F89
:1044C000391F9595879595958795280F391F95954F
:1044D00087959595879595958795820F931F089554
:1044E000429643E7489F9001499F300D1124C9012E
:1044F000E6E095958795EA95E1F70895CF92DF92EA
:10450000EF92FF920F931F93CF93DF937B018A016A
:10451000D090370895E09D1508F45FC091E09D0D9F
:1045200090933708EBE08E9FE0011124C257DA4FD9
:104530008881882349F081500E943D129C014427C4
:1045400037FD4095542F03C020E030E0A901D09200
:104550003708DE80FD2DF870CF2ED3FC0AC089818C
:104560009A81AA2797FDA095BA2F280F391F4A1FB5
:104570005B1FAB81B0E011960E94C5792C8130E0C1
:104580002F5F3F4F442737FD4095542F0E943C7AC0
:10459000CC2051F089819A81AA2797FDA095BA2F46
:1045A000280F391F4A1F5B1FD0FE07C0509540954A
:1045B000309521953F4F4F4F5F4FE114F10419F0B3
:1045C0008D81F70180830115110529F08E81869573
:1045D0008370F8018083C90102C080E090E0DF9120
:1045E000CF911F910F91FF90EF90DF90CF900895A2
:1045F00081E00895E82FF0E0E55EF84EE491862F23
:10460000992787FD909583589F4FEE5FE23038F4ED
:104610002AE0AC01249FC001259F900D112408952C
:10462000E82FF0E0E55EF84EE491E03F29F1ED3F40
:104630004CF4EE0FFF0BEA5EFA4F8081992787FD5D
:1046400090950895ED3FA1F0BCF0EF3F09F0A4F480
:104650008E2F992787FD909502962FE0289FF001D5
:10466000299FF00D1124E75CF74F83859485089509
:1046700080913D0190E0089580E090E00895CF9210
:10468000DF92EF92FF92CF93DF9300D0CDB7DEB7EA
:10469000F82E1A821982C4DFEF2DF0E0E55EF84EA5
:1046A0002491422F552747FD5095652F752F415F67
:1046B0005F4F4F30510590F54C5A5F4FFA010C9403
:1046C000587AAE014F5F5F4FBE016E5F7F4F8FE044
:1046D000820F14DFEA81F0E0E150FB4EE491EA83BF
:1046E0001DC024E22A8321E0298318C06CE370E016
:1046F0000E94077A6B017C0146E260E0C6010E94DD
:104700003372C70125E32A8309C0E22FEE0FFF0BA6
:10471000EA5EFA4F8081992787FD90954A816981E9
:104720000E9433720F900F90DF91CF91FF90EF9026
:10473000DF90CF9008950F939FE0499FF0011124DF
:10474000E75CF74F43855485022F0E9452660F9114
:1047500008958F929F92AF92BF92CF92DF92EF9285
:10476000FF920F931F93CF93DF9300D0CDB7DEB7A7
:10477000F82ED62EC22EB32E102F80E28A83E42F7D
:10478000FF27E7FDF095E55EF84EA4908E2D817031
:10479000982EE0FE20C0AFE0AA0DA43008F08CC037
:1047A0008BE0A89FD0011124FD01EB56FA4F8081C8
:1047B000882309F481C0AF0100E124E08F2D0E941D
:1047C000B66312FD03C008E10F0D06C00CE10F0D2A
:1047D00088EFD80E01C00F2D8E2D8870882EE3FC37
:1047E0001F7B81EFA8160CF43DC084EF8A152CF4D2
:1047F00082E08A0D8230F8F035C0AE014F5F5F4F26
:10480000BE016E5F7F4F8FE08A0D78DE29812130F7
:1048100011F4106203C0223009F41063EA81F0E061
:10482000E950FB4EE491EA83E7FE02C08C2D9B2DFC
:10483000C82EB92E17C012FD02C08CEF01C082E055
:10484000800F9110865F1770012F212F4C2D5B2D4B
:104850006D2D83500E945266E3E3EA0DEA838AEFEE
:10486000F80E0AC0882071F18DE38F0D212F4C2D99
:104870005B2D6D2D0E9414668E2D867069F0E2FE10
:1048800004C08AE08F0D1B7F02C08091450D212F4F
:104890004A816D2D0E9429638A810F900F90DF91CC
:1048A000CF911F910F91FF90EF90DF90CF90BF902D
:1048B000AF909F908F9008954F5F20E06D2D8F2DCA
:1048C000E6DD7FCF802FD2CF0F931F93CF93DF935F
:1048D000C82FD62F042F122F4AEC54E10E94EC630C
:1048E00040E3400F212F6D2F8CE08C0FDF91CF9193
:1048F0001F910F910C942963EF920F931F93CF9305
:10490000DF93C42F122F2E2DDE2DD3709DE7940F31
:104910009B3F80F043E84C0F8251D6DFDD2359F1F5
:1049200022E042E850E06EE770E08C2F90E00E94B9
:1049300068130CC0552747FD50950E941466DD236F
:10494000D1F0402F612F8C2F0E943714C82F8091F7
:104950000B028D3B81F48DE78C0F8B3F40F0EC2FE9
:10496000F0E0EE0FFF1FEA5FFB4FC08101C0CEE712
:1049700082E00E944A5D8C2FDF91CF911F910F91B1
:10498000EF900895EF920F93E22E0DE723E8B4DF46
:104990000F91EF900895CF93DF939EE0899FE00100
:1049A0001124CB50DC4F8C850E943E19882339F0AE
:1049B0008D850E943E19811104C081E003C080E012
:1049C00001C082E0DF91CF910895942F9695691BE5
:1049D000242F891B0C94B8669091140281E019165B
:1049E00024F0911101C080E0819510921402089585
:1049F00021E0AC0160E080E00C94EC630F931F9326
:104A0000CF93C62F0E941466B8018C2FCF911F91AF
:104A10000F910C941164EF92FF920F931F93CF9319
:104A2000DF93E82E142FFB01F490EB0122963196D0
:104A30004491222381F08091FA07882321F080910C
:104A40000208882351F02091FB0760E0812F0E942B
:104A50002D14182F02C000E002C00091FC07212F86
:104A6000AE016E2D8F2D0E94DA63812FDF91CF91E1
:104A70001F910F91FF90EF900895982F862F242F6C
:104A8000492F61EF71E1C7CF0F931F93CF93DF934E
:104A9000182FD62F022FBA018D2F0E941164C1E06A
:104AA000402F6D2F8C2F811BE8DFC81B8C2FDF91CF
:104AB000CF911F910F910895982F862F242F492F62
:104AC00060E573E1A8CF0F9390915A029F7021E0A7
:104AD000913009F020E000E040ED56E10E94DA63F9
:104AE0000F910895442321F050E08E5E0C941466DB
:104AF00048EE52E00C94EC63EF92FF920F931F93F9
:104B0000CF93DF93EC01062FF42E1091D907A091DB
:104B10002C08B0912D0820912E0830912F08EFE33A
:104B2000F1E0868197818A1B9B0B97FDCF9666E00B
:104B3000959587956A95E1F7482F8093FF078085C3
:104B40009185821B930B97FDCF9656E0959587959F
:104B50005A95E1F7982F8093FD07442311F0B7830E
:104B6000A683992311F0318720878091FE07811158
:104B700004C08091530685FF06C01092FF07109273
:104B8000FD071092FE078091FF07811108C08091F8
:104B9000FD07811104C082819381892B11F00E944D
:104BA0006614E090E8088FEFF81609F44DC0809184
:104BB000380881112DC08091E008882319F01092E7
:104BC000E0081E2D09DF18166CF41E1510F41F5F87
:104BD000C9F488818F1518F48F5F888301C018820B
:104BE00010E010C0882371F011110BC08881882358
:104BF00019F08150888301C0F88281E08093E00839
:104C000001C011500E3271F481E0809338080AC05F
:104C1000813041F40E3221F080910208811102C0EE
:104C2000109238088091D807B1990BC08F3F19F0C6
:104C30008F5F8D3338F091E090930208909338089D
:104C400001C080E08093D807E092FA0780910208C3
:104C500081112CC08091FD078823A1F04881481B59
:104C600047FD40E08F2D90E0242F332727FD30951E
:104C7000281739070CF04F2D4883E11608F41E2D34
:104C80001092FD078881882389F08091FF0788238F
:104C900069F0181B17FD10E08E2D90E0212F3327AF
:104CA00027FD3095281739070CF01E2D003679F1B5
:104CB00090F4023409F46BC028F40132E9F10E32A9
:104CC00031F184C0043409F442C008F46EC00534E4
:104CD00009F44DC07BC0053609F44BC040F40336DF
:104CE00009F466C0B0F5023609F454C06FC00E383E
:104CF00001F10F3B39F0013809F068C01092020849
:104D000081E022C018821092020810E05FC08FEF8D
:104D1000F81609F45BC081E090910208911180E0DF
:104D200080930208882309F451C081E080933808F9
:104D30004DC08EE80E94DC6880910208882319F03B
:104D40001092020843C080E00E9446143FC01E1526
:104D5000E9F1EE20D9F180910208811137C01E15CA
:104D600010F41F5F01C010E010920B022FC011233E
:104D700069F1EE2059F180910208811127C01123B9
:104D800019F0EE24EA94E10E10920B021EC0888105
:104D90008F15E1F080910208811118C088818F156C
:104DA00010F48F5F0DC018820EC08881882371F0C7
:104DB0008091020881110AC08881882319F08150EE
:104DC000888301C0F882E11608F41E2D20910208A4
:104DD00021110AC031E08091410190914201892B5B
:104DE00009F430E0832F01C081E080930108109323
:104DF000D907222311F082E001C081E08093FC07F3
:104E00001092E808DF91CF911F910F91FF90EF90E2
:104E10000895AF92BF92CF92DF92EF92FF920F93DD
:104E20001F93CF93DF93C82F86E195E1E1DD4AE040
:104E30006C2F8BED98E060DEC090DB08B090D90756
:104E400086E0CE3211F0C03671F48C1578F489EF1B
:104E50008C0D8093E9088C2F0E94DC6883E29BE430
:104E60000E94931962C08C1508F45FC081E08093A2
:104E7000E808E12CF12C18E06AEC74E1812F0E9423
:104E80001164AE2C41E34E0D612F8CE00E94B4639F
:104E9000E701CC0FDD1FCE5FDA4FD12CCA1005C061
:104EA000BD1003C00091FC0701C000E08091020822
:104EB000882309F486C0D1101BC0002329F062E2C8
:104EC00089810E943A14898329812D3018F448EA97
:104ED00055E105C02D3140F42D5F4AE957E1612FBE
:104EE0008CE30E94DA6315C02D5144ED52E1F7CFF7
:104EF000002331F04DE763E888810E9437148883EE
:104F00004881552747FD5095202F612F8CE60E9440
:104F10001466D39482E0D812C1CF185F8FEFE81ADD
:104F2000F80A103409F0A8CF41C089EFC80E0EE886
:104F300015E071E3E72EE8E0FE2E6BEC72E18F2DB9
:104F40000E9411644E2D6F2D8CE00E94B463E80125
:104F500020E048816F2D88E10E94B91049815A8173
:104F60006F2D8BE40E9442664B8150E04F5F5F4F94
:104F70006F2D80E60E9442664C8150E04F5F5F4F8C
:104F80006F2D8EE70E94426688E0F80EE394055F7D
:104F90001F4F88E2F812D1CF6C2D660F660F660F97
:104FA000685F20E04EE780E00E944D64DF91CF9182
:104FB0001F910F91FF90EF90DF90CF90BF90AF9037
:104FC0000895D1109DCF80CF1F93CF93DF93C82F2B
:104FD000D62F142F47E16BE2F8DC43E06AE28C2F16
:104FE0000E94C76443E06BE28FEF8C0F0E94C564A0
:104FF000812F69EF0E94E679382F375D8D2F67E0AA
:105000000E94E6798C0F25E045E0632F8250DF9106
:10501000CF911F910C949866CF92DF92EF92FF92FE
:105020000F931F93CF93DF93C2E3D8E04981688148
:105030008AE2CADF4A816B8186E5C6DFC4E2D8E036
:105040002896AAE3FA2E0DE510E0B7E3CB2E89915E
:1050500099919C5FB8010E94077ADD24D394D60E03
:10506000EC2CE61A4D2D6E2D8F2D0E94C7644D2D10
:105070006E2D81E08F0D0E94C7644D2D6E2D82E054
:105080008F0D0E94C76485E0F80E89E4F812DFCF27
:10509000DF91CF911F910F91FF90EF90DF90CF9014
:1050A00008954BE353E168E388E60C9427640F937B
:1050B0001F93CF93DF93D82F162FC42F022F47FFB4
:1050C00008C041E28AEF8D0F0E94296386E08C1BA5
:1050D000C82F2C2F43E557E1612F8D2F0E94DA63F3
:1050E000DF91CF911F910F9108950F931F93CF934D
:1050F000DF93162F042FC62FD0E0AE014F5F5F4F16
:10510000202F682F86E60E941466002329F06FEF97
:10511000CE010E943F14182F812FDF91CF911F9154
:105120000F9108950F93CF93DF93C42FD02FD27098
:1051300001FF03C00E94D31102C00E949D1100FF15
:1051400041C0DD23B9F1CD3274F084ED8C0F0E94A3
:105150007D112091570130E0280F311D87FD3A95D0
:105160002150310907C08C2F0E947D11282F332731
:1051700027FD309580915701482F440F4250C1E0E0
:105180006C2F681B822F0E94371490915701482F73
:10519000552747FD5095292F30E0421753073CF023
:1051A000C91B8C0F0E948D11CCE2C80F0BC00E944E
:1051B0008D1107C040915701642F61958C2F0E947B
:1051C0003714C82F8C2FDF91CF910F910895FF9244
:1051D0000F931F93CF93DF93182FF62EEA01022F20
:1051E0004981453249F429852295269527704EE557
:1051F00054E10E94DA6311C020610E94B9108981D4
:105200008551803150F48F8186FF07C0202F48ECF4
:1052100052E16F2D812F0E94EC63DF91CF911F919E
:105220000F91FF90089580919B03882329F085E2D8
:1052300091E20E94931981E00895CF93DF93C82FE4
:1052400088E00E9411646EEA71E188E20E941164B4
:10525000C13671F028F4CE3269F0C03659F012C070
:10526000CE3831F0CF3B71F480E00E9421720AC049
:10527000D2E001C0D1E08C2F0E94DC6881E00E9466
:10528000461401C0D0E08D2FDF91CF910895CF93C8
:105290009091D6079F3F19F46DE971E102C061E971
:1052A00071E1CBDF813019F0823019F127C0C09154
:1052B000D607CF3F19F40E94FE691BC08C2F0E94B5
:1052C000A8102FE130E02C1B3109CAE0C29FA001D9
:1052D000C39F500D1124BC01665F7F4F0E94677A07
:1052E000EBE9F3E0DF011D92CA95E9F782E00E9445
:1052F0004A5D8BE09EE4CF910C949319CF91089571
:105300000F93CF93C82F4FE06EE578E08091D307DD
:105310000E948F5C00E12AE04EE558E060E181E008
:105320000E94B6634FE360E182E40E94B46380911F
:10533000D407882319F067E671E102C06AE571E1DC
:105340008C2F7BDF813019F08230F9F024C08091FE
:10535000D4078823A9F088E491E10E94AC128091DF
:10536000D3070E94D75C882339F087E10E9421721D
:1053700082E08093D40709C080E00E94217205C0BA
:105380008091D3078F5F0E94846083E69AE2CF9179
:105390000F910C949319CF910F910895DF92EF9292
:1053A000FF920F931F93CF93DF93EC01062FD42E20
:1053B000F62E18E0E12CFF20B9F0F0FE0EC02D2DE6
:1053C00042E851E1612F82E10E94E763AE01612F63
:1053D00088E10E942764E394185FF694FE018491AB
:1053E00021968111FBCFE7CFCD2DCC0FCD0DCC0F6A
:1053F0002AEF210F4C2F67E082E10E94B86644EF4C
:105400004C0F60915B08660F660F660F685F20E0C7
:1054100088E10E944D64E0DA282FCAE5D8E099813E
:105420008B81882351F03091580D36FF08C0815090
:105430008B83811104C018821CC08FEF8B838091F5
:105440000B02813681F028F4803249F08E3239F037
:1054500012C08336C9F088F08E3829F00CC018824B
:105460001B8281E01AC00E94DC6810920B02188235
:105470001B8282E012C012162CF4EA949E1530F4BE
:105480009F5F04C0222339F0911191508B818823B2
:1054900011F08FEF8B83998380E090915B089F5F81
:1054A00020E000FF02C0915021F006952F5F2830C8
:1054B000C1F720935C08DF91CF911F910F91FF906E
:1054C000EF90DF900895DF92EF92FF920F931F937A
:1054D000CF93DF93C82F8CEA90E18ADAF090D2085C
:1054E00080915A08811105C04FE06C2F82ED98E041
:1054F00003DB66EA70E180E00E9411640E94AA5F0B
:10550000AC0160E086E60E9442661091D20880916C
:10551000D407823021F41092D1081092D4078091E0
:10552000030891E0980F191728F4123068F08FEFF4
:10553000810F0BC094E0980F911738F48CEF810F16
:105540008B3018F08AE001C080E080930308082FB8
:10555000D0E1EE24E3941013E12CDD24D394D00E9B
:105560002E2D4D2D6D2F82E10E94446680913A06CA
:10557000081305C04AE26D2F81E00E94B4634FE03A
:105580006EE578E0802F0E948F5CEE2031F08091F4
:10559000D108882311F001E101C000E12FE04EE5C0
:1055A00058E06D2F88E10E94B663D85FD03411F0C7
:1055B0000D2DCFCF80915A08882309F477C08091B0
:1055C000D20890913A06981302C0D9E501C0DEE7EF
:1055D0000E94C05C811101C0D6E980915C0682FF07
:1055E000DF734AE06D2F82E094E1D8DE813009F06C
:1055F0009CC0D0915C08D11105C081EC90E50E945F
:10560000591493C09FEF9D0F923060F50091D2081E
:1056100000933A0680938E0D8C2F0E94DC680E94C6
:10562000465E00933A06802F0E94555E80910501E8
:1056300082608093050181E00E944A5D0E94465E7F
:105640000E94A8190E94C319809155020E949014CB
:105650000E94A76F80915A08823079F2D23009F007
:1056600055C0CBCFD53031F48C2F0E94DC6810921E
:10567000D40704C0D33049F48093D4071093D307E0
:1056800080E899E20E94931950C0D63019F48093B3
:10569000620804C0D73039F410926208109366088B
:1056A00082EC9EE2EFCF8093D1083FC0C63638F43B
:1056B000C43688F4C036C1F0C13641F036C0C138B6
:1056C00029F1CF3B39F1CE3681F50EC08091D1085A
:1056D000882359F10FC090913A068091D20898170B
:1056E00009F48BCF82E00AC0109202088091D108A1
:1056F000882319F01092D10818C081E080935A08CD
:105700008C2F0E94DC6810925B080FC081E00E9421
:1057100046140BC01092D10810925A0880913A0694
:105720008093D20881E00E949C5D8091D1088823FB
:10573000F9F0CF2DDD27C7FDD095812F90E0C81758
:10574000D907B1F061E0610F81E08F0D0E946360C5
:1057500080913A06181303C0F0923A0606C090E012
:10576000C817D90729F410933A0681E00E944A5DD0
:10577000DF91CF911F910F91FF90EF90DF900895EF
:10578000CF92DF92EF92FF92CF93DF93FC01EB0178
:105790009C01DC010E94A6799B01AC01DE010E9404
:1057A000BB79272F382F492F5527DF010E94BB795E
:1057B0006B017C013CE0F694E794D794C7943A954A
:1057C000D1F724E630E02C1B3D0B0E94A6796E5CDD
:1057D0007F4F8F4F9F4F6C0D7D1D8E1D9F1D24E6AB
:1057E00030E040E050E00E941A7AC901DF91CF9189
:1057F000FF90EF90DF90CF9008951F93CF93DF93AA
:105800006115710519F1192F111F1127111F19F0B9
:1058100091958195910977FF0FC0719561957109F7
:10582000C0E0D4E09E01281B390BC901A9DF9E010D
:10583000281B390BC90101C0A3DF112329F022273E
:105840003327281B390B01C09C01C901DF91CF917F
:105850001F910895EF920F93CF93DF93382F862FE8
:10586000642F922F332319F02091FC0701C020E010
:10587000C091E6084EE0C49FE0011124CB50DC4FFC
:10588000933629F4032F4C854DDC8C8724C0923647
:1058900029F4032F4D8546DC8D871DC0E02FF0E0F5
:1058A000E90FF11DE90FF11DEE0FFF1FEE0DF11DC8
:1058B000EC0FFD1FEF01011106C0E22E04E62CE9FA
:1058C00048811AD807C048814C59E22E04E620E0EE
:1058D00013D884568883DF91CF910F91EF9008956C
:1058E00090E0E92FF0E0E852F94EE491E81721F05A
:1058F000EE2321F09F5FF5CF892F089580E0089572
:10590000823430F4E82FF0E0E852F94E84910895A3
:1059100080E20895DF92EF92FF920F931F93CF934F
:10592000DF93F82E162FEA01E22ED02E69E576E1FC
:10593000812F0E94116400E12E2DAE01612F82E4BF
:105940000E94B663DD2099F18F2D880F8F0D880F8F
:105950002091020846E0612F8E5B0E944D644E2D1F
:10596000440F4E0D440F4C5F6FEF610F29E080E450
:105970000E94B866809102088823C9F0CF0DD11D1E
:1059800088818111ADDF2D2D41E460E00E942D144E
:10599000B7DF488150E0282F332727FD3095421785
:1059A000530729F088838091FB070E944A5DDF91AD
:1059B000CF911F910F91FF90EF90DF900895FF928C
:1059C0000F931F93CF93DF93C82FD62FF42E122F50
:1059D000622F842F0E94E212FC01E53F81E0F8076C
:1059E00074F09BE09E0F9F1510F09CE09E0F40E32B
:1059F000490F202F6D2F8C2F0E94296307C0212F64
:105A000047E055E16D2F8C2F0E94DA63DF91CF9133
:105A10001F910F91FF9008957F928F929F92AF9266
:105A2000BF92CF92DF92EF92FF920F931F93CF938B
:105A3000DF93182FC091E9082AE0C29FE0011124EA
:105A4000C05FDA4F85E291E10E94F82443E0612FC4
:105A500087ED98E051D84091E9084F5C60E080E321
:105A60000E94B463B090D70878E0C72ED12CE3E051
:105A7000AE2EBD1003C09090FC0701C0912C82E0B7
:105A8000D81609F467C0E3E0DE1609F478C0F1E047
:105A9000DF1681F067E071E18C2D0E94116401E056
:105AA000911001C000E0292D48856C2D80E33ADB80
:105AB000888780C09110A092E8086CE3762E812C34
:105AC0008091D907881511F000E001C0092D40919F
:105AD000E9084F5F282D6C2D872D71DF992099F1F2
:105AE0008091D90788112FC080910108882359F12E
:105AF0008E01080D111D080D111DF801E080F180C7
:105B0000FBE0EF1AFEEFFF0A24EFE21621E0F206B7
:105B100024F454EFE52EFF24F39422E048EF51E003
:105B200064EF71E0C7010E9468138E159F0559F05C
:105B3000843FE1E09E0711F480E090E0855F9140B2
:105B4000F801918380838394F6E07F0E24E0821233
:105B5000B7CF30C0992051F089856FE08F700E94D7
:105B60003A148F709985907F982B998749854F704B
:105B7000292D206285E0489FA001112417C099209B
:105B800061F089856FE082958F700E943A1482954A
:105B9000807F99859F70982B9987498542954F7092
:105BA000292D2062E5E04E9FA00111246C2D86E690
:105BB0000E941466D394F8E0CF0E24E0D21259CF9D
:105BC000DF91CF911F910F91FF90EF90DF90CF90D9
:105BD000BF90AF909F908F907F9008951F93CF9329
:105BE000DF93C82FD62F142F44E051E10E94276481
:105BF00040E3410F6D2F8CE08C0FDF91CF911F910F
:105C00000C94B463BF92CF92DF92EF92FF920F9306
:105C10001F93CF93DF93C82F83E395E10E94F8246D
:105C200043E06C2F83ED98E00E947C25B090D30870
:105C3000C03611F0CE3649F4B092E9088C2F0E949C
:105C4000DC688CE09DE20E94931965EB70E180E1D5
:105C50000E941164F0E1EF2EF5E0FF2EA8E1DA2EAC
:105C600010E0CC24C3941B11C12CE7018985882343
:105C700031F02C2D4AE26D2D89E70E9429631F5FC8
:105C8000412F6D2D86E0AADF2C2D48856D2D88E1F2
:105C90000E949D11DCE3C0E00C2D2C2F412F6D2DB7
:105CA0008D2F8DDECF5FDA5FC430B1F78AE0E80E6A
:105CB000F11C88E0D80E1430A1F60E94831A682FD8
:105CC000660F660F660F615F29E04AE180E0DF91B1
:105CD000CF911F910F91FF90EF90DF90CF90BF90E9
:105CE0000C94B8661F93CF93DF93162FEC0111230A
:105CF00029F089910E94B4691150F9CFDF91CF91B9
:105D00001F910895CF93C82F0E94BB698F3F21F048
:105D10008C13FACF81E001C080E0CF910895CF933A
:105D2000C82F81E00E94B46980E00E94B4698C2F82
:105D3000CF910C94B469EEE5F8E01382128282E010
:105D40008093E20884E40C94B4690F932091640872
:105D50003091650842E3429FC001439F900D11249A
:105D600061EE71E00E94F379062F28E044E660E3DB
:105D70008EE00E94C3660F910895AC0168E184E251
:105D80000C9427649F92AF92BF92CF92DF92EF92D2
:105D9000FF920F931F93CF93DF93B82ECEE5D8E0F9
:105DA0008C81882319F08CEF90E102C084EF90E1A0
:105DB0000E94F824A89521E6B21659F08FEBB8128C
:105DC00017C00E94A2691092E20819821092D608A8
:105DD0000FC08AE50E94B46980913A060E94555E20
:105DE00089E08093E2081092020881E60E94DC6854
:105DF000C090D6084091E20850E04A30510508F0C2
:105E000084C1FA01ED59FF4F0C94587A8BE10E943E
:105E1000B4698BE10E94B46918821B8281E09FC043
:105E20008B81853030F48EE36DDF8B818F5F8B83C8
:105E30006CC18C81882341F01D8287E08093E20849
:105E400082E40E94B46961C176DF5FC127E08C2DD6
:105E5000622F0E94DA79829F202D112429838CEEF3
:105E600090E18BDF1CE00AE00E94BB698F3F09F4E0
:105E70004CC12091D4083091D5082F5F3F4F30930B
:105E8000D5082093D408833009F469C08D3009F413
:105E900080E02A819881FE01129FE00DF11D1124FE
:105EA000E90FF11D8187811116C09B8189819817A7
:105EB00050F081E0820F8A83883028F088E50E94C4
:105EC000B46983E04CC08EE40E94B4698B818F5F1B
:105ED0008B831882C9CF81E0890F8B3010F48883BF
:105EE000C3CF0883C1CF8A81982E883010F017E085
:105EF000912E4981480F41506B2D86ED98E00E940C
:105F00007C258981C81A8C2D873008F09DCF7E01B1
:105F100099E0E90EF11C00E010E0B8E0AB2EDD24C2
:105F2000C7FCD094091598F421E0C016D10609F0F9
:105F300020E02061A7016A2D8CE00E94EC6328E03C
:105F4000A20E0F5F1F4F8CE0E80EF11CEBCF90E626
:105F5000B912DBC082E50E94B4691D8284E080939F
:105F6000E208D3C082EE90E108DF8D81811120C06C
:105F70001F821E8282E7C6DE882309F44FC08DE0AF
:105F8000CEDE8C2D90E02981821B91092CE0289F88
:105F9000F001299FF00D11243996EC0FFD1F82ECC2
:105FA000838783E084876DE0CF019CDE188264C024
:105FB0008130A1F50E94BB698F3F2FEF920771F1ED
:105FC000988121E0290F2883FE01E90FF11D8187C7
:105FD00088818F3078F38E819F8102EC13E0081B5B
:105FE000190B0D30110510F00CE010E0A8016AE665
:105FF00078E0855B9D4F0E945E7A8E819F81800F45
:10600000911F9F838E83823C934008F48AC085E071
:106010008093E20885E60E94B469188296DE75C016
:106020008BED90E1AADE88850E944F5C882309F4FD
:106030006CC086E094CF82ED90E15CC08BEC90E187
:106040009CDE8D8181111AC01F821E8282E65ADE7B
:10605000882321F388850E94C25C8DE060DE6AE0BF
:106060008BE492E03FDE8BE00E94B46982EC0E94F8
:10607000B46983E00E94B46981E02FC0813049F4A3
:1060800083E640DE882351F282E08D831F821E82E8
:10609000C5CF8230D1F48E819F81823C934028F01D
:1060A00083E00E94B46984E018C08CE038DE8E8101
:1060B0009F816CE0855B9D4F15DE83E08D838E8133
:1060C0009F810C969F838E83A9CF833041F484E611
:1060D00019DE882309F4A2CF82E08D839FCF86E06A
:1060E00011DE882309F49ACF88E08093E20896CFE6
:1060F0008FEB90E142DE09C08AE704DE882329F0B5
:106100000E94AC6980E00E944614DF91CF911F91FC
:106110000F91FF90EF90DF90CF90BF90AF909F9046
:1061200008958EE678CF21E0411101C020E0405D66
:106130000C9429630E949B102091CF083091D008C5
:10614000AC01421B530B9A01283E334088F09093D8
:10615000D0088093CF0880915A028F70823041F42A
:1061600085E10E943E19882319F087E00C94217282
:1061700008950F9300E020E00E9452660F91089569
:106180001F93CF93DF93182F81EA90E10E94F824A8
:10619000163628F4143630F4113659F00FC01E3874
:1061A00041F00CC08091CE0891E089278093CE0801
:1061B00005C01092CE0880E00E9446148091CE085F
:1061C000882309F43FC0C6E0D1E0103641F48FEFD8
:1061D000888319821B821A8287E10E9421726BE6F2
:1061E00070E188E00E9411644981469550E068E0C2
:1061F00086E60E9442664881469550E060E186E668
:106200000E94426649818881481B469550E068E1BA
:1062100086E60E9442668A819B8129E1289FA0012F
:10622000299F500D1124569547955695479520E383
:1062300060E286E60E94146668E570E188E30E94E9
:10624000116429C0C9E3D8E061E470E180E00E94F4
:1062500011644091CE075091CF0768E08AE289DF50
:106260004C815D8168E08EE484DF4F81588560E178
:106270008AE27FDF49855A8584E0569547958A955D
:10628000E1F760E18EE475DF4091CC075091CD07D6
:1062900060E08EE46EDFDF91CF911F910895CF9380
:1062A000DF93282F30E095E0899FE0011124C05052
:1062B000DE4F4C818FE0829FF001839FF00D11240F
:1062C000E75CF74F9881898195878687442311F091
:1062D00090E080E09387848710861782158214826D
:1062E0001286118611821082DF91CF91089510924B
:1062F000CF071092CE0780E0D2CF81E0D0CF5F925F
:106300006F927F928F929F92AF92BF92CF92DF92C5
:10631000EF92FF920F931F93CF93DF930CEC17E054
:10632000F8018F0186818F5F868379E3A72E78E05D
:10633000B72EE4E0EE2EE2E0FE2E812C552453949D
:10634000E501811003C08091BA0502C08091BB05B0
:10635000882309F48FC18D324CF08C520E943E1973
:106360009E81891709F486C18E8302C00E943E195E
:10637000882309F47FC1811002C0B9DF01C0BDDFED
:1063800066246394F70132979080F701319770800B
:106390008EEF890D823028F4C0902808D09029080B
:1063A00002C0C12CD12C80913608882319F0C12C51
:1063B0006CEFD62EF3E0F91548F4E92DF0E0EE0F7E
:1063C000FF1FEE52F84FC080D18002C0992059F1D2
:1063D0002CE2271504F5F801848195812881398103
:1063E000822B932B2B81822B2681822B2A81822B3D
:1063F000892B09F41A8284ED870D0E943E198823A7
:1064000041F09A81911105C091E02B81211190E01A
:106410009B838A8308C0772029F0872D0E943E192C
:106420008B8301C05B828B81882379F061100DC062
:10643000FCEFDF1AD7FE03C02FE3C20ED11C46E0EB
:10644000D594C7944A95E1F701C0C12C8881998100
:106450008C0D911D998388830E949B10F801C48044
:10646000D5808C199D098436910508F46AC066812F
:1064700070E0888199810E94077A462F99838883EA
:10648000F80181100DC0208131812F5F3F4F318392
:106490002083228133812F5F3F4F3383228307C0C4
:1064A0001682F4E6CF0ED11CF801D582C4824423B3
:1064B00031F02F8138852F5F3F4F38872F83611050
:1064C00009C02B81222331F02C813D812F5F3F4F6A
:1064D0003D832C8377277595679589859A85680F05
:1064E000791F7A876987F7013497808191819C872A
:1064F0008B879920E1F0F1E09F1209C0711004C070
:10650000F801628173810EC06C817D810BC0F2E065
:106510009F1203C06F81788505C024E0769567954A
:106520002A95E1F79C01261B370B3C872B87F70147
:106530002081222331F02B853C85821B930B9C8785
:106540008B878394FFE0AF0EB11C25E0E20EF11CB7
:1065500032E08312F5CE09E318E0F8018F01F090E4
:1065600004028091000290910102C385D4852585A3
:1065700036852C173D0709F47FC0D687C587238150
:10658000222309F479C0FF2021F09C012C1B3D0B34
:10659000E9012091530622FF2DC0892B59F1CE31FC
:1065A000D10519F469E289E10BC0C431D10519F4B0
:1065B0006AE28AE105C0CA30D10529F46BE28BE1B9
:1065C0000E942B720AC0C630D1052CF4D7FD05C03D
:1065D0006C2F8CE1F5CF80E001C081E090915306F3
:1065E00093FF08C0882331F082E390E090933B0151
:1065F00080933A01D7FF05C0FF2019F0F801C38549
:10660000D4856CE370E0CE010E94077ADC01CB01F7
:106610004091530641FF1AC0AB2BC1F440915C0678
:1066200041FF07C0009741F046E260E00E943372EC
:1066300003C080E00E9421728091530683FF06C050
:1066400082E390E090933B0180933A01F8018385C7
:1066500094850A960A9780F48CE10E9421728091B9
:10666000530683FF09C082E390E090933B0180933F
:106670003A0102C0612C86CEDF91CF911F910F911C
:10668000FF90EF90DF90CF90BF90AF909F908F9052
:106690007F906F905F9008950F9304E12AE04BE4A0
:1066A00052E0682F88E10E94B6630F9108950F931E
:1066B0001F93CF93DF93D82F162FC42F423049F466
:1066C00080917F0682FF12C08FE10E94BB6825E1A6
:1066D0000AC0463059F480917F0684FF07C085E2E6
:1066E0000E94BB682BE1280F00E006C081E08C0F00
:1066F0000E943E19082F2C2F4CEE52E0612F8D2F57
:106700000E94DA63DF91CF911F910F9108956F92EC
:106710007F928F929F92AF92BF92CF92DF92EF9231
:10672000FF920F931F93CF93DF9391E09093FB071A
:106730009091C60190FF02C044E001C043E06AECC2
:1067400078E00E945521F82E4091EA084150682FC8
:106750008AEC98E00E947C25E090CA08D090FC0763
:106760000091570810E00C30110508F0C6C6F8017A
:10677000E359FF4F0C94587A86E795E10E94F8247C
:106780008091C60180FF02C06BE001C06AE06093A7
:10679000EA0841E04E0D675082E190E10E9401223B
:1067A000ACC689EE93E10E94F82486E08093EA0863
:1067B000EE2011F0C0E001C0CD2D40913B0650E02D
:1067C00009E010E12C2F68E086E60E94FE24CC232D
:1067D00051F04DE26AE080913B060E9437148093AD
:1067E0003B060E9406676DEB7FE080E10E9411642A
:1067F00081E0E8120CC040915701642F61958091AF
:106800003E060E94371480933E062D2D01C020E0E5
:1068100040913E0660E180E60E949D1141E092E0D9
:10682000E91240E08091590668E186FB882780F9EB
:106830000E943D259091590680FB96F99093590648
:10684000C0915506E3E0EE1207C068E78C2F0E9466
:106850003A14C82F2D2D01C020E04C2F440F440FB7
:106860004C0F60E286E60E947225CC2329F043E7B4
:1068700060E288E70E94B463C0935506C0915D064C
:10688000F4E0EF1206C068E78C2F0E943A14C82F7C
:1068900001C0D12C4C2F440F440F4C0F2D2D68E21A
:1068A00086E60E947225CC2329F043E768E288E758
:1068B0000E94B463C0935D0641E085E0E81240E0C9
:1068C0008091530660E383FB882780F90E943D2571
:1068D0009091530680FB93F9ACC480EA93E10E9447
:1068E000F82486E08093EA0865E97FE088E00E946A
:1068F0001164C0916906C95FE11008C0DD2DD06444
:1069000067E08C2F0E943A14C82F01C0D0E44C2FAE
:1069100050E02D2F68E086E60E941466C750C093B1
:10692000690621E0E21220E0409150064695469526
:106930004695477067E67FE080E10E940B258770EF
:10694000880F880F880F90915006977C982B909312
:10695000500640915C06443008F044E021E092E0AB
:10696000E91220E061E37FE088E10E940B2584309A
:1069700008F087E080935C06E3E0EE120AC044E68C
:1069800061E080915A060E94371480935A0621E4F0
:1069900001C020E440915A0650E060E286E60E9481
:1069A0001466F4E0EF1209C065E080915B060E9476
:1069B0003A1480935B0621E401C020E440915B0619
:1069C00050E000E21FE068E286E60E94FE24C091EB
:1069D0005306C695C1706CE975E180E30E941164AD
:1069E00041E085E0E81240E060E38C2F0E943D2505
:1069F0009091530680FB91F91CC488EB93E10E94AF
:106A0000F8248AE08093EA0895E09E1508F4C3C054
:106A10000E94512864EE7EE088E00E94116441E00B
:106A2000E11040E080916D0668E081700E943D2594
:106A300090916D0680FB90F990936D06C09153067E
:106A4000C17041E0E41240E060E18C2F0E943D25DE
:106A500081709091530680FB90F9909353068C13AC
:106A60000E94A81941E0E2E0EE1240E08091590650
:106A700068E185FB882780F90E943D2590915906A1
:106A800080FB95F990935906F3E0EF12D12CE09139
:106A90005606F0E0E95AFC4FD491CCE6ED2FE370B6
:106AA000F0E0E85FFA4E44912D2D60E28C2F0E94B9
:106AB0002963D695D695C650C43581F7DD2039F0C7
:106AC00067E1809156060E943A148093560614E2BC
:106AD000C0E0D0E02C2F4CE754E168E2812F0E9407
:106AE000E86220916E0630E00C2E02C035952795A5
:106AF0000A94E2F720FF06C020E042E168E2812F1D
:106B00000E944D642196185E143821F794E0E91232
:106B10000FC08091C60180FFFFC46FE080916E06B8
:106B20000E943A1480936E068091580D86FFF4C43B
:106B300080915106E5E0EE1213C09091020899236E
:106B400089F063E00E943A1490915106891761F030
:106B5000909159069F77909359068093510604C0EF
:106B600020E003C021E001C022E041E3480F60E3E0
:106B700082E10E942963D4E2C0E08C2F0E948E1033
:106B800020E0482F60E38D2F0E94B910CF5FD85EC0
:106B9000C43099F7B2C4F9E0FE1528F489E0809377
:106BA000CA0869E0E62E83E08093E808CFE6D6E0E5
:106BB00010E058E0F52E00E0212F42ED52E06F2D5D
:106BC0008EE10E94DA6301E086E0810FE81200E0C6
:106BD00024E0AE016F2D8091D9070E948A2C88E0B5
:106BE000F80E1F5F2496143031F787C481EC93E1CF
:106BF0000E94F82486E08093EA0861EC7EE088E059
:106C00000E941164E1100BC0CD2DC06448E768E21A
:106C100080913C060E94371480933C0601C0C0E47A
:106C20002C2F40913C0668E086E60E94226691E0A7
:106C3000E91209C04EE666EF809152060E943714B1
:106C40008093520601C0D12C80915206482F5527BF
:106C500047FD5095465F5F4F2D2D60E180E70E9414
:106C6000146621E0E2E0EE1220E08091500640EB55
:106C70005EE068E181700E9444259091500680FB9F
:106C800090F99093500621E0F3E0EF1220E080911C
:106C9000500640E458E160E2869581700E944425E8
:106CA0009091500680FB91F99093500621E084E08A
:106CB000E81220E08091500641EA5EE068E282FB43
:106CC000882780F90E9444259091500680FB92F914
:106CD0009093500621E095E0E91220E08091500663
:106CE00087FB882780F943E95EE060E30E94442542
:106CF0009091500680FB97F990935006FEC381ED6A
:106D000093E10E94F82486E08093EA08E11003C032
:106D100089E08093E80801E0E11000E02AE04EE518
:106D200056E068E08091D9070E948A2CC0915306F2
:106D3000C2FBCC27C0F96DE875E180E10E941164C7
:106D400041E0E41240E060E18C2F0E943D259091EB
:106D5000530680FB92F99093530621E0E2E0EE1295
:106D600020E08091530645E85EE068E182958170FD
:106D70000E9444259091530680FB94F9909353060A
:106D800021E0F3E0EF1220E08091590649E75EE050
:106D900060E2829581700E9444259091590680FBA3
:106DA00094F99093590621E084E0E81220E0809164
:106DB00053064FE65EE068E285FB882780F90E9473
:106DC00044259091530680FB95F990935306C0910A
:106DD0005906C7FBCC27C0F963E67EE080E30E943A
:106DE000116441E095E0E91240E060E38C2F0E94DD
:106DF0003D259091590680FB97F9909359067DC3E4
:106E000089ED93E10E94F82469E777E080E105C10C
:106E10008EE59EE00E94F82410E0C0E0C43018F037
:106E2000D8EFD10F01C0D12F80917F0601E00C0F68
:106E300082FF04C0C23011F442E005C084FF07C0E5
:106E4000C63029F446E06D2F80E331DC0EC020E02F
:106E5000402F6D2F8AE20E949D118FE08C0F0E94BF
:106E60001168482F6D2F84E45ED9C02F185F093058
:106E7000A9F66CE37EE080E10E941164D8E3C0E0F3
:106E80008C2F0E941168482F6D2F80E24CD9CF5F64
:106E9000D850C630A9F744E35EE068E184E50E947B
:106EA000276416E0C0E2D0E02D2F4CE754E16C2FB0
:106EB00084E50E94E862812F0E941168482F6C2FA0
:106EC0008CE631D981E0810F0E941168482F6C2F28
:106ED00088E729D9DF5FC85F1E5FD43029F780912A
:106EE0007F0686FF0CC06FE27EE088E00E9411649E
:106EF0008BE20E943E19482F68E088E714D9809100
:106F00007F0687FFFAC26AE27EE080E10E94116498
:106F10008CE20E943E19482F60E188E704D9EDC257
:106F200086E29EE00E94F82481E08093EA081092B5
:106F30005601D0E0C0E019E10D2D006241E46D2F53
:106F400088E10E94B46341E34C0F6D2F8EE10E94F3
:106F5000B4638C2F0E941316AC016D2F8AE20E943D
:106F60002964C43028F48C2F0E948E10815003C0F5
:106F7000C730D9F08C2FE82FF0E0EE0FFF1FEC5D4B
:106F8000F74F20813181129FF001139FF00D1124E2
:106F9000F7FF02C0E150FF4F5F2F550F550B4F2FEA
:106FA0006D2F8AE50E94426605C0402F6D2F8AE54D
:106FB0000E943666CF5FD85FC83009F0BFCF62E26B
:106FC0007EE088E20E94116440910001509101012D
:106FD00060E388E70E94426681E08093FE0780912B
:106FE0000208882309F489C24FE761E880913D06D1
:106FF0000E94371480933D0680C281EE93E10E9487
:10700000F82486E08093EA088090D9078091630095
:1070100081FF06C06BE17EE088E10E9411646DC2D1
:107020006BE07EE088E00E941164C7E4D6E0A12C0A
:1070300010E133E0732E992493949A0C20E0492DAB
:10704000612F80E00E94B910B12CEA1004C0709248
:10705000E8088B1419F020E0C12C02C0CD2C22E0EE
:10706000E2E0BE16D1F1F3E0BF1609F44DC081E0B5
:10707000B81689F0498142954695469543706EEF62
:107080007DE0812F0E940B258295880F880F807CE0
:1070900099819F731FC00981000F000F0595059509
:1070A0009DE00902F0011124F7FD3396AF015595DB
:1070B0004795559547952C2D612F82E40E941466C3
:1070C000C1FE3AC04FE161EE802F0E9437148F73EA
:1070D0009981907C982B99832FC06880E62DE7706A
:1070E0006E2E20E12E0F0C2D4AE957E1612F88E426
:1070F0000E94DA63C1FE20C063E0862D0E943A142C
:1071000087709881987F16C008810595059505952B
:107110002C2D402F612F8AE50E949D11C1FE0CC0CD
:107120004FE061EF802F0E943714880F880F880F7F
:1071300098819770982B9883B394F4E0BF1285CF11
:10714000185F2296103311F0A92C75CF84E0E81255
:107150000BC0CD2DC06248E266EF809157060E94B9
:1071600037148093570601C0C0E240915706552757
:1071700047FD5095465F5F4F03EF1DE02C2F60E306
:107180008EE40E94FE2404E211E0CFE3D6E090E317
:10719000D92EF801419151918F0129913991421BCA
:1071A000530B440F551F20E268E38D2D0E94146697
:1071B000F8E1DF0E80E9D812ECCF95E0E91215C0B6
:1071C000E0E6FE1214C01092020888E0E4E2F1E06A
:1071D000AFE3B6E001900D928A95E1F781E00E945D
:1071E0004A5D87E10E94217202C020E001C021E0D7
:1071F0004FEE5DE068E380E00E94EC637EC188ECC6
:1072000093E10E94F82488E08093EA08E11014C01A
:107210000E9451288091530621E047EE5DE068E02E
:1072200086FB882780F90E9444259091530680FBB5
:1072300096F99093530661C16CE97DE088E00E9465
:107240001164C0E008E0C0907F06C23051F0C33046
:1072500069F040918006C13079F442954F7010E199
:107260000DC0409182064F7010E408C04091820624
:1072700042954F7010E802C04F7014E0FF24F39461
:10728000FC0E21E0EF1020E068E77DE0802F0E94F7
:107290000B25D82F812F80958C21D11103C080938D
:1072A0007F0603C0182B10937F0680917F06C812BB
:1072B0000E94ED10C23051F0C33069F0C130A1F42A
:1072C000D295D07F909180069F7012C0DF70909110
:1072D0008206907F05C0D295D07F909182069F70E4
:1072E0009D2B9093820607C0DF7090918006907F5F
:1072F0009D2B90938006085F083211F0CF2DA3CF0D
:10730000F5E0EF1611F040E001C04D2D80918306AD
:1073100068E281700E943D259091830680FB90F980
:107320009093830686E0E81611F040E001C04D2DF1
:107330008091830660E3869581700E943D2590913F
:10734000830680FB91F99093830697E0E912D12C94
:10735000809183064D2D68E382FB882780F90E9487
:107360003D259091830680FB92F990938306C5C0DA
:107370008CEA93E10E94F82481E08093EA0810925D
:10738000CA08CEE5D8E010E0812F0E9413162E85A2
:107390003F85821793070CF49C013F872E874C8D05
:1073A0005D8D481759070CF4AC015D8F4C8F14307C
:1073B00060F02E853F85240F351F37FF02C02F5FF9
:1073C0003F4F35952795398328831F5F22961730C5
:1073D000D9F6809188088093FE07E0E2FE1621F03E
:1073E000FFEBFF120EC00BC08F5F809388088330C5
:1073F00041F487E10E94217281E00E944A5D10926F
:10740000880880918808813089F050F0823009F036
:1074100072C010925601ECE6F8E0CEE0D6E01FC054
:1074200067E67DE088E10E94116465C0CEE5D8E0A2
:10743000D12C18E9E12E1AE3F12E08E615ECFF86AF
:10744000EE861D8F0C8F8D2D0E94131689939993B4
:10745000D39487E0D812F3CF69E57DE043C0619112
:107460007191848595859B01281B390B37FF03C0DB
:10747000319521953109233331053CF1DF015097D6
:107480004D915C91598348839A01261B370BB901B2
:1074900037FF02C0615C7F4FB6E075956795BA957E
:1074A000E1F7261B370B3F872E87841B950B9C012A
:1074B00097FF02C0215C3F4FA6E035952795AA951E
:1074C000E1F7821B930B9D8F8C8F229698E0EA3711
:1074D000F90729F60E94115C9093390680933806CB
:1074E00067E47DE080E10E94116441EF53E168E1CF
:1074F00082E10E9427640E940C28DF91CF911F91A6
:107500000F91FF90EF90DF90CF90BF90AF909F9042
:107510008F907F906F90089529E04CE567E283E2B9
:107520000E94B86605CBCF93DF93C82FD62F462F86
:1075300060E2BDD841E04D0F68E28C2FB8D842E040
:107540004D0F60E38C2FDF91CF91B1C81F93CF9384
:10755000DF93EC01862F11E0683008F410E00E9400
:107560000D21FC019E013C5F37FD0DC0211588E017
:10757000380784F0112319F048E050E002C044E0DD
:1075800050E0E40FF51F8081992787FD9095982F93
:10759000882723C0832F112321F03327220F331F85
:1075A00002C086953170482F50E0E40FF51F6081CE
:1075B00040E052E0421B530B559547956403C001D0
:1075C000659F900D11246181359527956203A00177
:1075D000639F500D1124840F951F69E170E00E9494
:1075E000077ACB01DF91CF911F910895BF92CF927F
:1075F000DF92EF92FF920F931F93CF93DF93182F99
:107600007B010E94CB24C82E812F0E941B18811160
:1076100004C001E01E141F040CF400E08EE0189F6B
:10762000E0011124CB50DC4F84E0C89E600111249E
:10763000F601E00FF11DEC0FFD1FB080812F0E94BD
:107640001B188823A1F08B2D0E941818682F77270C
:1076500067FD7095C7019C5F97FD0196959587958D
:107660000E94FD2B7C01EE0CFF1C00E00BC08B2D5B
:107670000E941818682F772767FD7095C7010E9430
:10768000FD2B7C01CC0DDD1DC00FD11D8A8144E690
:1076900060E08C590E9402189701A82FBB27A7FD14
:1076A000B0950E94A07924E630E040E050E00E94CE
:1076B0003C7AE901812F0E941B188111D450CE0120
:1076C000DF91CF911F910F91FF90EF90DF90CF90BE
:1076D000BF900895DF92EF92FF920F931F93CF9385
:1076E000DF93D62E20EEF22EF80EC0E0DCEF0FE78F
:1076F00030E2E32ED11005C06091E708CE0126DF0D
:1077000004C0BE018091E60871DF97FD4F969C0191
:1077100095E0359527959A95E1F7122F0F3709F4E3
:10772000022F412F552747FD5095401B510907FD5A
:10773000539557FF03C0519541955109423030F49C
:107740006E2D611B8F2D0E9479640CC001171CF0F7
:107750009FEF940F01C090E06E2D611B691B8F2D70
:107760000E94C764112321F060E28F2D0E9479648A
:10777000F394A096C03284E0D80711F0012FBACF5D
:10778000DF91CF911F910F91FF90EF90DF900895BF
:10779000DF92EF92FF920F931F93CF93DF93D82E38
:1077A0008091E708EE24E394883008F4E12C0E94ED
:1077B0000D21EC0140E460E08CE50E94C764F12CEF
:1077C0000CE91FEF2F2D30E0EE2019F049E050E0DA
:1077D00002C045E050E0241735075CF5C90145E0DB
:1077E000880F991F4A95E1F7EE2019F064E070E0E8
:1077F00002C062E070E00E94077AE62FDE01A20F6D
:10780000B31F2C9130E22302C0011124B8010E9461
:10781000077ADF1005C0625E25E045E08AE304C018
:10782000615E23E043E08BE38E0F0E94B866F39421
:10783000C9CF60E08CE5DF91CF911F910F91FF9050
:10784000EF90DF9047CF5F926F927F928F929F92DF
:10785000AF92BF92CF92DF92EF92FF920F931F935E
:10786000CF93DF93882EAA24A3948091E7088830D1
:1078700008F4A12C8AE493E10E94F824AA2011F0D4
:1078800049E001C045E0682D8FED98E00E947C251D
:107890008FEB881202C01092DE084091E70850E09A
:1078A0004F5F5F4F21E060E08AE20E9414668091A2
:1078B000E7080E940D21EC01B090DF086090FC0702
:1078C000AA2019F0F9E07F2E02C0E5E07E2E5C2EA2
:1078D0000C2F1D2F65E0E62EF12C70E1972ECB2C9E
:1078E000D12C802F8519B81611F020E001C0262D6B
:1078F000F80141918F01552747FD5095692D88E189
:107900000E941466AA20A1F0F9E0EF1689F0CE14C7
:10791000DF0411F020E001C0262DFE01EE0DFF1D59
:107920004081552747FD5095692D80E30E941466DC
:1079300088E0980EEFEFEE1AFE0AF8E39F12D1CF1F
:10794000B71411F020E001C0262D43E453E168E3B1
:107950008CE00E94EC63B7103AC080910208882343
:10796000F1F180920B021091DE0820E044E06CEF10
:10797000812F0E942D14082F8093DE08811779F142
:10798000AA2011F024E001C022E0122F119530E06E
:1079900059E1F52EE12FFF27E7FDF0952E173F0760
:1079A00094F0EC0FFD1FE20FF31F1002A001112451
:1079B000F49EC001F59E900D1124B9010E94077A32
:1079C00060831F5FE7CF82E00E944A5D08C0CB0D55
:1079D000D11D44E66CE988810E94371488838B2D81
:1079E000DF91CF911F910F91FF90EF90DF90CF909B
:1079F000BF90AF909F908F907F906F905F90C8CE18
:107A0000EF92FF920F931F93CF93DF93C62FD0E097
:107A1000FE01EE0FFF1FE35FF94F21813281821BD0
:107A2000930B9C01BC01882777FD8095982F0AE075
:107A3000660F771F881F991F0A95D1F71216130634
:107A40001CF4258D368D02C02785308924363105FA
:107A500014F424E630E0442737FD4095542F0E946B
:107A60003C7A790121308CEF380744F0211584E00D
:107A700038073CF0E12CA4E0FA2E03C0E12CBCEF67
:107A8000FB2E0E94AF10882379F080915106082FB9
:107A9000017010E082E090E0801B910BC817D907BD
:107AA00019F4F194E194F108C701DF91CF911F918E
:107AB0000F91FF90EF9008952F923F924F925F9217
:107AC0006F927F928F929F92AF92BF92CF92DF92EE
:107AD000EF92FF920F931F93CF93DF93CDB7DEB753
:107AE000A1970FB6F894DEBF0FBECDBF8F879B87DF
:107AF0006D8B80915106880F880F9E012F5F3F4F3D
:107B00004901E12CF12C1D8E1C8E1B8E212C682E20
:107B1000712CA3014E535D4F3A0160726E8B5D89EB
:107B200051705D876D896270562E3E2C8E2D0E949D
:107B300013166E2D65DF8C0173E07E1570F054E036
:107B4000959587955A95E1F7F701EE5CF74F80839D
:107B5000F301EE0DFF1D449001C04E2CC42CD12C1E
:107B6000C601880F991F9A878987FC01EC5DF74F42
:107B700011830083C80117FD0F9634E09595879512
:107B80003A95E1F7282F87FD219522307CF481E09A
:107B900090E00C2C01C0880F0A94EAF7211102C072
:107BA000982F03C09091CB079823292A93E093152F
:107BB00008F473C0AD85A11158C08091570281FFB0
:107BC00054C05601AA0CBB1CF501E95BF94F5F01DB
:107BD0008181807C09F449C0808185958595859552
:107BE0000E943E19882309F440C080911502882321
:107BF000E1F1D501EC91E770F0E0DF01AA0FBB1FC6
:107C0000AC5DBE4FEE0FFF1FE15CF94F8D919C9173
:107C100020813181821B930B97FD0196AC01559514
:107C20004795F5012181322F330F330F3595359567
:107C30003403C001359F900D11246FE170E00E9464
:107C4000077A660F771F660F771F22952695269570
:107C50002370213009F09DC6060F171FF2E04F1266
:107C600004C07C8F6B8F21E02D8F3E89332339F048
:107C7000F601EE0FFF1FED53F84F11830083B8019B
:107C8000842DB4DC8C01632D8091EA060E942213BE
:107C9000880F991FD4018D939C93BE89BB2339F023
:107CA000F601EE0FFF1FE555F84F118300835520B5
:107CB000E1F0E3E0E315C8F0F2E04F16B1F0065F43
:107CC0001F4F0531110538F0F601EE0FFF1FE55586
:107CD000F84F11821082E1E0F0E0EC0FFD1F2985E2
:107CE0003A85E20FF31F118210823FEFE31AF30A85
:107CF00042E0840E911C57E0E516F10409F015CF1F
:107D000080915C0280FF27C062E08091EA060E94B9
:107D10002213182F0E94AF10012F81110195202FDF
:107D2000332727FD3095432F532F23583F4F4F4F75
:107D30005F4FA0E0B4E08091AF079091B007A81B1F
:107D4000B90B0E94C57920E034E040E050E00E9489
:107D50003C7A3E832D836E89662309F435C11091E8
:107D6000600212218091CB078095812319F088E170
:107D70000E9421721093CB070BEA17E0D8018D0106
:107D800080E094E0FD0197878687918B808B4091FE
:107D90006302442309F458C0A281B381E680F780CE
:107DA0009D010E94A0794B015C019701D7010E94BF
:107DB000A079860E971EA81EB91E842F0E94251832
:107DC0007C019C01DC010E94A079681579058A0577
:107DD0009B05D0F580E1C82ED12C40E050E8E0E0D2
:107DE000F0E89A01DA010E94A67986169706A8069D
:107DF000B90610F44E275F27F695E79521E0C21AE1
:107E0000D108C114D104E9F4F801228133814A0177
:107E1000A12CB12CD7010E94A079A50194010E9448
:107E20003C7AF8013383228326813781D7010E946F
:107E3000A079A50194010E943C7AF801378326833A
:107E400003C04E2B5F2BCDCF60916102862F807EC9
:107E500009F4BAC051100EC0F801228133818B8120
:107E60009C81280F391F868197814F815885840F07
:107E7000951F04C080E090E020E030E04091620275
:107E8000442379F04150E42FF0E0EE0FFF1F44311E
:107E900018F4E00FF11F02C0E452F84F4081518105
:107EA00002C040E050E062FF03C0319521953109E6
:107EB00063FF03C091958195910964FF03C05195BB
:107EC00041955109629566956770633009F463C006
:107ED000643009F469C0623059F1BC0197FF02C0F7
:107EE000695F7F4FF3E075956795FA95E1F7DC01DF
:107EF000A61BB70BBC0197FF02C061587F4F660FEE
:107F0000672F661F770BA61BB70B97FF02C0815028
:107F10009C4F892F990F990B85958595A81BB90BB7
:107F20007A01E21AF30A37FF2CC02F5F3F4F29C0B6
:107F3000B90137FF02C0695F7F4FF3E07595679520
:107F4000FA95E1F7D901A61BB70BB90137FF02C0BB
:107F500061587F4F660F672F661F770BA61BB70B05
:107F600037FF02C021503C4F232F330F330B259591
:107F70002595A21BB30B7A01E81AF90A97FD019621
:107F80009C0135952795240F351FB9016A0F7B1F7A
:107F90002A1B3B0B12C07A01E21AF30A240F351F89
:107FA000B901680F791F07C07A01E21AF30ABA0112
:107FB000680F791F9A01281B390BF801F38AE28AAE
:107FC000758B648B378B268BFF85FB8B2B852C8BDE
:107FD00045EA53E05A8F498F1E861D86B5E62B2E43
:107FE000B2E03B2E1F8A198A5D8559A3B101665FF5
:107FF0007F4F788B6F87C12CD12C7601D1018C916A
:1080000090E00197ED85FE858E179F0709F059C313
:10801000EF85F889389780810E9418188A8B7F89AC
:10802000672F70E07A8769876551794F5B01FB01A3
:10803000E056FF4F908040E061E00F8518890750BF
:108040001109D8018C910E943A18F8019081992366
:1080500059F0EF85F889399790819C50983020F439
:1080600090911502992399F0882391F0F10181856F
:108070008F7190E00090EA0602C0959587950A946A
:10808000E2F781709927F1E08F27817001C080E0CD
:108090002F8538892950310938A32F8FD9011C9198
:1080A000811131C0F501E056FF4F10821D32C9F435
:1080B000E985FA85EE0FFF1F29853A85E20FF31F48
:1080C000E55DF84FAFE8B2E0A70196010E94BB79E9
:1080D000BB2797FDBA95A92F982F872F808391836F
:1080E000A28388EF810F823008F0DEC2F101878120
:1080F0008670843009F4D8C280E0193009F0BCC021
:1081000000E01CEFBDC081E0911080E0982E2FEFC1
:10811000210F2C30B0F4822F90E0DC01AA0FBB1F9E
:10812000A555B84F0D911C91243008F091C0F10174
:10813000278126FF8DC0FC01EE0FFF1FED53F84F86
:1081400026C02431C0F483EF810FE82FF0E0DF0177
:10815000AA0FBB1FAC5DBE4F0D911C91843040F443
:10816000EE0FFF1FE15CF94F80819181081B190B15
:10817000000F111F6DC0243280F4F1018781E22FBE
:10818000F0E0EE0FFF1F86FF05C0EE54F84F0081B0
:1081900011815EC0E452F84FFACF243281F5F1012B
:1081A0009185929596959770B1F08EE0890F823106
:1081B00028F081E1890F853149F01CC08131D1F46B
:1081C00090917F0692FF16C01FE106C090917F0636
:1081D00094FDE4C30FC014E0812F0E945168811107
:1081E00035C081E0810F0E945168882361F100E071
:1081F00010E02EC00E941168882341F124C02C3267
:1082000060F4E22FF0E0EE0FFF1FE854FB4F008117
:10821000F8E00F02800111241BC02C3251F4C70179
:10822000B60124E630E040E050E00E943C7A89014B
:108230000FC040E050E060E070E082ED810F0E94EE
:108240007E228C0105C000E014E002C000E01CEFBB
:10825000F1018781982F907391F0829583708150FE
:1082600021E030E002C0220F331F8A95E2F7C901F6
:108270003989382B398B03C000E010E001C081E060
:10828000E985FA85E557F84F8083F101878183FD01
:108290000EC0EF85F88932978081882341F04DE741
:1082A00063E80E9402180E942518080F191FF101A7
:1082B000F681FE8FF11105C0F1018581882309F453
:1082C00021C180915C0283FF03C0F4E1F88F02C0FA
:1082D00024E6288F49855A85440F551FDA01A55198
:1082E000B94F3C91FD012181E985FA85E40FF51F25
:1082F000E55DF84F80819181A281AC016A2F7727DB
:1083000067FD70952A013B01BB2777FDBA95A72F22
:10831000962F852FB801681B790BCB01AB01465F07
:108320005F4F4531510550F0A32EB22EA114B10478
:1083300039F4F1012581211108C002C0A12CB12C12
:10834000911003C09C878B8737C0F10187818670AD
:108350008430D9F4E081F0E0EE0FFF1FEE5FF74FBD
:10836000A081B18120E034E60E94B5792B013C0167
:10837000FA89FF2351F02F2F332727FD3095432F04
:10838000532F0E943C7A29013A01BB2777FCBA950A
:10839000A72D962D852D9801281B390B3C872B87FF
:1083A0002115310549F0F101858137FF82958F70E4
:1083B000F88DF89F500111241A141B04B4F4809115
:1083C0003C01882331F021E0A21AB108A114B104C4
:1083D00049F0332777FC3A95272D162D052D1C865D
:1083E0001B8603C0AA24AA94BA2CE985FA85EE0F4D
:1083F000FF1FE551F94FB182A0824B855C85452B6B
:1084000009F473C04801AA2497FCA094BA2C5E8D8D
:10841000552309F466C080913C01882309F440C0CB
:108420006A89662379F0262F27FD219530E040E008
:1084300050E060E070E080E293E00E943C7ACA0184
:10844000B90104C060E070E080E293E0F1012681B0
:108450004B855C851416150644F0909580957095B3
:1084600061957F4F8F4F9F4F22952F7030E02115E0
:10847000310591F0A88DA29FA001A39F500D11245A
:108480009A01442737FD4095542F0E943C7A420EB2
:10849000531E641E751E04C04424582C692C7A2C6B
:1084A000BB2777FCBA95A72D962D852DEB85FC85EE
:1084B0001E161F0634F488169906AA06BB0634F069
:1084C00009C088159905AA05BB0524F44424582C35
:1084D000692C7A2C332777FC3A95272D162D052DFC
:1084E00004C04424582C692C7A2CE985FA85EE0FB7
:1084F000FF1F29853A85E20FF31FE55DF84F4082A3
:1085000051826282F1018781EF85F889369787FF72
:1085100026C080810E941818A82FBB27A7FDB09500
:108520001A161B0644F417FF62C024E630E02A1B2B
:108530003B0BD90109C0109709F459C01016110658
:108540000CF055C0AC59BF4F98010E94A07924E6A9
:1085500030E040E050E00E943C7A890148C06081F0
:108560008BE1860F873340F06058772767FD709561
:10857000C8010E94FD2B34C0862F992787FD909556
:10858000A92FB92F87309105F8F4FC01E758FF4F68
:108590000C94587A17FF2BC010C0101611066CF0FF
:1085A00026C017FF24C011950195110920C010168F
:1085B0001106C4F002C017FD18C000E010E017C09B
:1085C000101611067CF011C067FF06C011950195C9
:1085D000110936E0361B632F6750C8010E94A63A86
:1085E0008C0105C000E014E002C000E01CEFF101C6
:1085F000478140FD12C0AF8DB8A18C919FEF980FBD
:10860000943058F4FE013196E80FF11DE80FF11D8A
:10861000329780819181080F191F9801EA89AE2F46
:10862000BB27A7FDB0950E94A0794B015C0143FFD9
:1086300015C0EF85F88932978081882379F04DE75E
:1086400063E80E9402180E94251824E630E0DC014D
:108650000E94B579860E971EA81EB91EF10187816A
:1086600086958370813039F08230E1F0C80CD91CD6
:10867000EA1CFB1C19C0C501B40124E630E040E04F
:1086800050E00E943C7ACA01B901A70196010E94FC
:10869000CB7920E034E040E050E00E943C7A690170
:1086A0007A0102C075016401FAE02F0E311C2F8996
:1086B0002F5F2F8B4F855889465F5F4F588B4F87B1
:1086C0009DCC1092360880919B06882309F441C006
:1086D0008F01000F111F000F111FF801E556F94F10
:1086E00087849088A188B288FE89FF2319F0812CA5
:1086F000912C5401C701B60124E630E040E050E07F
:108700000E943C7AE091EA06F0E0EE0FFF1FE5568A
:10871000F94FA581B6810E94BB79680D791D8A1D2C
:108720009B1DF801E556F94F6787708B818B928B03
:108730002D8926FFF9C020919E0630919F0640E0CA
:1087400050E00E943C7AA4E6B0E00E94BB796B0145
:108750007C010D851E85000F111F0C5F174FC7018F
:10876000B60124E630E040E050E00E943C7AD801B7
:108770002D933C93698C7A8CF3013F018381948122
:108780008090FB04912C881699063CF0919481947A
:108790009108881699060CF44C01F301218184019B
:1087A000FAE02F02000D111D1124D3012C91F401C8
:1087B0004AE02402E00DF11D11249F01285E3340A0
:1087C00008511C4F033E54E0150714F002EE14E06C
:1087D00049012E316BEF360724F42EE1822E2BEF68
:1087E000922E302F212F8017910714F4382F292F24
:1087F000A32EB22EA814B9040CF45401C114D10450
:10880000E104F104A9F0F7FE04C0D501A819B909E3
:1088100003C0D801AA19BB09A70196010E94C57916
:1088200020EA36E841E050E00E943C7A69017A0192
:10883000C5010E94EC175C01AC0CBD1CC8010E9474
:10884000EC178A159B050CF45C01C4010E94EC171F
:10885000A816B9060CF45C01F3018281882319F093
:10886000B194A194B1089091C7049F7180E1891BD4
:10887000F9A1F81708F052C00D851E85000F111FD1
:1088800008531B4FD8018D018C91982F9F7309F4C9
:1088900045C0982F907C903409F440C09038F1F195
:1088A000880F880F859585950E943E19F801908163
:1088B000907C903C39F5882319F01092CB081BC0AE
:1088C0009091BC05209128083091290895FF06C099
:1088D0002D5E3F4F2732310520F00DC024313C4F33
:1088E00054F4AD8DAA2309F45BC02B8D3C8D24314B
:1088F0003C4F0CF455C09091CB08911101C081E020
:1089000080933608882351F0ED85FE85EE0FFF1F1A
:10891000E753FB4F80810E9425185C01F894AB89D6
:10892000BC89AD92BC927894ED85FE853196FE8728
:10893000ED872B893C892E5F3F4F3C8B2B8B498DDC
:108940005A8D4B5F5F4F5A8F498F709709F04CCB10
:108950001091580D798970FF05C0111103C08EE187
:108960000E942172898981FF07C0812F877F80340F
:1089700019F48FE10E942172998992FF15C0812F0D
:10898000877F803811F0103979F480E20E942172DB
:108990000BC0223009F062C98B0160C915E21CCC02
:1089A00091E09093CB08A7CFA1960FB6F894DEBFC5
:1089B0000FBECDBFDF91CF911F910F91FF90EF9030
:1089C000DF90CF90BF90AF909F908F907F906F90EF
:1089D0005F904F903F902F900895FF920F931F93B9
:1089E000CF93DF930E94831A182F8093EA0663E6E1
:1089F0008EE598E061D861E68EE798E05DD8CEE537
:108A0000D8E0E7EAF3E021813281499159918E8DD6
:108A10009F8D481B590B8081811103C05195419551
:108A20005109240F351F293E83E038073CF42831D3
:108A30008CEF38072CF428E13CEF02C028EE33E03D
:108A400032832183359628E0CE37D207E1F600E065
:108A5000023071F40F5F0430D9F786E00E944A5D5E
:108A600081E0DF91CF911F910F91FF900C942172C3
:108A7000602F812F0E942213EC01F12C602F8F2D8B
:108A80000E94E212853F21E092073CF4AC014C1BAE
:108A90005D0B602F8F2D0E943613F39484E0F81243
:108AA000EDCFD8CF8F929F92AF92BF92CF92DF92AD
:108AB000EF92FF920F931F93CF93DF9390914F0606
:108AC000292F2F70F22E1092560120915A08211151
:108AD000A5C09077813809F48BC088F4843209F4FA
:108AE00041C038F4823209F462C0833209F452C0C2
:108AF00095C0853209F440C0803809F18FC08438B0
:108B000041F160F4823809F460C0833809F086C00E
:108B100080EC90E30E94931983E85CC08E3879F072
:108B20008F3B09F46DC0853809F078C081E08093EF
:108B3000FE0787E893E30E94931985E828C092E036
:108B400090935A0810925B080E94DC6810920B0206
:108B500065C081E08093FE0783E69AE20E94931944
:108B600084E815C042E0F41259C08091E1088F5F9B
:108B7000833054F080E008C052E0F5124FC080917D
:108B8000E108815087FD82E08093E10847C00E94A0
:108B9000DC6844C0F39483E08F1508F4F12C9F291E
:108BA00090934F0681EA0E944A5D83E126C0FF2030
:108BB00011F0FA9402C0E3E0FE2E9F2990934F0635
:108BC00081EA0E944A5D84E118C080EC90E30E9433
:108BD000931982E8DF91CF911F910F91FF90EF9051
:108BE000DF90CF90BF90AF909F908F900C94DC68F7
:108BF0000E9477310E947D3187E10E9421720EC070
:108C000081E00E94DC6883E00E94DC6882E00E94D0
:108C1000DC6881E08093CD081092E10880915F02CA
:108C20000E943E19C82F882329F08091CD08811118
:108C300001C0D3DEC093CD0890913D0180913C06E8
:108C4000981710F4C6E001C0C4E080E00E944C33E5
:108C50004C2F406860E185E20E94366646E568E197
:108C600086E20E94B46324E040E060E18FE50E9468
:108C70009B2320E040E068E183E30E94ED110E9425
:108C8000831A882379F0482F60E186E20E94EE2D56
:108C900029E046E26FE085E20E94B866D0E07FE11D
:108CA000E72E3EC000E020915D0240E350E160E12C
:108CB00086E20E94DA6380915C0280FFEFCF4CE293
:108CC00050E160E188E30E942764E8CF559547951D
:108CD000559547954423B9F1443E0CF444EE142FC6
:108CE0004D310CF01CE18FEF8D0F46E3823008F020
:108CF00040C064E08C2F0E94C764D13069F180913C
:108D00005C0280FF29C06E2D611B635027E047E0A5
:108D10008DEF8C0F0E949866DF5FD43009F43DC060
:108D20008D2F0E948E10E82FF0E0E95DFF4EC49178
:108D30006D2F8091EA060E942213AC0197FFC6CFE7
:108D40004D5F5F4FC3CF1816190614F441E0C4CF2E
:108D5000492F440F440BC0CF43E06EE18FEF8C0FDF
:108D60000E94C76443E06EE181E08C0F0E94C764FB
:108D7000CACF6BE385EE8C0F0E94C5640FEF0C0F1A
:108D800043E06AE3802F0E94C56443E06CE3802FD8
:108D90000E94C564C10F6BE3B8CF91E09F1508F442
:108DA00089C00AED17E0E12C29E1D22E3BE1C32E68
:108DB000F801C191D1918F018E2D8370F1E0FF16E2
:108DC00039F18C9D802D112423E02E1510F068E2DE
:108DD00001C060E39E01D7FF02C0215E3F4F95E0D6
:108DE000359527959A95E1F7AE01421B530B9A01F1
:108DF000D7FF02C0C158DF4FAE01440F452F441FBB
:108E0000550B420F531F20E28F5D0E9414664DC028
:108E100053E05E1518F0A2E2AA2E02C0FEE5AF2EC6
:108E2000B82EBB0CBB0CB80EE6E28E2E8B0C8091DC
:108E3000610281FF03C060E075E002C060E074E0A1
:108E4000AE01D7FF04C0442755274C1B5D0BD49EB1
:108E5000F001D59EF00D1124CF019E5F0E94077A8C
:108E6000962E89E1861714F479E1972E25E543E3E0
:108E7000682D87EE8A0D0E948A6445E064E26B0DDE
:108E80008A2D0E94C7641C161D0614F4A39401C009
:108E9000A91867E26B0D492D8A2D0E94C5646B2DC0
:108EA0006B5D492D8A2D0E94C564E39498E0E91218
:108EB0007FCF27C0E2E0FE1218C00E940C2860910C
:108EC000E108C1E0C60F662329F0862F880F680FDE
:108ED000660F6D5F8AE00E94933A6C2F660F6C0FED
:108EE000660F84E60E94933A0CC024E041E068E2F9
:108EF00089E30E949B2320E840E060E38FE00E942A
:108F0000ED1180915A08882399F14EE06FE183E5D5
:108F100095E10E94CE2910925908813049F590912F
:108F20005C08911103C083E69AE220C0913039F4C5
:108F30009093FE071092380881EC90E517C09230AC
:108F400061F480935908E0914A01F0E0EE0FFF1FB1
:108F5000E35BFE4F8081918109C0933019F487E86B
:108F600093E304C0943021F480EC90E30E949319C1
:108F7000DF91CF911F910F91FF90EF90DF90CF90F5
:108F8000BF90AF909F908F900895AF92BF92CF9275
:108F9000DF92EF92FF920F931F93CF93DF936C01B9
:108FA000162FCBE9D6E00E94831AF82E4091CC0808
:108FB0008417E1F1442361F0EFEFE40F8AE0E89FCA
:108FC000F0011124E75EFA4F808182958F7001C015
:108FD00080E0FF2061F0EFEFEF0D9AE0E99FF001F4
:108FE0001124E75EFA4F90819F70891718F088234B
:108FF000D9F001C0892F682F70E080E092E00E94D4
:10900000077A7A83698381E090E09C01042E01C095
:10901000220F0A94EAF73881322B0F2C01C0880FF7
:109020000A94EAF7382B3883F092CC081062E12ECC
:109030008881882329F11C821B828E01B12CAA24ED
:10904000A39488818A21A1F0BF1491F0B092EA061E
:109050008B819C81F80125813681820F931F9C832F
:109060008B836E2DC6010E945C3DFE2DFF7DEF2E91
:10907000AA0CB3940E5F1F4F85E0B812E2CF09C06F
:10908000FE01EF0DF11DEF0DF11D80E094E69683DA
:109090008583FE01EF0DF11DEF0DF11D8B819C818C
:1090A00025813681820F931F9C838B83F092EA0681
:1090B0006E2D6064C6010E945C3D8881882309F49E
:1090C0003EC080913C018823D1F1FE01B0E0A1E0D7
:1090D00080E094E62581368118814A2F412331F1C1
:1090E00000913C0169817A81069FA001079F500D84
:1090F0001124BF1559F04217530718F4241B350BE0
:1091000017C02A2F20952123288310C0BC01621B81
:10911000730B4617570718F4240F351F09C02A2F61
:1091200020952123288320E034E602C020E030E0AF
:1091300036832583AA0FBF5F3296B53059F6DF918B
:10914000CF911F910F91FF90EF90DF90CF90BF9044
:10915000AF9008950F939CEF940F9D3138F450E039
:10916000425051098E5E0F910C941466413208F002
:109170004D51022F242F41ED55E10E94DA630F91EA
:109180000895CF92DF92EF92FF920F931F93CF93A8
:10919000DF93C82E8BE39DE00E94F8244091E908FC
:1091A00050E04F5F5F4F60E08EE40E944266C091E6
:1091B000E90889E0C89FE0011124CC53DA4F8C8183
:1091C000877011F04AE001C049E06C2D89EC98E00D
:1091D0000E947C251091C90816301CF462E17DE0E4
:1091E00002C06DEE7CE088E00E941164F090FC0704
:1091F00016300CF0ACC00E945128111107C06EE26D
:1092000088810E943A1488832F2D01C020E0488174
:1092100068E080E60E94B91088818823D9F08150E7
:109220000E943D126C0168EE7CE088E00E941164AF
:109230004881453250F0455202E0E02E00E09601B0
:1092400068E088E40E94A92305C0A60168E088E4DC
:109250000E944266113039F466E089810E943A1416
:1092600089830F2D01C000E02981253018F447EED5
:1092700055E103C0255048ED5CE060E18EE40E94BA
:10928000DA63123081F484E680933E0122E040E00C
:109290005DE760E073E88D819E810E9468139E8384
:1092A0008D832F2D01C020E048818D819E81453224
:1092B00050F04552B2E8EB2E022F9C0168E188E79E
:1092C0000E94A92305C0AC0168E188E70E941466EA
:1092D000133051F440915701642F61958A810E94A7
:1092E00037148A832F2D01C020E04A8160E280E696
:1092F0000E949D11143031F461E28B810E943A1476
:109300008B8301C0F12C2F2D4B8168E280E622DF98
:1093100021E0153009F020E04C81469546954695B0
:10932000437068EB7CE080E30E940B258370880F1C
:10933000880F880F9C81977E982B9C83DF91CF911B
:109340001F910F91FF90EF90DF90CF90089521E053
:10935000163009F020E04C8142954695437062EA50
:109360007CE088E00E940B2583708295880F807EC8
:109370009C819F79982B9C8321E0173009F020E095
:109380004C8147FB442740F966E97CE080E10E947C
:109390000B254C8180FB47F94C83042F077021E09B
:1093A000183009F020E0402F60E87CE088E10E945E
:1093B0000B2587709C81987F982B9C83801711F0D8
:1093C00018861F828C81877009F466C065E77CE08F
:1093D00080E20E9411648C818770813009F041C065
:1093E000193069F422E04FEF51E060E070E08F81C6
:1093F00098850E94681398878F830F2D01C000E025
:109400004F8158854C3FE1E05E077CF0202F47EC10
:1094100054E160E28CE60E94EC634F814B5C202FAC
:1094200060E288E70E94296333C0453FF1E05F07AF
:109430003CF0445F202F60E28CE60E94642428C048
:10944000202F60E288E70E941466002309F180E87B
:10945000C81204C08F8198850E947A141092020865
:1094600017C08230A9F4193059F44FE060E08F81C1
:109470000E943714482F50E058874F830F2D01C0AA
:1094800000E02F814EE556E160E28AE50E94DA6352
:10949000AAE0DA2E08E203C0F9E0DF2E00E26EE671
:1094A0007CE0802F0E9411644D2D50E0E12FFF27BA
:1094B000E7FDF095E417F50781F4E0E8CE120EC061
:1094C00089E0FE0111928A95E9F7109202081A309C
:1094D00029F488E08093C90801C0F12C2F2D44E6BF
:1094E0005CE0602F88E4DF91CF911F910F91FF9096
:1094F000EF90DF90CF900C94EC63CF93C62F20E0D9
:109500004EE1682F80E00E944D6480910B0280380C
:1095100031F4C0938F0D84E391E20E94931910926D
:109520000208CF9108951F93CF93DF93D82F162F62
:10953000237021F0223021F4C1E803C0C0E801C04B
:10954000CDE2612F8D2F0E94B4634C2F612F86E0F6
:109550008D0FDF91CF911F910C94B463909103080C
:10956000282F291B181644F4273014F0865005C004
:1095700027FD03C0892F01C080E080930308089570
:10958000CF92DF92EF92FF920F931F93CF93DF93CF
:10959000C82F8CE295E10E94F8244FE06C2F8DEDEE
:1095A00098E00E947C25F090DD088F2DD7DFD82E23
:1095B000C03621F0C43611F0CE3269F4F7FC0BC08E
:1095C000F092E7088C2F0E94DC6810920B0283E275
:1095D0009CE30E94931988E0E82E0F2D112707FDC8
:1095E0001095CD2DD0E0CC24C3940C171D0709F0A5
:1095F000C12C2C2D40E453E16E2D80E00E94EC63E1
:10960000AE014F5F5F4F88E08D1510F486E101C019
:1096100081E12C2D6E2D0E94146688E0E80ED39413
:1096200080E4E812DECFF7FC05C0F092E70884E69C
:109630000E94C83BDF91CF911F910F91FF90EF9057
:10964000DF90CF9008956F927F928F929F92AF920A
:10965000BF92EF920F931F93CF93DF9348E0682F51
:109660008CED98E00E947C2567EC74E180E00E941C
:109670001164C091E90841E34C0F60E08CE00E9466
:10968000B463A090DC088A2D69DF782E45E24C0F88
:1096900092E0E92E00E020E030E060E080E30E940C
:1096A000A923409103086CEF72E188E00E941664E0
:1096B00018E0BB24A7FCB0948BE0C89FE001112404
:1096C000C257DA4F4E01E7E08E0E911C23E0622E66
:1096D000472D50E0A416B50619F40091FC0701C00F
:1096E00000E0872D90E08930910508F093C0805804
:1096F0009F4FFC010C94587A202F4881612F82E4FF
:109700000E94B910002309F485C06EE288810E948E
:109710003A1488837FC001116092E80824E0A40114
:10972000612F8091D9070E948A2C74C049815A8187
:10973000202F612F8EE40E941466002309F46AC072
:1097400022E040E05DE760E073E889819A810E9451
:1097500068139A8389835EC0402F6B81812F0E949A
:1097600075288B8357C0402F6C81812F0E947528EC
:109770008C8350C0002329F067E08D810E943A1449
:109780008D832D814DEC54E1612F88E40E94DA63D2
:1097900041C0002349F08E8161E081700E943A143B
:1097A0009E8180FB90F99E838E8180FF02C04DE2F6
:1097B00001C04BE2202F612F88E40E9429632AC058
:1097C000002361F08E81869562E083700E943A14D6
:1097D0008370880F9E81997F982B9E834E8146953A
:1097E000437050E0202F612F84E50E94146612C060
:1097F00021E0A416B50609F020E04E8143FB442782
:1098000040F96EEE72E1812F0E940B259E8180FB54
:1098100093F99E837394185F103409F059CFDF9148
:10982000CF911F910F91EF90BF90AF909F908F902D
:109830007F906F9008956F927F928F929F92AF92D8
:10984000BF92CF92DF92EF92FF920F931F93CF932D
:10985000DF93C82E8091E5080E94A810EC014FE02C
:109860006C2D8AED98E00E947C258EEB92E10E949F
:10987000F82420E0488160E08A5F0E94E710A09011
:10988000DA088A2D6BDED82E4091030868E372E176
:1098900088E00E94166438E0F32EBB24B39444E0C1
:1098A000942E50E8852EAD1003C0E090FC0701C057
:1098B000E12C0D2D10E00031110508F097C1F801E1
:1098C000E757FF4F0C94587A19812E2DAE016F2D5A
:1098D00084E50E94E728153231F419851295169512
:1098E00017701B5D03C0163208F01A5FEE2009F4F2
:1098F0007DC147E361E0812F0E943714853268F013
:109900008C3210F0865009C085528295880F807E77
:1099100099859F71982B998785E2898367C12E2D40
:109920004A816F2D80E60E94C2248A835FC12E2D5A
:1099300048856F2D80E60E94C224888757C18F8199
:109940004E2D6F2D83FB882780F90E943D259F8136
:1099500080FB93F909C199818F81953080F486FB52
:10996000882780F94E2D6F2D9B2D981B892F0E94E3
:109970003D259B2D981B8F8190FB86F91FC086FB90
:10998000112710F969E272E18F2D0E9411644E2DAA
:109990006F2D812F0E943D259F8180FB96F9E4C0A9
:1099A0008F8181704E2D6F2D9B2D981B892F0E94CA
:1099B0003D259B2D981B8F8190FB80F98F8316C1CD
:1099C0008F8187FD08C08C81855E863340F410E06E
:1099D00047E152E107C011E04DE152E103C012E05E
:1099E00043E252E12E2D6F2D86E00E94EC63EE20C3
:1099F00009F4FCC062E0812F0E943A14181709F4A0
:109A0000F5C0823011F48C8201C01C829F8180FBE2
:109A100097F9AAC08F8187FF09C004E62CE94C8121
:109A20006F2D88E40E947C248C83E0C04C818BE104
:109A3000840F8733B8F010E8140F2E2D2064412FC7
:109A4000552747FD50956F2D86E60E941466EE203F
:109A500031F044E66CE9812F0E943714182F10581A
:109A60001C83C4C02E2D6F2D8CE00E945728EE2041
:109A700009F4BCC046E160EF8C810E9437148C83EE
:109A800090E6C912B3C087303CF087508093E70856
:109A900083E29CE30E9493198C8187FFA7C0809585
:109AA0008093E70883E29CE30E9493199FC001E042
:109AB000E11001C000E02E2D4B816F2D8EE40E943D
:109AC00092288B8393C0E1109092E8080FE310E096
:109AD0007724739466246A946F0C99859F719721FB
:109AE00021E009F020E040E3410F6F2D802F0E941C
:109AF0002963EE20E9F08091D907811319C029E08C
:109B000048E0662D8FEF800F0E94B86680E2C8168D
:109B100019F09EE2C9120CC08985972D98279F7174
:109B2000807E892B898782E00E944A5D109202081C
:109B3000770C1F5F095F153081F658C01F811295A1
:109B400013702E2D412F6F2D8EE40E947225EE2072
:109B500009F44CC063E0812F0E943A14837082950F
:109B6000807F9F819F7C982B9F8340C021E08BE06A
:109B7000A81220E04F81469543706BEF71E18F2D65
:109B80000E940B258370880F9F81997FECCF4D81B8
:109B900042954F706E2D8F2D0E94A4218295807F5B
:109BA0009D819F7009C04D814F706E2D8F2D0E9439
:109BB000A4218F709D81907F982B9D8317C04E812B
:109BC00042954F706E2D8F2D0E94A4218295807F2B
:109BD0009E819F7009C04E814F706E2D8F2D0E9407
:109BE000A4218F709E81907F982B9E83D39498E0C0
:109BF000F90E80E4F81257CEDF91CF911F910F91AB
:109C0000FF90EF90DF90CF90BF90AF909F908F909C
:109C10007F906F9008952F923F924F925F926F9234
:109C20007F928F929F92AF92BF92CF92DF92EF92EC
:109C3000FF920F931F93CF93DF93A82E8CE791E1B0
:109C40000E94F8248091D507882301F10E94EC241A
:109C5000882331F01CF072E6A72E02C063E6A62E20
:109C60002091D908211103C083E6A81661F030E0E5
:109C70008091D707992787FD90952817390721F4F8
:109C8000E2E6AE1201C0A12CA0920B0280915A080C
:109C9000811107C04091D7076A2D89ED98E00E9495
:109CA0007C256090D90880910B02803641F08F3B73
:109CB00019F08E32D1F403C01092D50716C09091DE
:109CC000D507992339F01092D50710920208109207
:109CD00038080BC090915A08911107C00E94DC68A7
:109CE00010920B028824839401C0812C862D36DCCF
:109CF000582E80915A08811110920B028091D5073D
:109D00008823E1F080910B029EE9980F9230B0F425
:109D100001E0823609F000E01091E508812F0E94F1
:109D2000A810EC01111175C101117DC1888182302B
:109D300010F08150888382E00E944A5D77247394FA
:109D4000B12C912CC52CD12C892D0E94A810EC018E
:109D5000B51488F06B2D70E06C197D0967307105C2
:109D600054F46F5F7F4F660F660F660F20E0472D3C
:109D700081E00E94E710FFE1F91508F4B8C02880DF
:109D80002710B5C02A96492C7E018AE0E81AF1080E
:109D9000B51408F49FC08B2D90E08C199D09873075
:109DA00091050CF088C00196382E330C330C330C1F
:109DB0008091D507811112C06B1010C04092E50848
:109DC0002092E308882031F010925B08E1E0E093F4
:109DD0005A08A12C11E080915A08811110E09414C6
:109DE00059F0F70127812695237000E047E751E1FC
:109DF000632D83E10E94DA6320E0A701632D80E3F5
:109E00000E94E728212F8E0108501109F801408196
:109E1000632D8DE20E94C224F8018083FE013797F2
:109E20004081442329F020E0632D88E40E949D11A5
:109E3000FE01369740814423B1F0F701878187FF07
:109E400003C020E044E60BC08BE1840F20E08733A1
:109E500028F4632D80E60E94572805C045E4632D51
:109E600080E60E942963F7018681811102C040E2E9
:109E700001C043E5F7018581882329F0433511F4BA
:109E80004AE201C044E4632D89E70E94B4638091F3
:109E9000D5078823F9F08091E40884111BC020E0E5
:109EA00046E6632D88E10E944D644092E508B09239
:109EB000D9086B2C0FC0079769F48091D5078823C8
:109EC00049F08091E408841105C08091D9088F5F22
:109ED0008093D908B3944394F0E24F1669F12A961F
:109EE000FE013A978081821509F44ECF25C06B1090
:109EF00021C07092E3089092E5086B2D6C19660FF3
:109F0000660F660F695F29E049E180E00E94B8664C
:109F1000882081F00E94132981110CC060E080919B
:109F2000E5080E94C3211092D5078BE19CE40E94B2
:109F3000931908C0B394492C739481E1781611F0F9
:109F4000942C02CF80915A08882309F44CC0A09227
:109F50000B024BE06FE387E394E10E94CE299091DE
:109F60005C088130D1F5913079F40E941329811178
:109F70000DC08091E5088F5F8093E50860E00E9446
:109F8000C3211092D50702C0923018F48BE19CE4F3
:109F90000EC0943079F48091E5088093D6078091C3
:109FA0000B020E94DC6810920B0287E499E20E9487
:109FB000931911C0953011F48FEFEFCF923041F427
:109FC0008091E5088F5F8093E50861E00E94C321DE
:109FD00081E08093D50710925A088091E50880931C
:109FE000E40810920208BA94B092D707DF91CF919B
:109FF0001F910F91FF90EF90DF90CF90BF90AF90A7
:10A000009F908F907F906F905F904F903F902F9098
:10A010000895113208F092CE103219F4002329F07D
:10A020008DCE002311F01F5F01C01150812F0E94BF
:10A03000A810FC0198818FEF890F803108F07ECE47
:10A040002081213108F07ACE291302C08BE009C0AB
:10A05000002309F46FCE903108F06DCE9F5F988396
:10A060006ACE815029F09081288121939993F9CF6C
:10A070001093E40860CE9F92AF92BF92CF92DF928E
:10A08000EF92FF920F931F93CF93DF93D82F8EE51C
:10A090009CE00E94F82447E06D2F88EC98E00E9435
:10A0A0007C25C091C8088C2F59DAA82EDE3211F019
:10A0B000D03659F4C8304CF4C093E9088D2F0E9473
:10A0C000DC6881EC98E40E949319E8E0BE2ECC2E67
:10A0D000DD24C7FCD094F9E09F2EEA2CF12C9E9C45
:10A0E000E0019F9CD00D1124CC53DA4FA7014F5FA4
:10A0F0005F4F0BE51CE020E06B2D81E10E94FE2408
:10A1000020E048816B2D8EE10E94B91020E04A8149
:10A110006B2D86E30E949D1120E04B816B2D8EE418
:10A1200019D89C819770913021F0923039F441E434
:10A1300001C043E26B2D82E70E94B4638C81887179
:10A1400029F048E46B2D88E70E94B463CE14DF0445
:10A1500031F420E048E76B2D80E00E944D6488E0F8
:10A16000B80EA39480E4B812B8CFDF91CF911F91BD
:10A170000F91FF90EF90DF90CF90BF90AF909F90A6
:10A1800008953F924F925F926F927F928F929F922B
:10A19000AF92BF92CF92DF92EF92FF920F931F93F5
:10A1A000CF93DF9392E09093FB0746E067EC78E073
:10A1B0000E945521E82E4091EA084150682F87EC13
:10A1C00098E00E947C2580915708863091F038F401
:10A1D000813061F08530A1F482E09EE20FC08930C9
:10A1E00059F08A3069F48BE390E508C08BE09EE477
:10A1F00005C080EC9AE402C089E097E20E949319BE
:10A20000F090C708C091FC070091570810E00E308D
:10A21000110510F00C94DD5BF801E756FF4F0C942C
:10A22000587A80E695E10E94F8248DE08093EA0850
:10A2300041E04F0D66E081E49CE00E9401220C9415
:10A24000DD5B81ED93E10E94F8242AE02F1510F0E8
:10A250000E94512880E18093EA0885E08F1508F478
:10A26000E6C0F11003C089E08093E80801E0F11036
:10A2700000E02AE04BE452E068E08091D9070E94B8
:10A280008A2C91E0F91210C0E0E6EE1204C0809131
:10A2900055020E94901461E3809155020E943A1485
:10A2A000809355022C2F01C020E04091550250E0D0
:10A2B0004C5F5E4F00E31CE060E188E50E94FE24F5
:10A2C0006BEF7BE088E10E94116411E0D0E08091A7
:10A2D0007F0682FF20C08EEF8D0F8430E0F4409126
:10A2E000FA04D23051F4242F30E035952795359576
:10A2F000279545E468E18EE40CC0D43071F4242F36
:10A3000030E094E0359527959A95E1F749E468E1C6
:10A310008AE509D902C081E001C080E090917F0602
:10A3200094FF0CC0D63039F420910C0641E468E16A
:10A3300086E6F9D818C0D73009F4D8E0882399F018
:10A340008091FA04812301E009F400E04D2F50E0F0
:10A350004A53594E8D2F880F8D0F880F21E068E1E9
:10A360008E5B0E94B663110FDF5FD83008F4AFCF69
:10A37000F2E0FF121DC029E048E367E181E40E949A
:10A38000B86620E6E21619F08EE2E81211C08E2DB2
:10A390000E94DC680E94BA128093FA0485E20E944F
:10A3A000BB6880930C061092020882E00E944A5D0E
:10A3B00041E093E0F91240E08091BC0560E28295B3
:10A3C00081700E943D259091BC0580FB94F990938B
:10A3D000BC05E4E0FE1209C0C06264E68091FB04A3
:10A3E0000E943A148093FB0401C0C0E24091FB0438
:10A3F00050E02C2F68E288E70E94146621E0F5E027
:10A40000FF1220E04091C7044295469547706FEDDA
:10A410007BE080E30E940B258295880F807E9091DF
:10A42000C7049F71982B9093C7040C94DD5B2AE0BE
:10A430002F1508F487C068E97BE088E00E9411646A
:10A4400041E086E0F81240E08091610268E0869584
:10A4500081700E943D259091610280FB91F990935B
:10A46000610291FF1BC0C091BC05C5FBCC27C0F9A0
:10A4700021E097E0F91220E04C2F68E87BE080E1D2
:10A480000E940B2581709091BC0580FB95F99093FB
:10A49000BC058C1791F00E94A8190FC0E5EAF3E003
:10A4A000808187FD1082818118160CF41182359607
:10A4B00023E0E53FF207A0F3D6CFC091BC05C6FB71
:10A4C000CC27C0F941E088E0F81240E068E18C2F29
:10A4D0000E943D2581709091BC0580FB96F9909378
:10A4E000BC058C130E94A8190E94AF10882311F09C
:10A4F00041E801C040E860E280E60E94B46341E0C8
:10A5000099E0F91240E080915C0268E281700E945B
:10A510003D2590915C0280FB90F990935C0241E0B4
:10A52000EAE0FE1240E080915C0260E38295817077
:10A530000E943D2590915C0280FB94F990935C020F
:10A540000C94DD5B64E57BE088E00E94116421E00F
:10A55000FBE0FF1220E040915D0262E37BE088E0D7
:10A560000E940B2580935D022CE0F21204C001E0F2
:10A57000C11103C001C0C0E000E02C2F40915F0278
:10A5800060E186E60E94922880935F0241E08DE0C0
:10A59000F81240E080915C0268E183FB882780F933
:10A5A0000E943D2590915C0280FB93F990935C02A0
:10A5B00041E09EE0F91240E08091570260E286950A
:10A5C00081700E943D259091570280FB91F99093F4
:10A5D0005702DAE2CD2EDBE0DD2EE6011FE301E0DB
:10A5E00086E0B82EAC2EAC18FE014491809160023A
:10A5F000802321E009F420E068E2812F0E94296392
:10A60000FFE0FF121DC0B092E8088091D9078A11BF
:10A6100017C029E048E067E28FEF810F0E94B8661B
:10A6200020E2E21619F08EE2E8120AC08091600280
:10A6300080278093600282E00E944A5D10920208A7
:10A64000000F2196195F103769F60C94DD5B80ECE2
:10A6500096E10E94F8248AE08093EA0894E09F152E
:10A6600028F00E945128E12C10E003C0EE24E3946E
:10A6700015E0E5E0EE9EE0011124C050DE4FD090E1
:10A68000FC0766E778E088E00E94116441E34E0D24
:10A6900068E08EE10E94B463F11202C02D2D01C06A
:10A6A00020E048815981022F68E087E40E945266C9
:10A6B000F11214C08CE380933E014CE364EC80E023
:10A6C0000E94371448815981480F511D87FD5A95C2
:10A6D0005983488357FF02C01982188281E0810F95
:10A6E000F81207C063E18A810E943A148A8341E02C
:10A6F00001C040E0E11002C021E001C021E860E1BA
:10A700008CE30E94ED1182E0810FF81205C0DD207C
:10A7100019F02D2D03E002C020E002E04B8168E13A
:10A720008AE50E9492288B8321E083E0810FF81252
:10A7300020E04C816EE578E080E20E940B258C835E
:10A740001C5FF112D12CE11003C04091BA0502C088
:10A750004091BB05DD2011F003E001C002E02D2D8A
:10A7600068E28FE40E949228E11003C08093BA054A
:10A7700002C08093BB05E0E0F2E08081918190937C
:10A78000590280935802828180935602838180937C
:10A79000C60480915702948190FB80F98093570200
:10A7A000858196819093F7048093F6048781809346
:10A7B000F80480858093F9048091BC05918590FB15
:10A7C00087F98093BC05F9C781E495E10E94F824DC
:10A7D00086E08093EA08C091FC076FED7AE088E09C
:10A7E0000E94116421E0F11020E040916102429545
:10A7F0004695477067EC7AE088E00E940B258295C9
:10A80000880F807E909161029F71982B90936102D6
:10A81000F1E0FF1209C064E2809162020E943A14E2
:10A82000809362022C2F01C020E04091620260E11F
:10A8300086E60E94B91022E0F21208C064E6809118
:10A8400063020E943A148093630201C0C0E02C2F7F
:10A850004091630268E184E50E94722541E083E053
:10A86000F81240E08091610260E282FB882780F963
:10A870000E945C259091610280FB92F990936102A5
:10A8800041E094E0F91240E08091610268E283FBCC
:10A89000882780F90E945C259091610280FB93F9E2
:10A8A0009093610241E0E5E0FE1240E08091610298
:10A8B00060E3829581700E945C259091610280FB2B
:10A8C00094F99093610279C789E395E10E94F82495
:10A8D00085E08093EA0810925601D091E60820E0C6
:10A8E000F11009C043E060E08D2F0E942D14D82F95
:10A8F0008093E60821E041E04D0F68E080E00E948F
:10A90000B9108D2F0E94CB24182F00E0282F4BEB7D
:10A910005AE068E08AE20E94DA636BE97AE088E054
:10A920000E941164ED2FF0E0EE0FFF1FEC5DF74F7A
:10A9300040815181453651052CF44C395F4F24F04C
:10A94000C2E003C0C0E001C0C1E08D2F0E941B180F
:10A95000811106C0CC2329F081E0F81202C002C0A8
:10A96000C0E080E0EE24E39400E0212F48E168E1BC
:10A970000E942A2CC13011F081E0F81280E0E12C15
:10A9800000E0212F48E160E30E942A2CCC2319F03B
:10A9900081E022E0F21280E0EE24E39401E0212F36
:10A9A00048E268E10E942A2CC13019F081E092E06F
:10A9B000F91280E0E12C01E0212F48E260E30E94DF
:10A9C0002A2C81E0E3E0FE1280E0E12C00E023E6A7
:10A9D00040E36EE10E942A2C81E0F4E0FF1280E067
:10A9E000E12C00E022E648E36EE10E942A2C8091EF
:10A9F000E6080E941B18882311F08CE301C08CE547
:10AA000040E460E00E94C76481E08093440961E013
:10AA10008CE50E946A3B8091E608E82FF0E0EE0F9B
:10AA2000FF1FEC5DF74FC081D181BE010E94F63A55
:10AA30008C0189E18C9F90018D9F300D112437FF8F
:10AA400002C021503F4F532F550F550B432F60E34A
:10AA500082E70E94426689E1809F9001819F300DCC
:10AA6000112437FF02C021503F4F532F550F550B74
:10AA7000432F68E084E50E944266CE01409697FF2E
:10AA800002C0CE018F967C01A5E0F594E794AA95CB
:10AA9000E1F7E8016096D7FF02C0E801AF96F5E064
:10AAA000D595C795FA95E1F7D195C195D1096C2F48
:10AAB000635E47E08CE58E0D0E94C7646C2F605E7C
:10AAC00047E089E58E0D0E94C5641092440975C661
:10AAD000E0905A022E2D2F70E22ED22E81E0281700
:10AAE00041F092E0291739F0E5E02E1731F0C4E08B
:10AAF00005C0C6E003C0C3E001C0C7E08DE095E13A
:10AB00000E94F824C093EA08D091FC07C091D907AD
:10AB10006CE87AE088E00E941164F11013C0809123
:10AB20005C0267E08295869587700E943A14829550
:10AB3000880F807E90915C029F71982B90935C02AD
:10AB400021E001C020E040915C02429546954770AB
:10AB50004F5C68E082E70E942963EE2049F08DE0B7
:10AB60008E0D8F70CC24C394823020F0C12C02C093
:10AB7000CC24C394F1E0FF1202C0CC2311F000E01A
:10AB800001C00D2F2E2D40E65AE060E184E20E94C4
:10AB9000DA63CC2079F16CE57AE080E10E941164FF
:10ABA00021E0F21202C0C13011F000E001C00D2F0F
:10ABB00020915B022E5F4EE35AE060E188E40E9440
:10ABC000DA6381E0F81202C0C23011F020E001C067
:10ABD0002D2F40915E0292E34902A0011124445DB1
:10ABE0005E4F60E180E70E941466E1E0FE1267C0FC
:10ABF00082E01AC040915B02F5E0EF1201C04F7095
:10AC000021E0F21202C0C13011F020E001C02D2F6E
:10AC1000552747FD509507E31AE060E18EE70E9453
:10AC2000FE2481E0F81284C08093E8088091010836
:10AC3000882309F451C0C13051F018F0C23031F10D
:10AC40002FC066E08E2D0E943A14D82E29C0CC2049
:10AC500019F044E06EEF13C095E0E9120EC0809148
:10AC60005B024FE060E08F700E94371490915B02AE
:10AC7000907F980F90935B0213C04CE760E0809147
:10AC80005B020E94371480935B020AC0CC2041F023
:10AC90004AE06CEF80915E020E94371480935E025E
:10ACA00080915A02982F9F70807F2D2D2F70822BBC
:10ACB00080935A029D1581F010925B020DC0E2E074
:10ACC000FE120CC044E16CEE809164020E943714C5
:10ACD0008093640221E203C0CC2051F120E2409134
:10ACE0006402F5E04F02A00111244F515F4F08E2CA
:10ACF0001AE068E18CE40E94FE246FE17AE080E2D1
:10AD00000E94116421E083E0F81220E0409161028A
:10AD1000417065E17AE080E20E940B25909161022A
:10AD200080FB90F990936102E4E0EE2E18E203C0FC
:10AD300072E0E72E18E195E0D912EFC069EE79E0F4
:10AD4000812F0E941164D0903C0521E0FE1020E08C
:10AD50004D2D4F7161E979E0812F0E940B25909173
:10AD60003C05907E980F90933C0500915B02492F23
:10AD7000552747FD50952D2D30E04217530749F4D4
:10AD8000402F50E064E0559547956A95E1F747708C
:10AD900001C040E088E0810F31E03E0D9F7179F005
:10ADA000933081F0953089F0973091F0993099F097
:10ADB0009B30A1F09C30A9F461E079E014C065E714
:10ADC00079E011C067E679E00EC06BE579E00BC071
:10ADD00064E379E008C062E279E005C06FE079E001
:10ADE00002C069EF78E021E0F31220E00E940B2519
:10ADF0000F78D02EE0E18E9FD00C1124D0925B0210
:10AE000040E1B42EB10E52E0C52ECE0CAD2CAA1CE2
:10AE1000AA24AA1CFC1002C0CC2311F000E001C03F
:10AE20000D2F2A2D4FEE58E06B2D84E20E94DA633D
:10AE3000FC1002C0C13011F020E001C02D2F409164
:10AE40003D05552747FD50956B2D8EE70E941466F2
:10AE500067EE78E08B2D0E941164FC1022C081E027
:10AE60008093E808C1110FC0809101088823C9F0C0
:10AE700061E08A2D0E943A149D2D9F778111906880
:10AE800090935B020EC0C13061F480910108882369
:10AE900041F04FE761E880913D050E9437148093AF
:10AEA0003D0528E1B22EB10E33E0A32EAE0CD090BA
:10AEB0003C05D6FACC24C0F8FA1002C0C13011F01B
:10AEC00000E001C00D2F2C2D43EE58E06B2D88E7DC
:10AED0000E94DA63FA101AC081E08093E808C11179
:10AEE00005C061E08B2D0E947D4A10C0C13071F415
:10AEF00080910108882351F061E08C2D0E943A1462
:10AF00009D2D9F7B8111906490933C0584E08E0D74
:10AF1000F81253C460E280E250C0F2E0DF1212C0C7
:10AF20006AED78E0812F0E94116421E0FE1020E09C
:10AF300040913C056BEB78E0812F0E940B258093BC
:10AF40003C053BC421E0D21238C461EA78E0812F8D
:10AF50000E94116421E0FE1020E040913C056FE565
:10AF600073E1812F0E940B2580933C0521E081E055
:10AF70008E0DF81220E040915A02429543706BE624
:10AF800073E188E0810F0E940B2583708295807F9A
:10AF900090915A029F7C982B90935A0282E08E0DDA
:10AFA000F81205C061E080E1810F0E947D4A83E0D4
:10AFB0008E0DF81202C460E288E1810F0E947D4A82
:10AFC000FCC38DE498E00E94F8248CE08093EA08AA
:10AFD00083E08093E808B090D9078F2D0E94AE4A95
:10AFE000982E98E0D92EF91003C08090FC0701C07C
:10AFF000812C4CE46D2D80E00E94B46388E08915BB
:10B0000010F448E301C041E3490D6D2D85E00E9435
:10B01000B46391E0B91629F0E2E0BE1629F0712C74
:10B0200001C0782CA12C02C0A82C712C492D50E015
:10B03000EA01CC0FDD1FC40FD51FCF55DB4FBB205E
:10B0400011F000E001C0082D2A812F7047EE55E174
:10B050006D2D8DE00E94DA638A818F700E94A210AC
:10B06000C82E81111CC0188115327CF015526981DF
:10B07000812F0E94FA229C0102E8E02E0A2D412F26
:10B080006D2D84E60E94A92323C04981552747FDE1
:10B0900050952A2D6D2D83E60E94146619C0F1E0AB
:10B0A0008F130DC0272D48816D2D86E30E949D11C1
:10B0B0002A2D49816D2D8DE40E949D1134C022E01E
:10B0C00082130DC02A2D49816D2D80E50E94B91093
:10B0D000272D48816D2D86E30E94B91024C0488138
:10B0E00047FF04C04095872D8062782E552747FD85
:10B0F00050954F5F5F4F09E418E0272D6D2D89E4CF
:10B100000E94FE24498147FF04C040959A2D906219
:10B11000A92E552747FD50954F5F5F4F2A2D6D2D66
:10B120008BE60E9414664A8142954F7049300CF0BC
:10B130004F5FE3E0BE1611F020E001C0282D6D2D19
:10B1400088E60E949D1180910108882309F462C05D
:10B15000882009F45FC0F1E0BF1631F1BF1698F006
:10B1600022E0B216D9F183E0B81254C08A816FE0B0
:10B1700082958F700E943A148295807F9A819F7089
:10B18000982B9A8347C08A816EE08F700E943A1490
:10B190008F709A81907F982B9A830E94A210C81674
:10B1A000C9F11882198236C091E0C91659F0C91642
:10B1B00090F0E2E0CE1679F0F3E0CF122BC043E638
:10B1C0006EEC04C040915701642F619588810E9404
:10B1D000371488831FC04EE260E0F8CF21E0C2162A
:10B1E00071F0C21648F082E0C81671F093E0C912FF
:10B1F00011C043E66EEC0AC04DE763E807C040911A
:10B200005701642F619502C04EE260E089810E947F
:10B21000371489839394E8E0DE0EF0E4DF12E3CE86
:10B22000CCC28CE495E10E94F82481E18093EA0885
:10B2300083E08093E808A090D9078F2D0E94AE4A42
:10B24000982E2FE02F15A0F0EF2DF0E0EE0FFF1F4E
:10B25000E652F84F4081518157FF02C04F5F5F4F68
:10B260005595479544525A4F60E08EE40E944266DD
:10B2700080910B02803819F58FE08F1540F14F2D2A
:10B2800050E0FA01E919F109EE0FFF1FE652F84FFD
:10B2900020813181A11013C085E0849FF001859F3A
:10B2A000F00D1124EB55FC4F8281882319F0319564
:10B2B000219531093483238382E0ECD3E7D458E02D
:10B2C000E52E65E0562E7AE0C72ED12C93C090E192
:10B2D000F912F5CF89E18093000880E80E94DC68CC
:10B2E0000E94ED44ECCFE92DF0E05E9EE0015F9E10
:10B2F000D00D1124CB55DC4FEE0FFF1FE652F84F57
:10B30000808191814A812B813C81442319F03195C0
:10B3100021953109821B930B833391050CF06EC08C
:10B320008E3C9F4F0CF46DC01DE266246394690C43
:10B3300020E0462D6E2D80E00E94E710412F6E2DFB
:10B340008BE40E94B4638091610281FF5EC03DE79F
:10B35000732EB12C44244A944E0C372C3194F9109E
:10B3600057C0AB1055C02091FC078091010888237D
:10B3700009F450C0222309F44DC010925601822EC8
:10B380008091FB04882309F453C00B811C810115B3
:10B39000110509F041C0C801B6010E94077A82E098
:10B3A000B81609F466C093E0B91609F486C0E1E066
:10B3B000BE1609F442C020624B815C816E2D8DE285
:10B3C0000E941466882059F022E048EE53E068E1BC
:10B3D0007CEF8B819C810E9468139C838B83B39448
:10B3E00024E0B212BCCF88E08E0D803409F47EC018
:10B3F000E82E962CE0E19E1276CF6AC0411103C080
:10B40000EEC14111ECC11FE790CF24E6722EA1CF0F
:10B4100020E0ABCF812CB4CF90E0801791075CF097
:10B42000919581959109081719070CF0B4CF03C0C5
:10B4300000E010E0B0CF8C01AECF18811456AB0104
:10B44000410F511D17FD5A954338FFEF5F0714F464
:10B4500043E85FEF6E2D88E40E941466882009F4AB
:10B46000BECF49E1632D812F0E9437148C59888308
:10B47000B6CF89818C59AB01480F511D87FD5A9574
:10B480004E37510514F04DE750E06E2D86E60E94D0
:10B490001466012B31F029E048E3642D82E30E9419
:10B4A000B866882009F49BCF8981472D67EE8C59B7
:10B4B0000E9437148456898392CF422F6E2D8A8141
:10B4C0000E945C2591E0811101C090E09A8387CFB2
:10B4D00021E0E0E1FE1220E080910008811181C1AD
:10B4E00048E358E06E2D82E10E94EC6366C188E279
:10B4F00098E00E94F82489E18093EA08C090D90777
:10B500008F2D0E94AE4AD82E88E0E82E90E1B92E09
:10B510008091C704D11021C0F11010C01092E8082A
:10B52000C091FC0760E18F710E943A148F71909175
:10B53000C704907E982B9093C70401C0C0E040914F
:10B54000C7044F7150E0485F5F4F08E118E02C2FAF
:10B550006E2D8CE60E94FE242AC18F719B2C981AB6
:10B56000CD2DD0E0FD1003C082E08093E808C1310A
:10B57000D1052CF4CC0FDD1FCA53DB4F04C0CC0F18
:10B58000DD1FC65DDA4F10E0FD1009C0C11207C013
:10B590000091FC07002321F0B2E0AB2E02C000E0D6
:10B5A000A12C9D1408F49EC0111118C020E04D2D4F
:10B5B0006E2D80E00E94E7104881429546954695A1
:10B5C00043702A2D60E178E08E2D0E940B25829534
:10B5D000880F880F807C98819F7331C088811130DB
:10B5E00089F580905701982F907C903811F4A9E14B
:10B5F0008A2E482F440F440F4595459547314CF00E
:10B6000029EE240F49EF57E06E2D85E40E94DA639E
:10B6100005C0202F6E2D85E40E949D11AA2009F4FB
:10B62000C2C06091570161958881880F880F482DAD
:10B63000859585950E9437148F739881907C982BFF
:10B640009883B1C0982F907C4981903491F447FD44
:10B6500003C04F3024F401C040E0242F01C02FE08C
:10B6600029834EE556E16E2D88E70E94DA634FE0AC
:10B6700015C0903831F5880F880F89358CF047FD5B
:10B6800004C049301CF049E001C040E049834F5FED
:10B69000202F6E2D80E60E94472249E060E01BC00B
:10B6A0004F360CF04FE64983552747FD50954058DB
:10B6B0005F4F202F6E2D88E70E9414664FE660E8EA
:10B6C0000AC0552747FD5095202F6E2D88E70E9410
:10B6D00014664DE763E8AA2009F465C089810E94D9
:10B6E000371460C0111122C066EF77E08E2D0E94E2
:10B6F000116420E04D2D6E2D86E10E944466AA2043
:10B7000069F0409157014150888160E08F710E943B
:10B7100037148F719881907E982B988348814F7150
:10B72000202F6E2D8EE10E949D113DC08881113029
:10B7300081F4482F4295469547702A2D68EC77E0B2
:10B740008E2D0E940B258295880F807E98819F7197
:10B7500076CF82958695877090E04981069764F050
:10B76000493008F049E049834F5F202F6E2D80E675
:10B770000E94472269E010C04B3F38F450E0202F70
:10B780006E2D86E60E94146606C0485F202F6E2D3F
:10B7900084E50E9464246FEFAA2029F0898190E05B
:10B7A0000E943F1489831F5F133009F0EDCED394BC
:10B7B00088E0E80E90E4E912ABCEDF91CF911F91C3
:10B7C0000F91FF90EF90DF90CF90BF90AF909F9040
:10B7D0008F907F906F905F904F903F9008951EE7FD
:10B7E000A4CD20E07DCE1F93CF93DF93EC011AE030
:10B7F00088810E94702C0E94802C89931150C1F77F
:10B80000DF91CF911F9108959C01265F3F4FFB016F
:10B810004491DC014D93CD013196A217B307C1F7D6
:10B820000895EEE0F6E080E090E021913191820F02
:10B83000931F26E0E632F207C1F7089587E7EDE0AF
:10B84000F6E0DF011D928A95E9F78BE080930D0603
:10B8500089E180933B068AE580933C0681E08093F2
:10B86000510686E180933E06EEE0F6E020E032E00D
:10B8700080E093E02193319395878487938F828F23
:10B88000B6E0EC31FB07B1F763EB78E18EE596E0CB
:10B89000BBDFC7DF90933906809338060895EF9297
:10B8A0000F931F9361E0680F88ECE82E02EC13E021
:10B8B0002BE432E042E085EF98E0FCD521E0823CC9
:10B8C000934009F020E0822F1F910F91EF9008958F
:10B8D000CF93C82F22EC33E0EBE4F2E0DF01C901A3
:10B8E0001D920197E9F768EA78E1CF018DDF8C2F8F
:10B8F00090E06AE070E001960E94077A605D6093D4
:10B900005002805D8093510284E080933B0582E089
:10B9100080935D020E94446A8C2FCF91C0CF0F9319
:10B920001F93CF93DF93EB01042F803120F561E06B
:10B93000680F85EF98E00FD410E0A80160E270E096
:10B94000CE010E94787A4AE050E0BE0185EF98E08F
:10B9500085D40A9781F485EF98E0EFD3C00FD11F0B
:10B96000009749F06AE070E00E94077A805D8A9350
:10B97000862F972FF5CFDF91CF911F910F910895CB
:10B980008F5F93C361E0680F85EF98E0E4D382ECAA
:10B9900093E0EBE4F2E0DF019C011D922150304086
:10B9A000E1F742EC53E0BF0185EF98E057C4FF9206
:10B9B0000F931F93CF93DF93CDB7DEB768970FB682
:10B9C000F894DEBF0FBECDBF01E0080F102F10317D
:10B9D000B0F4FF24F394F10E8F2D67D381110DC0C5
:10B9E000602F85EF98E0B7D361E0610F28E532E082
:10B9F00042E0CE0140960ED506C01F2DE8CF103193
:10BA000079F780E017C04FE050E0BE016F5F7F4FD5
:10BA100085EF98E0BDD3882349F0482FBE016F5FC2
:10BA20007F4FCE0140967DD4A895EDCFCE014096B4
:10BA300017D581E068960FB6F894DEBF0FBECDBF74
:10BA4000DF91CF911F910F91FF900895EF920F9387
:10BA50001F9361E080E798E10E945E198EE598E10E
:10BA60000E94AC12E6D298ECE92E07E710E02DE038
:10BA700036E041E060E085EF98E01CD5873791051E
:10BA800021F08FE498E10E94911980E01F910F91BD
:10BA9000EF901ECFCF93C82F8770A1F0909100092F
:10BAA000982B909300090E949B109093FF0880931D
:10BAB000FE088C2F90E024E0959587952A95E1F774
:10BAC00080930109CF910895CF93DF93D4D2811150
:10BAD00002C080E02EC04DD287FDFBCF60E085EF35
:10BAE00098E039D387E7EDE0F6E0DF011D928A9513
:10BAF000E9F747E750E0BF0185EF98E0AFD38EE567
:10BB000096E071DE80910D068B3040F481E08093E9
:10BB1000C7018BE080930D0681E0BCDFC091380641
:10BB2000D09139067EDE21E0C817D90709F020E060
:10BB3000822FDF91CF910895EF920F931F93CF93B0
:10BB4000DF9310924309C0910009CC2309F498C0F7
:10BB5000909101099F5C9093430981111CC00E9440
:10BB60009B102091FE083091FF08821B930B883CAC
:10BB7000910508F485C080910109882361F0815006
:10BB800080930109882339F00E949B109093FF084D
:10BB90008093FE0875C0109201098091EB08811115
:10BBA0006FC0DC2FD470C2FD02C081E001C083E011
:10BBB0008093EB08C0FF2CC082E3809343098091FF
:10BBC00000098E7F8093000944E1E42E07E710E02E
:10BBD0002DE036E041E061E18CEE98E06BD48737F0
:10BBE000910519F461E180E02FC08091F208823064
:10BBF00051F480910009816030C08091F208823058
:10BC000029F1D1113BC08EEB98E10E94911936C009
:10BC1000C1FF34C083E38093430980910009897F89
:10BC20008093000934E1E32E02EC13E02BE432E0D0
:10BC300042E061E18CEE98E03DD4823C9340E9F62D
:10BC400080913A0661E18F5F3ED218C08091000971
:10BC5000D11102C0826001C08660809300090E94F9
:10BC60009B10885C91099093FF088093FE08809157
:10BC7000910D833019F4A8951092910D1092EB0854
:10BC8000DF91CF911F910F91EF900895809100095E
:10BC9000882351F081E050DF8091910D8330B1F71E
:10BCA000A8951092910DF2CF0895EF92FF920F9305
:10BCB0001F93CF93DF93C82F803108F0BFC062DE9F
:10BCC0008F3F910509F010F48C2F02DE8BE492E097
:10BCD0008ADD8091F304811107C080915C02869512
:10BCE00083708E5F8093F30480915A02982F92950F
:10BCF000969596959370933029F090933C05806CBF
:10BD000080935A0280913B05823008F062C010E0B7
:10BD1000812F0E94A810EC0189818150843018F491
:10BD20000E948E1089831F5F103291F7C1EAD4E020
:10BD300000E010E08A818F700E94A210882389F0B1
:10BD40008230C1F4C8018E559B4F7C01FC0180817B
:10BD5000882339F085302CF481500E948E10F70131
:10BD600080838881882331F0853024F481500E94BB
:10BD70008E10888323960D5F1F4F04321105D1F674
:10BD800088E3E5EFF3E0AEE5B8E001900D928A9527
:10BD9000E1F7CEE5D8E010E00EE0812F0E948E1092
:10BDA0008150089FD0011124AB50BC4FFE01802F61
:10BDB00001900D928A95E1F71F5F2E96143069F776
:10BDC00083E998E10E94911982E080933B0562DE4D
:10BDD0005DDF80913B058330F8F480E090E0FC016A
:10BDE000EF55FB4F2281322F3F703C3019F4207FFA
:10BDF0002A6022832281322F3F703D3019F4207F48
:10BE00002B60228303968432910549F783E0809367
:10BE10003B0582E03FDE3ADF80913B05843070F4E1
:10BE2000809168068093FA0480E898E10E94911955
:10BE300084E080933B0582E02DDE28DFE0E0F2E045
:10BE40008091560282838091C60483838091580238
:10BE500090915902918380838091570281708483ED
:10BE60008091F80487838091F90480878091F6049B
:10BE70009091F704968385838091BC0587FB882782
:10BE800080F981870E9477310E947D31DF91CF91C7
:10BE90001F910F91FF90EF90089540E450E060E013
:10BEA00070E082E099E00C946D6741E050E062E060
:10BEB00070E084E099E00C946D67CF93DF931F925C
:10BEC000CDB7DEB7698390E1899FB001112441E0CD
:10BED00050E0CE0101960E946D670F90DF91CF91E7
:10BEE0000895CF93DF931F92CDB7DEB790E1899F7E
:10BEF000B001112441E050E0CE0101960E947F7A0A
:10BF000089810F90DF91CF910895CF93DF93D82F40
:10BF1000C82F8C2FE6DF882321F08C2FE2DFC82F7B
:10BF2000F8CF609104098C2FC8DFD0930409DF910A
:10BF3000CF91BBCFCF93C0910409CC2341F08C2F7C
:10BF4000D0DF80930409B1DF60E08C2FB6DF8C2F47
:10BF5000CF910895CF93DF9380910409C0E0D0E0A2
:10BF6000882319F02F96BDDFFBCFCE01DF91CF9153
:10BF70000895DF92EF92FF920F931F93CF93DF9379
:10BF800080E8EBE4F2E0DF011D928A95E9F7C6E074
:10BF9000D9E0F12CB4E1FB1205C08091040904E062
:10BFA00019E002C08E01888190E0E12CDD24D39459
:10BFB000DF0C0097E9F09C01245031092C37310542
:10BFC00030F4FC01E55BFD4F2081222361F0EE207F
:10BFD00021F060E08E2D71DF03C0F80110825DDF7B
:10BFE00080E090E0E6CFD082E82E7BDF90E0E1CFEA
:10BFF000F3942396F5E1FF12CDCFC4E0D0E0FE012B
:10C00000E55BFD4F8081811107C0609104098C2F91
:10C0100054DFC093040949DF2196C038D10579F770
:10C0200080E0DF91CF911F910F91FF90EF90DF9013
:10C030000895CF9380E4E2E0F9E0DF01982F1D92AC
:10C040009A95E9F794E0909302098093030980E1BF
:10C050008093050984E0C1E0C80F6C2F2EDFCF3735
:10C0600011F08C2FF8CF60E08FE727DF84E080931A
:10C070000409CF9112CF40E450E060E070E082E02C
:10C0800099E00E947F7A80910309811103C080E4C6
:10C090008093030980910209843029F481E0909112
:10C0A0000309903409F080E0089590E0FC01EE0F60
:10C0B000FF1FE80FF91FEE5FF64F81E094819111A9
:10C0C00001C080E00895CF93DF9390E0EC01CC0FA6
:10C0D000DD1FC80FD91FCE5FD64F8C819D81AE81E9
:10C0E00070E0FB01EE0FFF1FE60FF71FEE5FF64F4C
:10C0F0002481358146812C833D834E8384839583BF
:10C10000A683DF91CF91C9CECF9390E09C01220FFF
:10C11000331F280F391FF901EE5FF64FC481F90173
:10C12000EA5FF64F108211821282B7DECC2319F03B
:10C130008C2FCF91EACECF910895FC01808190E0C1
:10C14000FC01EE0FFF1FE80FF91FE95FF64F918129
:10C1500080819F700895CF93DF93FC0160831282EA
:10C16000118270E0CB01880F991F860F971FEC0199
:10C17000CE5FD64F2C812383148215821682FC0158
:10C18000E85FF64F808182958F70DF91CF9108959F
:10C19000AF92BF92CF92DF92EF92FF920F931F93D5
:10C1A000CF93DF931F92CDB7DEB78C01FC01808166
:10C1B00090E0FC01EE0FFF1FE80FF91FE95FF64F5B
:10C1C00080812181922F9F70F80121813281821B11
:10C1D000930B7A018417950708F47C015B016701D2
:10C1E000C114D10421F1F8018381882301F1648114
:10C1F0006F5F648370E0F0E18F9F600D711D11240B
:10C2000041E050E0CE0101960E947F7A8981F501DC
:10C2100081935F01F80184818F3028F0148283813B
:10C2200060DEF8018383F1E0CF1AD108D9CFF8019D
:10C23000818192818E0D9F1D8C199D09928381832E
:10C240008E2D8C190F90DF91CF911F910F91FF9040
:10C25000EF90DF90CF90BF90AF9008957F928F9234
:10C260009F92AF92BF92CF92DF92EF92FF920F9385
:10C270001F93CF93DF934C016B018A01C0E0D0E0A4
:10C280005C0125E0A20EB11CC017D107D8F5F4015E
:10C2900085818F7781F0F4014581F42FFF777F2E20
:10C2A0002F2F30E0C8018C1B9D0B8217930758F489
:10C2B000702E7C1A08C041E050E0B501C40168DF6F
:10C2C000813049F31FC0E72CF12CC6018C0F9D1F54
:10C2D00047FF06C0A70160E070E00E94787A0BC0BB
:10C2E000A701BC01C40154DF871529F0FE01E80F46
:10C2F000F11DCF0108C0CE0DDF1DF4018581871926
:10C300008583C2CFCE01DF91CF911F910F91FF9016
:10C31000EF90DF90CF90BF90AF909F908F907F90E5
:10C320000895AF92BF92CF92DF92EF92FF920F9358
:10C330001F93CF93DF93EC018B01D42E8B8181115E
:10C3400010C089819A81892B61F4E880F12CF2DD9B
:10C350008B83F701EE0FFF1FEE0DFF1DEE5FF64F13
:10C360008483CD2C8FE0A82ECC2009F43CC0EF8034
:10C37000F8840E949B10E81AF90AF7FE02C082E0D6
:10C3800004C08B81811103C081E08E832CC09C810D
:10C390009F3058F01C82A5DD811104C0CBDD682FD1
:10C3A0008B818BDD8B819DDD8B838B81882361F37A
:10C3B0006C819A2D961BBC2C9C1508F4B92EEB2C85
:10C3C000F12C70E090E1899F600D711D11246F5F69
:10C3D0007F4FA701C80181D50E0D1F1D8C818B0DCC
:10C3E0008C83CB18C1CF6D2D70E06C197109298138
:10C3F0003A81260F371F3A8329838D2D8C19DF91BF
:10C40000CF911F910F91FF90EF90DF90CF90BF9051
:10C41000AF900895EF92FF920F931F93CF93DF9306
:10C42000EC01F62EE42E890196DE6F2D70E0FB0103
:10C43000EE0FFF1FE60FF71FE95FF64F1082E29441
:10C4400030EFE322E1820E949B10800F911F9887BA
:10C450008F83DF91CF911F910F91FF90EF900895FF
:10C460001F93CF93DF93EC01888190E0FC01EE0FE6
:10C47000FF1FE80FF91FE95FF64F898180839A81DA
:10C480009F708181807F892B81838B81882321F01C
:10C4900028DD182F81110AC010E0FFDC112311F0F4
:10C4A000812F33DDDF91CF911F91089560E08B8163
:10C4B00004DDF3CF7F928F929F92AF92BF92CF9283
:10C4C000DF92EF92FF920F931F93CF93DF931F9210
:10C4D000CDB7DEB76C0159012E2D30E09BDF1982FC
:10C4E0004501E12CF12C77247394F40181914F01E3
:10C4F0009981811108C071104CC08081811105C0E3
:10C50000772473941BC071100AC080E09F3718F421
:10C51000E016F10661F5772081F0782E01C0712CCC
:10C52000992329F19068998341E0BE016F5F7F4FA5
:10C53000C601F7DE8130D1F026C0782E9923B9F0FC
:10C5400041E0BE016F5F7F4FC601EBDE8130D9F461
:10C550004981B701641B71096A0D7B1DC601E1DECB
:10C560009981891719F0981B99830DC019828981C7
:10C570008F5F8983A895FFEFEF1AFF0A0E151F053D
:10C5800008F0B3CF08C089818F778701081B110994
:10C5900002C0872DBBCFC60163DFC8010F90DF91BA
:10C5A000CF911F910F91FF90EF90DF90CF90BF90B0
:10C5B000AF909F908F907F90089580E094E0E5E4A5
:10C5C000F9E0DF019C011D9221503040E1F7089510
:10C5D000FF920F931F93CF93DF93FA01149131963B
:10C5E0007491795F769576957695DA011396FA01CE
:10C5F00032964491249FA00DB11D11246695669535
:10C60000669590E0F0E86F9F800D911D112420E069
:10C6100030E060E08B5B964F412F50E0671799F058
:10C620000A2FEC01C20FD31FFD01FE2EF01AF116E6
:10C6300020F4F490F9923196F8CFA40FB51F6F5FF4
:10C6400020583F4FEBCFDF91CF911F910F91FF907B
:10C650000895CF93DF93382F463128F4842F880F25
:10C66000840F880F7EC086E0830F20FD08C021FD67
:10C6700002C090E005C09091580D96FFFACF91E06E
:10C68000687FA32FB0E050E1659FA00DB11D11247C
:10C69000AB5BB64F22FF3DC04E3211F088E0830FF6
:10C6A00024ED240F2F3010F44B5211C02FEB240F28
:10C6B0002A3110F441530BC02FE9240F2A3110F412
:10C6C000465305C04F3511F44AE201C040E06EE028
:10C6D000469FA00111244852574E27E0FA01349199
:10C6E0003796E491211102C0E0E030E04F5F5F4FE8
:10C6F000992311F03095E095FCE0A43CBF0730F49D
:10C700003C93ED01C058DF4FE8831196215030F77C
:10C7100028C023FF07C0892F81958D9385E0830F63
:10C7200031E001C030E025E0429FF0011124E250E9
:10C73000F44E25E04491332311F0243041F05DE0C4
:10C74000A534B50718F4911140954C9311962150DA
:10C7500031962111EFCF6DE0A534B60710F4919515
:10C760009C93DF91CF91089520E073CFEF92FF92D9
:10C770000F931F93CF93DF93F62E122F902F90716C
:10C78000E92EFA01112379F0EE2011F0408101C069
:10C790004491EF012196442331F0202F6F2D59DF72
:10C7A0001150FE01EFCFDF91CF911F910F91FF90BC
:10C7B000EF9008950F93FA0194914F5F5F4F929F0E
:10C7C000400D511D1124292FD1DF0F9108950F9392
:10C7D00000E0CCDF0F910895FF920F931F93CF934A
:10C7E000DF93162F022F922F9071F92EEA01FF206E
:10C7F00011F0488102C0FE014491442361F04F31A1
:10C8000031F4185F103438F480E02196F0CF202FF7
:10C81000612F1FDFFACFDF91CF911F910F91FF9012
:10C820000895AB0120E0682F80E0D6CFFB014423C0
:10C8300041F09491992351F09F3109F44150319680
:10C84000F6CF20E0AF01682F80E0C6CF089520E04A
:10C85000C3CFFF920F931F93CF93DF93082FF62E32
:10C86000EA0114E1180F15504C2F4F704A301CF09C
:10C87000495C28E002C0405D20E06F2D812FE9DE99
:10C8800084E0D695C7958A95E1F71013ECCFDF9138
:10C89000CF911F910F91FF900895222321F0909145
:10C8A000580D96FD0895480F687FE82FF0E090E15D
:10C8B000699FE00DF11D1124EB5BF64F8E1B982F45
:10C8C0009E0F941720F4908190959193F8CF08953E
:10C8D0002DE08534920760F4FC01208130914409F9
:10C8E000332319F0262B313009F02627FC01208351
:10C8F0000895262F287F6770E62FF0E0E857F14E65
:10C90000649190E030E1239F800D911D11248B5B99
:10C91000964FDECFEF92FF920F931F93CF93DF934B
:10C92000F42E47FF02C0840FF194962F987FC82FF2
:10C93000D0E080E1989FC00DD11D1124CB5BD64F74
:10C940006770E62FF0E0E857F14EE490FF20B1F079
:10C950008DE0C534D80790F4022F10E020FF08C006
:10C960006E2DCE01B5DF15950795202F206803C0E9
:10C9700015950795202FFA942196E8CFDF91CF9156
:10C980001F910F91FF90EF9008952FEFC3CF1F934A
:10C99000CF93DF93142F47FF02C0640F1195962F9A
:10C9A000987FC82FD0E080E1989FC00DD11D112441
:10C9B000CB5BD64F862F877099F0E82FF0E0E857D1
:10C9C000F14E64916195180F185017FF0DC0E12FBB
:10C9D000FF27E7FDF095E057F14EE4916E0F04C09C
:10C9E00018303CF018506FEFCE0172DFC058DF4FA7
:10C9F000F7CF111654F4E12FFF27E7FDF095E85724
:10CA0000F14E64916150CE0163DFDF91CF911F91B0
:10CA100008953F924F925F926F927F928F929F9272
:10CA2000AF92BF92CF92DF92EF92FF920F931F933C
:10CA3000CF93DF93182FB62E802F05FF04C004FF7D
:10CA400004C002E003C000E001C001E0982F9F771E
:10CA5000C92EE7FE04C0E1946624639401C0612CF2
:10CA600057FF0AC050954095309521953F4F4F4F45
:10CA70005F4F7724739401C0712C82FF06C098E049
:10CA80009093450DE8E0DE2E05C096E09093450DAD
:10CA900075E0D72E86FF28C071101D0D283E83E05B
:10CAA00038074105510514F01D0D05C02436310528
:10CAB0004105510514F01D0D05C02A303105410511
:10CAC00051050CF01D0D002381F0023031F42436A5
:10CAD0003105410551054CF41D0D2A303105410544
:10CAE00051051CF41D0D01C01D198091450D810FCC
:10CAF0008093450D023011F490EFC90E8824839481
:10CB000052E0A52E912CFF24E7FCF09466E0562E0F
:10CB10005B0CE82DF0E0EE16FF060CF45DC06AE059
:10CB200070E0C9010E94077A382EEB0140E3442EE1
:10CB3000480E2C2D442D6B2D812F8BDD08112FC01D
:10CB4000C2FE1AC08FEF830D833008F4A394CE0188
:10CB50006AE070E00E94077A823011F08430D9F4E4
:10CB600084E3481204C099249394910E15C099242B
:10CB70009A94910EA39410C03EEF432E410E8FEF76
:10CB8000810FC0FE04C047E06B2D01DF02C0652DA0
:10CB9000B0DE142D01C0912E209709F000E09E0117
:10CBA000442737FD4095542F211531054105510586
:10CBB00081F4002331F0023059F491E0981540F0EF
:10CBC00008C0C4FE09C0611004C080EFC80E01C0D7
:10CBD00000E01D1983949DCF992059F09A944A2D15
:10CBE0006CE06B0D892DD1DE4A2D6DE06B0D892D2A
:10CBF000CCDE772031F02C2D4DE26B2D812F8D195D
:10CC000028DD80E0DF91CF911F910F91FF90EF9091
:10CC1000DF90CF90BF90AF909F908F907F906F905C
:10CC20005F904F903F900895EF920F93022F9A01DB
:10CC3000442737FD4095542FF5E0EF2EEADE0F91A3
:10CC4000EF900895CF93DF93D62FC22F206250E04C
:10CC5000EBDFC7FD08C02C2F46E76D2F8091450DF7
:10CC6000DF91CF91F6CCDF91CF91089590913D0166
:10CC700020913C06921710F422E001C020E0242B02
:10CC8000492FE0CF20E0D0CFEF920F93022F005F2B
:10CC9000242F30E040E050E0A2E0EA2EBADE0F910F
:10CCA000EF900895DF92EF92FF920F931F93CF932F
:10CCB000DF93182FE62EEA01F22E822F8470D82EF1
:10CCC00022FF05C01D5F57FF0FC087E103C057FF5C
:10CCD0000BC08FE02F2D4DE26E2D912F981B892FC9
:10CCE000B8DCD195C195D1092F2D20234AE36E2DB3
:10CCF000812FAFDC6CE370E0CE010E94077A462FF3
:10CD0000C82FD1101E5F2F2D6E2D812FBDDFDD208E
:10CD100011F085E101C08FE0810F202F4C2F6E2D87
:10CD2000DF91CF911F910F91FF90EF90DF90ACCFEB
:10CD30000F931F93CF93DF93C82FD62F142F022F5B
:10CD4000422F25DE123030F0402F6D2F8FEF810FF4
:10CD50008C0F1DDE6FEF6D0F600F412F8C2F15DED6
:10CD6000412F6D2F8C2FDF91CF911F910F910DCE01
:10CD7000CF93C091440991E090934409D9DFC093C7
:10CD80004409CF9108950F931F93CF93DF93182FEA
:10CD9000C62FD22FE42FF0E03297053608F004E6D4
:10CDA0000E9FC0010F9F900D112464E670E00E9459
:10CDB000077A062F2D2F6C2F812FDADF002361F0E9
:10CDC000D150DC0FCF5F1F5FCD1730F4402F6C2F99
:10CDD000812FDBDDCF5FF8CFDF91CF911F910F91D6
:10CDE0000895A998AB988BBBAD9AAD98AB9AA99AC8
:10CDF0000895CF93C82F81E08093420981E8F1DF45
:10CE00008C2FEFDF10924209CF91089580913B065D
:10CE1000F0CFCF93DF9381E080934209AA982AE074
:10CE20002A95F1F700C0AA9A8CED95E0E5E0EA9525
:10CE3000F1F7000001970097C9F7AC98CEECD8E164
:10CE4000FE018491CEDF2196F8E1C83DDF07C1F7EE
:10CE5000DF91CF91DBCF1F93CF93DF9340914309B5
:10CE6000442321F08091580D86FD32C081E08093EB
:10CE7000420910EBC5E4D9E084E0B3DF80E1B1DF23
:10CE8000812FAFDFA998AB9AFE019E0120583F4F3A
:10CE900080818BBBAD9AAD9881818BBBAD9AAD98EB
:10CEA00082818BBBAD9AAD9883818BBBAD9AAD98D7
:10CEB0003496E217F30761F7EF01AB9AA99A1F5F67
:10CEC000183BD1F610924209DF91CF911F9108953E
:10CED0004A5260E080E059DDC9CFBF92CF92DF9225
:10CEE000EF92FF920F931F93CF93DF937B018A0101
:10CEF000080F191FEC01E81AF90A6701CC0EDD1EB4
:10CF0000C017D107C1F0B9908091EB088270E19B06
:10CF100005C08823E1F30E940E1CF6CFDFBACEBA1B
:10CF2000E09A8DB3B81649F3BDBA8FB7F894E29A78
:10CF3000E19A8FBFE2CFDF91CF911F910F91FF90C8
:10CF4000EF90DF90CF90BF9008958091890D10925F
:10CF5000890D0895FC0180818F70880F61118160B7
:10CF60008F709081907F982B908381818F5F8183D8
:10CF70008281882351F09F7041F4833621F0842F01
:10CF800080628093890D118212828281883069F1DA
:10CF900048F4813091F188F0823039F1843009F021
:10CFA0003FC023C08F35C1F018F48031F1F00895EF
:10CFB000813649F0823671F1089580818F708F300B
:10CFC00079F581E62BC040664093890D10923601B9
:10CFD000109235018FE522C08181803211F44068C2
:10CFE00016C08832E9F480E119C09181903328F0AD
:10CFF00090E09595879582831182828190E00197D8
:10D00000218130E082239323892B51F440644093A3
:10D01000890D08958181803418F088E0828311821F
:10D0200008955091630041B1282F30E02F30310531
:10D030006CF4F901EE0FFF1FE20FF31FE45AF24FF9
:10D0400090819F7081E09F3051F52AC090E0FC01F3
:10D050003F97E930F10518F5E955FF4F0C94587AE0
:10D06000942F947019C091B1927016C0952F10C072
:10D07000952F9095987010C053FF11C091B102C0C8
:10D08000942F9095907408C0942F907105C0942FA0
:10D09000917002C0942F907281E0911101C080E0E4
:10D0A00008958D3208F062C09FEF980F993010F408
:10D0B000825FB7CF51EE580F5330D8F491B19095AD
:10D0C00094705523C9F0409180064F70415021E083
:10D0D00030E0042E01C0220F0A94EAF730915B0D74
:10D0E0003223523041F0932B21E009F020E0922FBF
:10D0F00003C090E001C0932F85528330F0F491B1CA
:10D100009695917021E09227882369F140918006DD
:10D1100042954F70415021E030E0042E01C0220FB3
:10D120000A94EAF730915B0D3223823009F1932B98
:10D1300081E009F080E0982F16C0863019F4209124
:10D14000820605C0873079F42091820622952F70DF
:10D15000215081E090E0022E01C0880F0A94EAF786
:10D1600090915B0D982381E0911104C080E00895B7
:10D17000932FF9CF0895CF93C82F93DF811107C064
:10D1800081E08C0F8EDF882321F081E003C080E0F6
:10D1900001C082E0CF9108958F7090E08F309105AB
:10D1A00051F0FC01EE0FFF1FE80FF91FE45AF24F98
:10D1B00082E68283118208958F7090E08F3091050E
:10D1C00049F0FC01EE0FFF1FE80FF91FE45AF24F80
:10D1D00083E682830895EF92FF920F931F93CF937C
:10D1E000DF938091590D90915A0D019690935A0DAD
:10D1F0008093590D8093580D96B3909580918A0D28
:10D20000882321F0282F2877292349F4892F807635
:10D2100009F07DC093FD77C094FF77C080E1182F9F
:10D220001660192380938A0DCCE5DDE000E011FB48
:10D23000662760F9402FCE018DDE0F5F169523968D
:10D240000630A9F780910A0281110EC0F0B2F09465
:10D2500080916D0686FF09C08F2D837FF82E809107
:10D26000600E8C70F82A01C0F12CC0E9DEE100E00C
:10D2700010E076E0E72EEC1AFE0184914C2F4E0D63
:10D280008F2161E009F460E0C8018259924F62DEAB
:10D2900021960D5F1F4F0831110571F79091100213
:10D2A00061E0C92FC07295FF60E04EE086E89DE026
:10D2B00051DE86B390E0809590958E7799278C2BE0
:10D2C00019F089E0809355018091600E86FD02C0BF
:10D2D000817402C0817082609091630092FF8860C7
:10D2E0009091630095FF8062989B84609C9B806412
:10D2F000B79B806180935B0DDF91CF911F910F9160
:10D30000FF90EF90089588E08ACF80E088CF80E694
:10D3100086CF929A1092980089E18093990080912B
:10D320009B008D7F80939B0086E080939D00809181
:10D330009B0087FF03C080919C00F9CF88E9809310
:10D340009A00089581E080938E0D80930A02809167
:10D350006D0686FFDECF089580916D0686FF1092E0
:10D360009A0010920A02F3C590919B0095FFFCCFA2
:10D3700080939C000895E6E4FDE0918980898917F7
:10D3800049F0DF01A90FB11D8C919F5F9F70918BB8
:10D3900090E008958FEF9FEF08951F920F920FB6C0
:10D3A0000F9211242F938F939F93EF93FF9380916C
:10D3B0009A008F7780939A007894E091560D81E0DF
:10D3C0008E0F8F7090919C002091570D821731F035
:10D3D000F0E0EA5BF24F90838093560DF8948091D1
:10D3E0009A00806880939A00FF91EF919F918F91AE
:10D3F0002F910F900FBE0F901F90189580E491E031
:10D40000E5E6F2E0DF019C011D9221503040E1F79A
:10D410000895FF920F931F93CF93DF93182FF62E4B
:10D42000C5E6D2E090E08881181738F0882329F00B
:10D43000903201F19F5F2A96F6CF9032D9F02FE11A
:10D4400030E0291B31090AE0029FA001039F500D23
:10D450001124BE01CE010A960E94677AFE01119244
:10D460000A95E9F7188384E68A838F8188608F8321
:10D47000CE0102C085E692E0FC01F182DF91CF91FE
:10D480001F910F91FF900895CF93DF9300D000D0AC
:10D49000CDB7DEB7E0915606F0E0E95AFC4FE491D3
:10D4A00084E09E2F9370A1E0B0E0AC0FBD1FA90FE8
:10D4B000B11D8C93E695E695815099F79FDF61E069
:10D4C0008981A7DF62E08A81A4DF63E08B81A1DF2D
:10D4D00064E08C810F900F900F900F90DF91CF91AF
:10D4E00098CF80E49CE99BBD8ABD87B7806187BFE8
:10D4F0001FBC8AE08EBD08950F931F93CF93DF93D7
:10D5000010915C02129516951770882331F0A3EEE6
:10D51000BDE0833021F420E103C0ABE9BDE028E0A9
:10D5200090915B02990F910F920F60915E0224E639
:10D530006202B0011124685A7D4F0091640248EEE6
:10D5400053E004039001059F300D1124285330450A
:10D55000261B370BFD0132966D937C93409161023F
:10D5600041FF03C040E055E002C040E054E083309A
:10D5700011F418EF190FCC27DD27C41BD50B191791
:10D58000F0F4A12FB0E0AA0FBB1FA652B84F0D9028
:10D59000BC91A02D4A175B070CF4DA01AC17BD074C
:10D5A0000CF4DE01A854B44F2A1B3B0BA61BB70B8F
:10D5B000B183A083738362831F5F3496E0CF2832E8
:10D5C00093E2390710F428E233E231832083882381
:10D5D00031F0285E334030938C0D20938B0D1382F5
:10D5E0001282DF91CF911F910F9108951F920F9298
:10D5F0000FB60F9211242F933F934F938F939F93C6
:10D60000EF93FF9388B391E0892788BBE0910E01E7
:10D61000F0910F018081982F9F709F3039F04091D9
:10D620002D0E949F402D1124415001C04FEF242F07
:10D6300030E037BD26BD90E024E0959587952A958A
:10D64000E1F7009731F43196F0930F01E0930E016A
:10D6500001C08083493C40F080915A028F7086302F
:10D6600011F4C09801C0C09A8091910D816080939F
:10D67000910DFF91EF919F918F914F913F912F913C
:10D680000F900FBE0F901F9018951F920F920FB61C
:10D690000F9211242F933F938F939F93EF93FF93B8
:10D6A00088B391E0892788BBE0911001F0911101C6
:10D6B000808128B539B580FD03C0205E3F4F02C090
:10D6C000205F3F4F39BD28BD90E095958795009725
:10D6D00069F4CF010196909311018093100181812B
:10D6E000811105C087B7877F87BF01C08083809184
:10D6F000910D81608093910DFF91EF919F918F919A
:10D700003F912F910F900FBE0F901F901895EDE74E
:10D71000F0E08081857E808317981F9AAAE8B0E0A8
:10D720001C9210928B0082E88C93808180628083AF
:10D730000895EDE7F0E080818F7D8083179AAAE855
:10D74000B0E01C9210928B008AE08C9380818861FB
:10D75000808308951F920F920FB60F9211248F931A
:10D760009F93EF93FF9380912B0E882321F01F9AB4
:10D7700010922B0E04C01F9881E080932B0EE09135
:10D780000A01F0910B018081918190938700809331
:10D79000860080918B0D90918C0D909385008093E5
:10D7A000840082819381892B11F0329608C0809188
:10D7B00061028095817080932B0EE3EEFDE0F09383
:10D7C0000B01E0930A018091910D81608093910D8E
:10D7D000FF91EF919F918F910F900FBE0F901F902F
:10D7E0001895E2E9FDE09081969596952781222390
:10D7F00011F096959695982B908321812F5F218328
:10D800008085281750F0A281B3819D012F5F3F4F83
:10D81000338322839C93108211820895FF920F9389
:10D820001F93CF93DF93C82F80915A028F7082305D
:10D8300069F09C2F88E0D0E0292F2078D20F990F33
:10D840008150D1F7D07859E0F52E03C048E0F42E8E
:10D85000D0E810E080E190E00C2F0170901302C03E
:10D86000805F02C0BEDF80E1C695CD2B1F5FF11641
:10D8700018F0D0E8902FF0CF805FDF91CF911F910B
:10D880000F91FF90AECF882339F08091980D8F5F74
:10D890008093980D80E803C01092980D80ECA1DF72
:10D8A0008091980D8530C0F70895CF93DF93C82FEE
:10D8B000E091970DE827F0E0EE0FFF1FE856F14EDC
:10D8C000259134915091960D40E0242735273093CF
:10D8D000970D2093960DD8E08C2F8078D4DFCC0F55
:10D8E000D150D1F7DF91CF910895CF9380EC79DFBC
:10D8F000C6E080E876DFC150E1F780ECCF9171CFD0
:10D900008031E0F4E82FF0E0EE0FFF1FE652F84F11
:10D9100020813181C901880F991F820F931F97FDC4
:10D92000039695958795959587959C5F181619068A
:10D9300044F48E3F27E092073CF4089580E094E0A1
:10D94000089581E090E008958EEF97E008956F923A
:10D950007F928F929F92AF92BF92CF92DF92EF927F
:10D96000FF920F931F93CF93DF931F92CDB7DEB734
:10D9700072E9672E7DE0772EF3013F018BE99DE090
:10D9800093838283108211821582148281E08783BF
:10D9900082E08087F0905A02FF2DFF70FF2EF8136F
:10D9A0002BC080E180932D0E80918D0D86FF0DC0E0
:10D9B00080913C05811102C080E805C0813011F4DE
:10D9C00080E901C088E980938D0D80918D0D87FFDE
:10D9D00005C087E126DB882309F4BBC080918D0D4B
:10D9E00087FDBDC085E10E943E19882309F4B7C0B8
:10D9F00080918D0D8062B6C084E180932D0E86E00B
:10DA0000F81302C08FE01EC085E508DF80913C0559
:10DA10008F5F8F7580938D0D90918F0D90FF03C058
:10DA2000806880938D0D95FF05C080918D0D80627B
:10DA300080938D0D80918D0DF1DE80915B02EEDE85
:10DA400080913D05EBDE0AED17E0C12CD12CE12CD5
:10DA5000912C35E0A32EB12C48EF842EF801819152
:10DA600091918F01880F991F880F991F1816190619
:10DA70001CF424E030E002C02CEF3FEF820F931F34
:10DA8000B5010E94077AF5E0CB01FF1202C09C5F4E
:10DA900002C080529C4F97FD07C0811528E0920775
:10DAA0002CF08FEF97E002C080E090E0AA2797FD6E
:10DAB000A095092C03C0880F991FAA1F0A94DAF7B2
:10DAC000C82AD92AEA2A8BE0890D89838C2DA6DE03
:10DAD000CD2CDE2CEE24E981E850E983E830B0F764
:10DAE00093E0990D892F869586958695992E889D28
:10DAF000900C1124F7E00A3F1F0709F0AFCF26E092
:10DB0000F21204C080E08ADE80E088DEF3018181C9
:10DB1000A281B381882319F08FE08C9304C0FD01AA
:10DB20008291806F80838BE99DE090930F018093B9
:10DB30000E010F90DF91CF911F910F91FF90EF9009
:10DB4000DF90CF90BF90AF909F908F907F906F901D
:10DB5000089580918D0D8F7780938D0D3FCF8091AB
:10DB60008D0D8F7D80938D0D80918D0D57DE809171
:10DB70005B0254DE0AED17E0F12C6DE0D62EF801C1
:10DB8000819191918F01D89E9001D99E300D1124E1
:10DB900055E0359527955A95E1F73E5F37FD07C06B
:10DBA0002F3FF3E03F0734F4E22E832F06C0E12C31
:10DBB00080E003C0EE24EA9483E09F2D990F990F33
:10DBC000892B2CDE8E2D2ADEF39426E0F212D7CF9D
:10DBD0009DCFCF92DF92EF92FF920F931F93CF933F
:10DBE000DF93C0915A02CF708091590685FF04C01F
:10DBF000809147028111C4E080918E0D8111CFEF99
:10DC00008091900D8C1709F468C0C093900D1EBCD4
:10DC10001DBC1CBC87B7837C87BF80917D008E7F35
:10DC200080937D008CE386BF8FE380937C008C2FF4
:10DC300090E08730910508F050C0FC01E055FF4F9F
:10DC40000C94587A64DD4DDC08C161DD88E59BE108
:10DC500099BD88BD80EA9FE0909379008093780019
:10DC600087B7886087BF80917D00816080937D0049
:10DC70001FBC82E08EBD44C04ADD88EC90E09093EA
:10DC80007900809378008CE291E09DBD8CBD80EEA0
:10DC90009BEA97BD86BD87B7806287BF80917D0074
:10DCA000816080937D001FBC8AE18EBD16C0C430A8
:10DCB00021F484E021DCC09803C013DC83E01CDC89
:10DCC00080E593EC909387008093860088E893E149
:10DCD00090938500809384002CDDC23009F4BAC093
:10DCE00038F4CC2309F4B9C0C13009F0B8C008C079
:10DCF000C33009F4B2C0C550C23008F0B0C0AAC0E9
:10DD00007894F0902D0E87B7877F87BF80917D0034
:10DD10008E7F80937D00E2E9FDE08BE99DE09093AA
:10DD20001101809310018CE99DE093838283158219
:10DD30001482108211821682178284E080878FEF0E
:10DD400080939B0DD2DD80915B02AFDD40918F0D02
:10DD500080913C0540FF0CC090E4890290011124A1
:10DD600080915A028695869586958670822B04C08E
:10DD700020E48202C0011124842B97DD80E095DD30
:10DD8000E0905C02E294E694A7E0EA228F2D817095
:10DD9000D82EF0FE02C098E0E90EF8E0CF2ECE0CAF
:10DDA0008E2DAEDD8C01D110185F802F7EDD81E0DD
:10DDB0008E0DA6DDEC01D110D85FE394E3949C2F87
:10DDC0009295907F812F8F70892B6FDDCE01E4E0DB
:10DDD00096958795EA95E1F768DDEC10E1CF80E054
:10DDE00064DDC091960D8091970D5FDD8C2F5DDD18
:10DDF0007CDD8091930D882319F080E0F2DCF9CF6F
:10DE0000E091940DF091950D1082E8E7F0E08081AB
:10DE100091819C012854344F39BD28BD805B994BBA
:10DE200091838083C09A88E086BF81E080937C00E4
:10DE300087B7886087BF80917D00816080937D0077
:10DE400080913C05813011F0F39401C0F12CF092E7
:10DE50002D0E05C078947BDD02C080E04DDBDF91A4
:10DE6000CF911F910F91FF90EF90DF90CF90089589
:10DE70001F920F920FB60F9211242F933F934F933F
:10DE80005F936F937F938F939F93AF93BF93CF9342
:10DE9000DF93EF93FF938CB59DB520912C0E222339
:10DEA00021F0C09A10922C0E04C0C09821E020935B
:10DEB0002C0EC0910C01D0910D01FE0121913191E8
:10DEC0003BBD2ABDF0930D01E0930C01E6E0F1E0CB
:10DED000282F3181381708F481833081231708F403
:10DEE00080838A819B81892BD1F48BE99DE090937B
:10DEF0000D0180930C018091610280958170809367
:10DF00002C0E87B78F7E87BF64DE80915A028F7098
:10DF100011F0833021F487B7806187BF78948091B6
:10DF2000910D81608093910DFF91EF91DF91CF91E1
:10DF3000BF91AF919F918F917F916F915F914F9121
:10DF40003F912F910F900FBE0F901F9018958091C9
:10DF500061028095817080932C0E80932B0E81112D
:10DF600001C0C09A80915A028F70865F8093900D95
:10DF700010928E0D2ECE1F920F920FB60F9211247B
:10DF80002F933F934F935F936F937F938F939F93C1
:10DF9000AF93BF93EF93FF9380915A028F708130BC
:10DFA00011F1863029F0853031F080E492EA05C025
:10DFB00080E89EE302C080E99DE397BD86BD209185
:10DFC0007800309179002F3F310538F4885893411B
:10DFD000909379008093780007C088EC90E090934C
:10DFE000790080937800F5DDFF91EF91BF91AF91BB
:10DFF0009F918F917F916F915F914F913F912F9161
:10E000000F900FBE0F901F9018951F920F920FB692
:10E010000F9211242F933F934F935F936F937F93AE
:10E020008F939F93AF93BF93EF93FF9380915A0287
:10E030008F7078949091900D981769F0943059F4FE
:10E0400080914702882321F08091590685FD02C006
:10E05000C0DD02C084E050DAFF91EF91BF91AF9133
:10E060009F918F917F916F915F914F913F912F91F0
:10E070000F900FBE0F901F9018958091830680FD22
:10E0800005C0809165008B7F809365000895CF93D4
:10E09000DF93EC01F2DF1C821D82188219821EA61A
:10E0A0001FA6DF91CF910895F2CF21E0FC0184817A
:10E0B000811101C020E0822F0895FC01218180811F
:10E0C000281B277098E0921B81E0933008F480E0D1
:10E0D0000895CF93DF93EC018C818823F1F0815078
:10E0E0008C838A819B81890F8A838EA58823D1F1B5
:10E0F0008FA59FEF980F9FA7882351F080918306EB
:10E1000080FD30C0809165008460809365002AC0E6
:10E11000B4DF80915B068FA725C01B98AEDF8D8191
:10E12000882319F081508D831DC0888199818917BA
:10E13000C9F090E0FE01E80FF91F26812A832689A5
:10E140002C8326852B83268D2D8320A92EA71FA601
:10E1500026A13FEF320F36A3211104C0019687702C
:10E1600099278883DF91CF910895EF92FF920F93C3
:10E170001F93CF93DF93EC01F62E142FE22E9DDF39
:10E18000882309F451C08091C60181FD4DC0302F14
:10E190003295369536953370402F4F70333009F4F1
:10E1A0003FEFFF2021F080915A06865FF80E8091A4
:10E1B00050068873803129F48BEA189F112D1124A1
:10E1C00002C0883111F4169509C0883211F4110F7C
:10E1D00005C0803319F4812F880F180F288104FFA0
:10E1E0000DC0FA821C83ED8205FB882780F98EA77B
:10E1F0001FA63B8329834423B9F001C04F5FE98107
:10E20000F0E0CF01019687709927281769F0EC0F8D
:10E21000FD1FF682168BE68E05FB002700F900AB8A
:10E22000415046A336878983DF91CF911F910F918B
:10E23000FF90EF9008950F931F93CF93DF93EC011E
:10E24000062F642F80915006869586958695877057
:10E25000388129813213F0C010E00332110508F033
:10E26000EBC0F801E954FF4F0C94587A00E326C044
:10E2700000E321E0C0C002EA22E04AE064E6DAC03E
:10E280000AE222E045E06FE5CE016FDF01E22AE01D
:10E2900045E06FE5CE0169DF0AE222E045E06FE587
:10E2A000C9C002EC23E04AE060E5CE015EDF02E493
:10E2B00023E04AE06CE3CE0158DF00E221E065C0D4
:10E2C00001E221E045E066E4CE014FDF22E04FE0CD
:10E2D00062E3CE014ADF22E04FE062C002E221E0C9
:10E2E00045E06EE6CE0141DF03E221E045E097C064
:10E2F00000E025E045E062E3CE0137DF25E045E0C0
:10E300006AE5CE0132DF02E024E043E06EE692C02F
:10E3100003E22AE045E060E5CE0127DF01E224E1E7
:10E3200045E060E5CE0121DF03E22AE045E038C0A8
:10E3300002E625E044E16AE07DC002E22AE044E032
:10E3400062E3CE0112DF01E224E148E066E4CE019F
:10E350000CDF02E22AE048E062E3CE0106DF01E2E0
:10E3600024E144E04DC00AE22AE002C002E222E3D6
:10E3700045E04BC001E203C002E201C003E22AE033
:10E3800044E160E057C002E122E04AE039C002E423
:10E3900023E044E16CE3CE01E8DE02EE23E044E159
:10E3A00060E548C000E321E048E22AC0813009F47A
:10E3B00043C000E121E04AE06BE43CC08130E1F180
:10E3C00000E121E04AE061E435C000E121E046E0FF
:10E3D00031C000E3D9CF813079F100E1D5CF00E140
:10E3E00012C003E303C002E301C001E323E04FE0F6
:10E3F0000CC001E329E144E103C000E321E04EE168
:10E4000066E418C001E321E04AE068E713C002E3D4
:10E4100021E04AE06AE70EC003E321E04AE06CE74E
:10E4200009C000E520E04AE062E804C000ED20E019
:10E430004AE062E3CE0199DEDF91CF911F910F9107
:10E44000089546E4682F88EC91E0F5CE462F682FBA
:10E4500088EC91E0F0CE90915C0691FF03C0862F8E
:10E460000C949414EECFCF92DF92EF92FF920F9321
:10E470001F93CF93DF93EC01062F142F47FF03C0A8
:10E48000842F0E949414D7FF06C0D195C195D1095D
:10E490008AE10E949414002369F0023019F464E6C2
:10E4A00070E002C06AE070E0CE01B1D7262FC22F23
:10E4B000D72FF82E64E670E0CE01A9D79B01FB01AF
:10E4C000EC016115710591F16A307105C4F06AE0E3
:10E4D00070E0C9019CD76B017C01653171051CF4AA
:10E4E0008EE68C0D05C08CE88C0D0E9490148EE693
:10E4F0000E949414F701309769F001E001C000E038
:10E5000084E68E0F0E949414011104C0209741F1FB
:10E510008C2F0AC0209721F1CE016AE070E077D7F6
:10E520009E01281B390BC901845713C084570E94D0
:10E5300090140023A9F0023079F46AE070E08F2D86
:10E5400090E065D7C82F86E0860F0E9494148CE86F
:10E550008C0F0E94901404C086E08F0D0E949414CA
:10E5600011161CF4812F0E949414DF91CF911F91FA
:10E570000F91FF90EF90DF90CF900895863050F488
:10E58000E82FF0E0E659F14FCB019F706AE070E0B0
:10E590002AD760830895CF93C82F843091F48AE0FE
:10E5A0009B01829FB001839F700D112480912C0FDD
:10E5B000882309F441C070932B0F60932A0FCBE29C
:10E5C0003BC0873031F580912C0F6A30710510F413
:10E5D000816001C0836080932C0F80912C0F81FF9C
:10E5E00004C0CB016AE070E0FED620912A0F309182
:10E5F0002B0F121613062CF044275527461B570BDA
:10E6000001C0AB01240F351F3093950E2093940E5B
:10E6100013C08F3F31F47093950E6093940EC4E055
:10E620000BC08E3F31F47093970E6093960EC5E049
:10E6300003C08C3208F0ACC080915702EC2FF0E0A0
:10E6400084FD07C0EE0FFF1FE457F14F7183608315
:10E650001AC0C43071F1EE0FFF1FE457F14F718300
:10E660006083C53081F42091960E3091970E4AE078
:10E67000429FC001439F900D11249093950E80936B
:10E68000940EC4E016C0C03291F48091F0048295DB
:10E690008F7090E08617970718F4681B790B02C0FB
:10E6A00060E070E07093CD0E6093CC0E71C0C73007
:10E6B000F8F4E0E7FEE04C2F50E0440F551FDA017C
:10E6C000A457B14F2D913C91E40FF51F4685578516
:10E6D0004217530714F4378726874081518141152B
:10E6E000510519F024173507C4F53183208335C04F
:10E6F000C031D1F4862F82958F7091E0980F2091D0
:10E70000690E291728F4963008F096E09093690E68
:10E710009B012F703327322F2227672F7727260F51
:10E72000371FB901CF912ACFCC30B9F4A091A40EF4
:10E73000B091A50E2CE330E018D62091F3042111FE
:10E7400003C021E02093F30430E040E050E072D6B3
:10E750003093A50E2093A40E1BC0C232C9F4809141
:10E76000CE0E9091CF0E4AE0489F9001499F300D08
:10E770001124260F371F45E1429FC001439F900D92
:10E7800011246BE070E02FD67093D90E6093D80EF1
:10E79000CF9108958A3308F08151803331F0893365
:10E7A00031F08E3228F080E003C087E201C08BE2B6
:10E7B000E82FF0E0E856FF4D8491EDCEE4EEFEE068
:10E7C0009091570293FD32C09081911110C08E3507
:10E7D000D9F581E0808385818823B1F11582648138
:10E7E00070E0762F66278381682B8281D3CF8E35A8
:10E7F00011F481E014C08D3519F481E0818308950E
:10E800002181222319F0118220E68227913019F408
:10E81000828382E004C0923021F4838383E080838A
:10E820000895848381E08583108208959091060F76
:10E83000903510F483830895682F70E0762F662753
:10E840008381682B84E0A7CE08951F920F920FB6A4
:10E850000F9211248F939F93EF93FF93E8E0FFE0D3
:10E860008585882359F081508587868591E0980FAA
:10E870009687E80FF11D80818CB901C05598FF91F2
:10E88000EF919F918F910F900FBE0F901F90189551
:10E890009EE79093080F8093090FEAE0FFE083E87A
:10E8A000860F8230A0F082E06083E1E0E80FF0E0C4
:10E8B000E85FF04F40832183128213821482158215
:10E8C00016829EE79783875F8093150F08956052A5
:10E8D0008DE78083319683E0E7CFFC0181818283DD
:10E8E00010820895CF93DF93EC01842F2B813C811C
:10E8F000260F311D3C832B839091660E911103C02E
:10E9000054E060E102C052E064E09D819F5F961791
:10E9100010F49D8313C01D8202C0359527955A952A
:10E92000E2F729839A81921710F4291B01C020E095
:10E930002883622F70E02FDE1C821B82DF91CF9133
:10E940000895FF920F931F93CF93DF93EC0188817B
:10E95000873F21F148F4863FB9F589818093EC0E19
:10E960008B818093EA0E30C08D3FF9F08E3F61F5C8
:10E9700040E069818EEE9EE0B5DF41E06A8184EF80
:10E980009EE0B0DF42E06B818AEF9EE0ABDF6C81FE
:10E99000669543E080E09FE0A5DF16C08981809303
:10E9A000ED0E8B818093EB0E0FC0198117701D5FE8
:10E9B000239603E03AE5F32E011730F48991FEDE49
:10E9C000F092060F0F5FF8CF83E28093070FDF917D
:10E9D000CF911F910F91FF9008958F929F92AF92C8
:10E9E000BF92CF92DF92EF92FF92CF93E7E1FFE0E9
:10E9F0004181A8E1BFE080E090E02D91BC01620F71
:10EA0000711D872F9927860F971F99277FE0A032C6
:10EA1000B70799F78F3F910509F01CC189E68093EC
:10EA2000070F403109F016C18381813F41F5F48021
:10EA300082818330F1F028F4813069F08230A1F0D6
:10EA400009C1843069F0853009F004C143E06F2DBD
:10EA500080E09FE012C042E06F2D8AEF9EE00DC083
:10EA60006F2D70E088E297DD40E06F2D8EEE9EE026
:10EA700004C041E06F2D84EF9EE034DFEBC08111D4
:10EA800008C08FEF8093060F64817581828182DEDA
:10EA9000E1C09FEF9093060FC480D580E680F78099
:10EAA000228122952F7030E1839FC0011124282BF1
:10EAB000213409F475C0F0F4203209F465C040F443
:10EAC0002031D1F1213109F0C5C0B60187E2C1C0C2
:10EAD0002033E1F1203409F460C0213209F0BAC0DA
:10EAE000C701B6012AE030E040E050E0A3D4B9010C
:10EAF00086E2AFC0233809F4A3C060F4203809F4DB
:10EB00005CC0223809F44FC0203509F0A3C0B6011B
:10EB10008CE09FC02039D9F1213909F43BC0243859
:10EB200009F098C0C701B60124E630E040E050E0AB
:10EB300081D4B90181E18DC0C701B6012AE030E07E
:10EB400040E050E099D4B9018FEF83C08C2D90E064
:10EB500054E0959587955A95E1F78093690ECC2DF1
:10EB6000CF7099278F2D7E2D6D2D8C2F07DDC7013E
:10EB7000B601E4E19695879577956795EA95D1F783
:10EB800081E08C0FFBDC66C0B60180E262C0B6019A
:10EB900089E25FC0B6018AE25CC0B6018AE059C072
:10EBA000B6018BE056C0C701B60124E630E040E074
:10EBB00050E062D4B9018EEF4CC0460157014EE1DE
:10EBC000B694A794979487944A95D1F7C701B60154
:10EBD0009F7320E137E240E050E02CD46B017C01D0
:10EBE000CA01B9012CE330E040E050E023D4A4E6B0
:10EBF000A29FF001A39FF00D1124E60FF71FC82D6F
:10EC0000C170BF0181FE0EC087E1C5DCB60188E19D
:10EC1000C2DCCC2319F067E570E002C065E470E067
:10EC200089E117C08AE1B7DCB6018BE1B4DCCC2303
:10EC300019F063E570E002C06EE470E08CE109C099
:10EC4000C701B60128EE33E040E050E0F3D3B9014C
:10EC500086E0A1DCCF91FF90EF90DF90CF90BF9046
:10EC6000AF909F908F9008951F920F920FB60F92C2
:10EC700011242F933F934F935F936F937F938F93C1
:10EC80009F93AF93BF93CF93EF93FF93579878944D
:10EC90009BB18CB1C0912F0F9C7109F08BC09091EA
:10ECA0002E0F9230C1F030F4992309F43FC0913017
:10ECB00049F081C0943009F44BC048F1953009F413
:10ECC0004FC079C08E3709F476C08B31A1F092E045
:10ECD00090932E0F13C08D3711F483E036C08E371A
:10ECE00069F48091660E882319F090932E0F62C00C
:10ECF00087E19FE026DE10922E0F5DC0C33108F041
:10ED00005AC0EC2FF0E0E95EF04F80830DC092E036
:10ED100090932E0FC33108F04EC0EC2FF0E0E95E67
:10ED2000F04F90E298279083CF5F45C08E3751F423
:10ED30008091660E882311F082E001C081E080930B
:10ED40002E0F38C08B31B9F584E080932E0F33C07D
:10ED500095E090932E0F8093650E1092640E2BC059
:10ED60009091640E91110CC0982F9F7391F494B3FD
:10ED7000906C94BB95B3807C9F73892B85BB09C035
:10ED8000913019F480930E0204C0923011F48093F4
:10ED900013028091640E8F5F8093640E9091650ED4
:10EDA000891309C010922E0F8091630E80688093A2
:10EDB000630E01C0C0E08091660E882331F0C93037
:10EDC00020F00BDE10922E0FC0E0C0932F0FF894AE
:10EDD000579AFF91EF91CF91BF91AF919F918F91F2
:10EDE0007F916F915F914F913F912F910F900FBE47
:10EDF0000F901F9018951092A90E1092A80E1092C5
:10EE0000AB0E1092AA0E1092D30E1092D20E109248
:10EE1000680E1092670E1092D50E1092D40E8CE1EF
:10EE2000E0E7FEE0DF011D928A95E9F70895CF93B0
:10EE3000C82F8093660EDFDF1098189880916D06BA
:10EE400085FD0BC0C11109C080915A028F708530B9
:10EE500011F487E003C087E601C080E189B9109210
:10EE6000900059981AB886E0809395005F9B02C085
:10EE70008CB1FCCF1092150F88EB8AB9CF91089511
:10EE80001F93CF93DF931F92CDB7DEB790915A02B5
:10EE90009F7081E0913009F080E09091660E8913B7
:10EEA000C6DF8091070F882351F081508093070FB0
:10EEB000811107C01092930E1092920E02C080E052
:10EEC00001C081E09091060F992329F0811182E021
:10EED00091509093060F80932D0F2091630E222363
:10EEE00009F44CC08091620E882321F081508093F8
:10EEF000620E44C08091150F811140C091E0392FFE
:10EF0000322321F48F5F990F8830C9F790959223AF
:10EF10009093630E843028F420E040E060E0875056
:10EF200016C0863070F48170282F30E0D901A651C8
:10EF3000B14FF901E451F14F2C9140E060818A50CA
:10EF400006C0863039F420E040E060E081EFA0DCCC
:10EF500085E00FC0873091F4E8E0FFE08BE180832B
:10EF6000838381E081838091660E828384E085873C
:10EF70008AE08093620E1092160F559A10917405D4
:10EF8000112309F477C01330F0F48091070F882320
:10EF900009F445C01150E12FF0E0DF01AA0FBB1FBB
:10EFA000A457B14F2D913C91EE0FFF1FEE0FFF1FA5
:10EFB000E851FB4F4081429FC001439F900D1124B7
:10EFC00064E670E029C0133049F48091060F88236D
:10EFD00031F18091CC0E9091CD0E23C081E2810F52
:10EFE0000E94F8228823D9F0AE014F5F5F4F60E0A6
:10EFF00070E08CEF810F0E947E222981211108C0D0
:10F000002AE0AC01249FC001259F900D112409C066
:10F01000223039F46AE070E0E6D1CB0102C080E032
:10F0200090E097FF02C080E090E02091670E309161
:10F03000680E280F391F21315EE03507BCF02051E2
:10F040003E40E4EDFEE080819181019691838083D2
:10F05000DF019C978D919C91119701968D939C93C4
:10F06000BA97808191810196918380833093680E55
:10F070002093670E0F90DF91CF911F91089510920A
:10F08000690E8091630E8F608093630E089586B33E
:10F0900080958E7708958FEF8ABB1BBA91E897BB56
:10F0A0009EE798BB9EE394BB91EC95BB11BA82BBE3
:10F0B00098E092B997EF93B91092610010926200B4
:10F0C00094E1909364009BEF9093650080938D0D85
:10F0D000D4B714BE80E487B985E886B987E083BFDA
:10F0E0008CE981BF82E085BD83E487BF1FBC8AE0D5
:10F0F0008EBD10928B0082E880938A0080E280931C
:10F100007D00789482E595E490934C0180934B01C7
:10F110000E94645D882319F00E94096706C00E945E
:10F120001E5C0E9409670E94265D91E080B3809575
:10F13000837C813419F49093C601F8CF823849F466
:10F14000F89466E072E088E00E9411640E942B67E8
:10F15000FFCFD0903A068D2D0E94555E98DF982FF4
:10F160009670963031F48091C60182608093C6011A
:10F1700025C0C0E081FD05C08695CF5FC630D1F7C0
:10F180001DC08C2F0E94C05C8823C1F0C0933A063A
:10F190008C2F0E94555E81E00E944A5D0E94DD62D4
:10F1A00024E04EEF51E060E086E10E94EC6388E1EC
:10F1B0000E944C330E942B670E9475120E94ED1032
:10F1C00080916D0686FD0E94896981E080933901F6
:10F1D0000E94651A1092390180916906895F0E9428
:10F1E0009614D3FD76C08091530684FF05C08091AC
:10F1F000500682FD47C03DC080915C06882319F00F
:10F200006CE187E028D90E9441190E94DD6220E06C
:10F2100046E753E060E080E00E94E8628091590692
:10F2200084FD08C000E12AE04EE556E068E380E096
:10F230000E94B6630E942B670E9475120E94661698
:10F240000E9437168C010E949B10EC01C057DE4FC4
:10F250000E942B670E9441190E9466160E94371671
:10F260007C0115DF8111C3CFE016F10609F45DC002
:10F27000BECF0E94AA5F883C910520F48FEE91E0FA
:10F280000E9491190E94661680912101909122019D
:10F290006EE070E0A8D060933D010E94A8190E9422
:10F2A000C31990915006987B21F48FED91E00E9454
:10F2B00091198091C701882331F084EB91E00E947D
:10F2C00091191092C7010E947512809155020E94F7
:10F2D0009014909105019260909305011092EA06B6
:10F2E00060E08AED97E00E94C5470E94A76F8DE01D
:10F2F00028E130E00FB6F894A89521BD0FBE81BD7E
:10F3000023E63AE230934E0120934D0180913A0674
:10F31000D81629F081E00E944A5D0E94465E81E095
:10F32000809348020E940E1CFDCF0E949B10C817BC
:10F33000D90709F08DCF5BCF88EC91E00C94547025
:10F3400005D0332312F48A1B9B0B10C0A29FB0017F
:10F35000B39FC001A39F700D811D1124911DB29F09
:10F36000700D811D1124911D0895F0DFB7FF0895E0
:10F37000821B930B0895EADFA59F900DB49F900D1B
:10F38000A49F800D911D11240895B7FFF4CFF3DFE2
:10F39000821B930B0895DB018F939F93ECDFBF914A
:10F3A000AF91A29F800D911DA39F900DB29F900DD4
:10F3B00011240895991B79E004C0991F961708F04D
:10F3C000961B881F7A95C9F78095089587FB082EAC
:10F3D000062687FD819567FD6195ECDF0EF491951A
:10F3E00007FC81950895AA1BBB1B51E107C0AA1F0A
:10F3F000BB1FA617B70710F0A61BB70B881F991FD6
:10F400005A95A9F780959095BC01CD01089597FB79
:10F41000072E16F4009406D077FD08D0E4DF07FC31
:10F4200005D03EF4909581959F4F08957095619514
:10F430007F4F0895A1E21A2EAA1BBB1BFD010DC030
:10F44000AA1FBB1FEE1FFF1FA217B307E407F50794
:10F4500020F0A21BB30BE40BF50B661F771F881F70
:10F46000991F1A9469F760957095809590959B0106
:10F47000AC01BD01CF010895052E97FB16F4009451
:10F480000FD057FD05D0D6DF07FC02D046F408C0E8
:10F4900050954095309521953F4F4F4F5F4F0895C0
:10F4A00090958095709561957F4F8F4F9F4F0895F0
:10F4B000EE0FFF1F0590F491E02D0994FB01DC0194
:10F4C00002C001900D9241505040D8F7089568173E
:10F4D000790768F4FB01DC01E40FF51FA40FB51FE9
:10F4E00002C002900E9241505040D8F70895E6CFE6
:10F4F000DC0101C06D9341505040E0F70895DC01FC
:10F50000CB01FC01E199FECF06C0FFBBEEBBE09A48
:10F5100031960DB20D9241505040B8F70895F894CD
:02F52000FFCF1B
:10F52200F00064000A02FF000000E30D9B0D9B0D3A
:02F532009B0D2F
:00000001FF
